:020000040800F2
:10000000E0BE0020FD3E000813700308E93E000832
:10001000E93E0008E93E0008E93E0008E93E000824
:10002000000000000000000000000000E93F0008A0
:10003000E93E000800000000813F000835A90008E3
:100040008941000889410008894100088941000868
:100050008941000889410008894100088941000858
:100060008941000889410008894100088941000848
:100070008941000889410008894100088941000838
:100080008941000889410008894100088941000828
:100090008941000889410008894100088941000818
:1000A0008941000889410008894100088941000808
:1000B00089410008894100088941000889410008F8
:1000C00089410008894100088941000889410008E8
:1000D00089410008894100088941000889410008D8
:1000E00089410008894100088941000889410008C8
:1000F00089410008894100088941000889410008B8
:1001000089410008894100088941000889410008A7
:100110008941000889410008894100088941000897
:100120008941000889410008894100088941000887
:100130008941000889410008894100088941000877
:100140008941000889410008894100088941000867
:100150008941000889410008894100088941000857
:100160008941000889410008894100088941000847
:100170008941000889410008894100088941000837
:100180008941000889410008894100088941000827
:100190008941000889410008894100088941000817
:1001A0008941000889410008894100088941000807
:1001B00089410008894100088941000889410008F7
:1001C00089410008894100088941000889410008E7
:1001D00089410008894100088941000889410008D7
:1001E00089410008894100088941000889410008C7
:1001F00089410008894100088941000889410008B7
:1002000089410008894100088941000889410008A6
:100210008941000889410008894100088941000896
:100220008941000889410008894100088941000886
:0402300089410008F8
:1002380081F0004102E000BF83F0004330B54FEA8F
:1002480041044FEA430594EA050F08BF90EA020FFC
:100258001FBF54EA000C55EA020C7FEA645C7FEA8F
:10026800655C00F0E2804FEA5454D4EB5555B8BFB2
:100278006D420CDD2C4480EA020281EA030382EA23
:10028800000083EA010180EA020281EA0303362DB5
:1002980088BF30BD11F0004F4FEA01314FF4801C88
:1002A8004CEA113102D0404261EB410113F0004F9A
:1002B8004FEA03334CEA133302D0524263EB430351
:1002C80094EA050F00F0A780A4F10104D5F1200EEF
:1002D8000DDB02FA0EFC22FA05F2801841F100014A
:1002E80003FA0EF2801843FA05F359410EE0A5F11E
:1002F80020050EF1200E012A03FA0EFC28BF4CF04F
:10030800020C43FA05F3C01851EBE37101F0004504
:1003180007D54FF0000EDCF1000C7EEB00006EEB11
:100328000101B1F5801F1BD3B1F5001F0CD349089B
:100338005FEA30004FEA3C0C04F101044FEA4452F2
:1003480012F5800F80F09A80BCF1004F08BF5FEA79
:10035800500C50F1000041EB045141EA050130BD59
:100368005FEA4C0C404141EB0101013C28BFB1F56B
:10037800801FE9D291F0000F04BF01460020B1FAB6
:1003880081F308BF2033A3F10B03B3F120020CDA89
:100398000C3208DD02F1140CC2F10C0201FA0CF067
:1003A80021FA02F10CE002F11402D8BFC2F1200CCC
:1003B80001FA02F120FA0CFCDCBF41EA0C01904082
:1003C800E41AA2BF01EB0451294330BD6FEA0404CB
:1003D8001F3C1CDA0C340EDC04F11404C4F12002B6
:1003E80020FA04F001FA02F340EA030021FA04F3C8
:1003F80045EA030130BDC4F10C04C4F1200220FA1F
:1004080002F001FA04F340EA0300294630BD21FA5C
:1004180004F0294630BD94F0000F83F4801306BF22
:1004280081F480110134013D4EE77FEA645C18BF16
:100438007FEA655C29D094EA050F08BF90EA020FAD
:1004480005D054EA000C04BF1946104630BD91EAA5
:10045800030F1EBF0021002030BD5FEA545C05D1A8
:100468004000494128BF41F0004130BD14F58004E7
:100478003CBF01F5801130BD01F0004545F0FE415B
:1004880041F470014FF0000030BD7FEA645C1ABF90
:10049800194610467FEA655C1CBF0B46024650EAC7
:1004A800013406BF52EA033591EA030F41F40021F3
:1004B80030BD00BF90F0000F04BF0021704730B579
:1004C8004FF4806404F132044FF000054FF000014E
:1004D80050E700BF90F0000F04BF0021704730B50F
:1004E8004FF4806404F1320410F0004548BF4042E4
:1004F8004FF000013EE700BF42004FEAE2014FEA39
:1005080031014FEA02701FBF12F07F4393F07F4F13
:1005180081F06051704732F07F4208BF704793F016
:100528007F4F04BF41F40021704730B54FF4607429
:1005380001F0004521F000411CE700BF50EA01022C
:1005480008BF704730B54FF000050AE050EA0102D5
:1005580008BF704730B511F0004502D5404261EB45
:1005680041014FF4806404F132045FEA915C3FF486
:10057800D8AE4FF003025FEADC0C18BF03325FEA23
:10058800DC0C18BF033202EBDC02C2F1200300FAD4
:1005980003FC20FA02F001FA03FE40EA0E0021FAF9
:1005A80002F11444BDE600BF70B54FF0FF0C4CF4E7
:1005B800E06C1CEA11541DBF1CEA135594EA0C0F99
:1005C80095EA0C0F00F0DEF82C4481EA030621EAD4
:1005D8004C5123EA4C5350EA013518BF52EA03350F
:1005E80041F4801143F4801338D0A0FB02CE4FF0C1
:1005F8000005E1FB02E506F00042E0FB03E54FF0F1
:100608000006E1FB03569CF0000F18BF4EF0010EE8
:10061800A4F1FF04B6F5007F64F5407404D25FEAE4
:100628004E0E6D4146EB060642EAC62141EA555197
:100638004FEAC52040EA5E504FEACE2EB4F1FD0CD9
:1006480088BFBCF5E06F1ED8BEF1004F08BF5FEA57
:10065800500E50F1000041EB045170BD06F0004609
:1006680046EA010140EA020081EA0301B4EB5C04B6
:10067800C2BFD4EB0C0541EA045170BD41F48011AE
:100688004FF0000E013C00F3AB8014F1360FDEBFD3
:10069800002001F0004170BDC4F10004203C35DAAF
:1006A8000C341BDC04F11404C4F1200500FA05F332
:1006B80020FA04F001FA05F240EA020001F00042D3
:1006C80021F0004110EBD37021FA04F642EB060149
:1006D8005EEA430E08BF20EAD37070BDC4F10C0473
:1006E800C4F1200500FA04F320FA05F001FA04F237
:1006F80040EA020001F0004110EBD37041F1000123
:100708005EEA430E08BF20EAD37070BDC4F120052D
:1007180000FA05F24EEA020E20FA04F301FA05F295
:1007280043EA020321FA04F001F0004121FA04F23D
:1007380020EA020000EBD3705EEA430E08BF20EA0D
:10074800D37070BD94F0000F0FD101F00046400047
:1007580041EB010111F4801F08BF013CF7D041EAC9
:10076800060195F0000F18BF704703F000465200CD
:1007780043EB030313F4801F08BF013DF7D043EA9E
:100788000603704794EA0C0F0CEA135518BF95EA54
:100798000C0F0CD050EA410618BF52EA4306D1D1DB
:1007A80081EA030101F000414FF0000070BD50EAFA
:1007B800410606BF1046194652EA430619D094EA84
:1007C8000C0F02D150EA013613D195EA0C0F05D16E
:1007D80052EA03361CBF104619460AD181EA0301C2
:1007E80001F0004141F0FE4141F470014FF000007A
:1007F80070BD41F0FE4141F4780170BD70B54FF015
:10080800FF0C4CF4E06C1CEA11541DBF1CEA135594
:1008180094EA0C0F95EA0C0F00F0A7F8A4EB050476
:1008280081EA030E52EA03354FEA013100F088806D
:100838004FEA03334FF0805545EA131343EA126336
:100848004FEA022245EA111545EA10654FEA0026EB
:100858000EF000419D4208BF964244F1FD0404F5A4
:10086800407402D25B084FEA3202B61A65EB030500
:100878005B084FEA32024FF480104FF4002CB6EBBD
:10088800020E75EB030E22BFB61A754640EA0C003D
:100898005B084FEA3202B6EB020E75EB030E22BF7D
:1008A800B61A754640EA5C005B084FEA3202B6EBBE
:1008B800020E75EB030E22BFB61A754640EA9C007D
:1008C8005B084FEA3202B6EB020E75EB030E22BF4D
:1008D800B61A754640EADC0055EA060E18D04FEA0B
:1008E800051545EA16754FEA06164FEAC30343EAAB
:1008F80052734FEAC2025FEA1C1CC0D111F4801F78
:100908000BD141EA00014FF000004FF0004CB6E770
:1009180011F4801F04BF01430020B4F1FD0C88BF0F
:10092800BCF5E06F3FF6AFAEB5EB030C04BFB6EB1A
:10093800020C5FEA500C50F1000041EB045170BD0D
:100948000EF0004E4EEA113114EB5C04C2BFD4EB3A
:100958000C0541EA045170BD41F480114FF0000EBE
:10096800013C90E645EA060E8DE60CEA135594EA3A
:100978000C0F08BF95EA0C0F3FF43BAF94EA0C0F3D
:100988000AD150EA01347FF434AF95EA0C0F7FF4B2
:1009980025AF104619462CE795EA0C0F06D152EA06
:1009A80003353FF4FDAE1046194622E750EA4106EA
:1009B80018BF52EA43067FF4C5AE50EA41047FF4FB
:1009C8000DAF52EA43057FF4EBAE12E74FF0FF3C60
:1009D80006E000BF4FF0010C02E000BF4FF0010C31
:1009E8004DF804CD4FEA410C7FEA6C5C4FEA430CAA
:1009F80018BF7FEA6C5C1BD001B050EA410C0CBFF9
:100A080052EA430C91EA030F02BF90EA020F00205A
:100A1800704710F1000F91EA030F58BF994208BFC1
:100A280090422CBFD8176FEAE37040F0010070477E
:100A38004FEA410C7FEA6C5C02D150EA013C07D1D5
:100A48004FEA430C7FEA6C5CD6D152EA033CD3D020
:100A58005DF8040B704700BF8446104662468C461A
:100A68001946634600E000BF01B5FFF7B7FF00284D
:100A780048BF10F1000F01BD4DF808EDFFF7F4FF76
:100A88000CBF012000205DF808FB00BF4DF808ED01
:100A9800FFF7EAFF34BF012000205DF808FB00BF24
:100AA8004DF808EDFFF7E0FF94BF012000205DF846
:100AB80008FB00BF4DF808EDFFF7CEFF94BF0120FB
:100AC80000205DF808FB00BF4DF808EDFFF7C4FFF4
:100AD80034BF012000205DF808FB00BF4FEA410247
:100AE80012F5001215D211D56FF47873B3EB625278
:100AF80012D94FEAC12343F0004343EA505311F09F
:100B0800004F23FA02F018BF404270474FF0000030
:100B1800704750EA013005D111F0004008BF6FF06E
:100B2800004070474FF00000704700BF4FEA410295
:100B3800B2F1E04324BFB3F5001CDCF1FE5C0DD933
:100B480001F0004C4FEAC0024CEA5070B2F1004F7D
:100B580040EB830008BF20F00100704711F0804F80
:100B680021D113F13872BCBF01F00040704741F445
:100B780080114FEA5252C2F11802C2F1200C10FA49
:100B88000CF320FA02F018BF40F001004FEAC1232D
:100B98004FEAD32303FA0CFC40EA0C0023FA02F3D1
:100BA8004FEA4303CCE77FEA625307D150EA0133A7
:100BB8001EBF4FF0FE4040F44000704701F0004077
:100BC80040F0FE4040F40000704700BF80F0004055
:100BD80002E000BF81F0004142001FBF5FEA41030D
:100BE80092EA030F7FEA226C7FEA236C6AD04FEA0D
:100BF8001262D2EB1363C1BFD21841404840414052
:100C0800B8BF5B42192B88BF704710F0004F40F403
:100C1800000020F07F4018BF404211F0004F41F41F
:100C2800000121F07F4118BF494292EA030F3FD0EB
:100C3800A2F1010241FA03FC10EB0C00C3F12003FE
:100C480001FA03F100F0004302D5494260EB40008D
:100C5800B0F5000F13D3B0F1807F06D340084FEAF8
:100C6800310102F10102FE2A51D2B1F1004F40EBED
:100C7800C25008BF20F0010040EA03007047490055
:100C880040EB0000013A28BFB0F5000FEDD2B0FAF2
:100C980080FCACF1080CB2EB0C0200FA0CF0AABF15
:100CA80000EBC25052421843BCBFD04018437047B3
:100CB80092F0000F81F4000106BF80F400000132B9
:100CC800013BB5E74FEA41037FEA226C18BF7FEA90
:100CD800236C21D092EA030F04D092F0000F08BFD2
:100CE8000846704790EA010F1CBF0020704712F0B9
:100CF8007F4F04D1400028BF40F00040704712F1F8
:100D080000723CBF00F50000704700F0004343F05C
:100D1800FE4040F4000070477FEA226216BF084692
:100D28007FEA23630146420206BF5FEA412390EA55
:100D3800010F40F4800070474FF0000304E000BF4B
:100D480010F0004348BF40425FEA000C08BF7047FC
:100D580043F0964301464FF000001CE050EA0102C0
:100D680008BF70474FF000030AE000BF50EA0102D5
:100D780008BF704711F0004302D5404261EB4101C2
:100D88005FEA010C02BF84460146002043F0B643E7
:100D980008BFA3F18053A3F50003BCFA8CF2083A0C
:100DA800A3EBC25310DB01FA02FC634400FA02FC15
:100DB800C2F12002BCF1004F20FA02F243EB02001C
:100DC80008BF20F00100704702F1200201FA02FC7E
:100DD800C2F1200250EA4C0021FA02F243EB020071
:100DE80008BF20EADC7070474FF0FF0C1CEAD052B5
:100DF8001EBF1CEAD15392EA0C0F93EA0C0F6FD076
:100E08001A4480EA010C400218BF5FEA41211ED053
:100E18004FF0006343EA501043EA5111A0FB01313F
:100E28000CF00040B1F5000F3EBF490041EAD37114
:100E38005B0040EA010062F17F02FD2A1DD8B3F190
:100E4800004F40EBC25008BF20F00100704790F0FF
:100E5800000F0CF0004C08BF49024CEA502040EA51
:100E680051207F3AC2BFD2F1FF0340EAC250704717
:100E780040F400004FF00003013A5DDC12F1190F55
:100E8800DCBF00F000407047C2F10002410021FAC7
:100E980002F1C2F1200200FA02FC5FEA310040F1DF
:100EA800000053EA4C0308BF20EADC70704792F058
:100EB800000F00F0004C02BF400010F4000F013A90
:100EC800F9D040EA0C0093F0000F01F0004C02BF8B
:100ED800490011F4000F013BF9D041EA0C018FE7FA
:100EE8000CEAD15392EA0C0F18BF93EA0C0F0AD000
:100EF80030F0004C18BF31F0004CD8D180EA010026
:100F080000F00040704790F0000F17BF90F0004FBE
:100F1800084691F0000F91F0004F14D092EA0C0FA0
:100F280001D142020FD193EA0C0F03D14B0218BF33
:100F3800084608D180EA010000F0004040F0FE4079
:100F480040F40000704740F0FE4040F44000704715
:100F58004FF0FF0C1CEAD0521EBF1CEAD15392EA94
:100F68000C0F93EA0C0F69D0A2EB030280EA010C84
:100F780049024FEA402037D04FF0805343EA11111D
:100F880043EA10130CF000408B4238BF5B0042F17B
:100F98007D024FF4000C8B4224BF5B1A40EA0C0020
:100FA800B3EB510F24BFA3EB510340EA5C00B3EB52
:100FB800910F24BFA3EB910340EA9C00B3EBD10F40
:100FC80024BFA3EBD10340EADC001B0118BF5FEA92
:100FD8001C1CE0D1FD2A3FF650AF8B4240EBC250BB
:100FE80008BF20F0010070470CF0004C4CEA50207C
:100FF8007F32C2BFD2F1FF0340EAC250704740F4CB
:1010080000004FF00003013A37E792F0000F00F0BC
:10101800004C02BF400010F4000F013AF9D040EA3A
:101028000C0093F0000F01F0004C02BF490011F4CE
:10103800000F013BF9D041EA0C0195E70CEAD153C6
:1010480092EA0C0F08D142027FF47DAF93EA0C0FAD
:101058007FF470AF084676E793EA0C0F04D14B0291
:101068003FF44CAF08466EE730F0004C18BF31F043
:10107800004CCAD130F000427FF45CAF31F000433D
:101088007FF43CAF5FE700BF4FF0FF3C06E000BFD6
:101098004FF0010C02E000BF4FF0010C4DF804CDF9
:1010A8004FEA40024FEA41037FEA226C18BF7FEA09
:1010B800236C11D001B052EA530C18BF90EA010F0B
:1010C80058BFB2EB030088BFC81738BF6FEAE1709A
:1010D80018BF40F0010070477FEA226C02D15FEA36
:1010E800402C05D17FEA236CE4D15FEA412CE1D0A2
:1010F8005DF8040B704700BF844608466146FFE769
:101108000FB5FFF7C9FF002848BF10F1000F0FBD4A
:101118004DF808EDFFF7F4FF0CBF012000205DF843
:1011280008FB00BF4DF808EDFFF7EAFF34BF0120C8
:1011380000205DF808FB00BF4DF808EDFFF7E0FF61
:1011480094BF012000205DF808FB00BF4DF808EDB2
:10115800FFF7D2FF94BF012000205DF808FB00BF15
:101168004DF808EDFFF7C8FF34BF012000205DF8F7
:1011780008FB00BF4FEA40024FEA41037FEA226CB6
:1011880002D15FEA402C08D17FEA236C02D15FEAE2
:10119800412C02D14FF0000070474FF0010070471A
:1011A8004FEA4002B2F1FE4F0FD34FF09E03B3EB6C
:1011B80012620DD94FEA002343F0004310F0004FAC
:1011C80023FA02F018BF404270474FF00000704702
:1011D80012F1610F01D1420205D110F0004008BFA1
:1011E8006FF0004070474FF00000704742000ED289
:1011F800B2F1FE4F0BD34FF09E03B3EB126209D44A
:101208004FEA002343F0004323FA02F070474FF0FF
:101218000000704712F1610F01D1420202D14FF074
:10122800FF3070474FF00000704700BF7BB972B9BC
:101238000029BEBF00204FF0004106E008BF00288B
:101248001CBF6FF000414FF0FF3000F077B8ADF1F0
:10125800080C6DE904CE002909DB002B1ADB00F02D
:10126800A9F8DDF804E0DDE9022304B07047404244
:1012780061EB4101002B1BDB00F09CF8DDF804E07A
:10128800DDE9022304B0404261EB4101524263EBC5
:1012980043037047524263EB430300F08BF8DDF8D9
:1012A80004E0DDE9022304B0404261EB41017047EC
:1012B800524263EB430300F07DF8DDF804E0DDE91A
:1012C800022304B0524263EB4303704753B94AB94F
:1012D800002908BF00281CBF4FF0FF314FF0FF3036
:1012E80000F02CB8ADF1080C6DE904CE00F062F8FE
:1012F800DDF804E0DDE9022304B07047D0B5FFF75C
:10130800FBF800220B4B06460F46FFF74DF900F09D
:1013180017F80446FFF7CEF80022074BFFF744F909
:1013280002460B4630463946FEF786FF00F008F8BD
:101338002146D0BD0000F03D0000F041704700BFDD
:101348004A0011D212F5001211D20DD56FF478733C
:10135800B3EB62520ED44FEAC12343F0004343EA91
:10136800505323FA02F070474FF00000704750EADC
:10137800013002D14FF0FF3070474FF00000704746
:1013880010F8012B11F8013B012A28BF9A42F7D027
:10139800D01A7047034611F8012B03F8012B002AD5
:1013A800F9D17047034613F8012B002AFBD1181A0C
:1013B800013870472DE9F04786468C460846089E56
:1013C800154674461946002B40F0C1808542B2FA92
:1013D80082F245D94AB1C2F1200300FA02FC9540D5
:1013E80094402EFA03F343EA0C0C4FEA154EA8B2C8
:1013F800230CBCFBFEF80EFB18CC08FB00F943EAF3
:101408000C43994528D9EB1808F1FF3704D29945C0
:1014180002D9A8F102072B44A3EB0903A4B2B3FB3A
:10142800FEFC0EFB1C330CFB00F044EA0344A04214
:1014380014D92C190CF1FF3304D2A04202D9ACF113
:1014480002032C44241A43EA07401EB1D440002367
:1014580034607360BDE8F0874746DDE76346F1E72F
:1014680092BB431B01214FEA154EAFB2200CB3FBD0
:10147800FEFC0EFB1C330CFB07F840EA03439845BF
:1014880061D9EB180CF1FF3004D2984502D9ACF1C0
:1014980002002B44A3EB0803A4B2B3FBFEFC0EFB33
:1014A8001C330CFB07F744EA0344A7424DD92C1917
:1014B8000CF1FF3304D2A74202D9ACF102032C4449
:1014C800E41B43EA0040C0E7C2F120039540944082
:1014D80020FA03F12EFA03F34FEA154E9040AFB20B
:1014E8000343B1FBFEFC0EFB1C10190C0CFB07F8A8
:1014F80041EA0041884522D969180CF1FF3004D22D
:10150800884502D9ACF102002944A1EB08019BB23D
:10151800B1FBFEFC0EFB1C110CFB07F743EA014371
:101528009F420ED9EB180CF1FF3104D29F4202D929
:10153800ACF102012B44DB1B41EA004193E7604612
:10154800E3E76146F7E76046A4E76346B8E7834206
:1015580006D916B9002108467CE7C6E900E0F9E794
:10156800B3FA83F78FB9834201D3724508D8BEEB2B
:10157800020460EB030301209C461EB9002169E7C1
:101588003846FAE7C6E9004CF8E7C7F1200CBB403B
:101598000EFA07F522FA0CF42EFA0CF1BA401C43A5
:1015A80020FA0CF3B8404FEA144901431FFA84FEAD
:1015B800B3FBF9F809FB18300B0C08FB0EFA43EAE9
:1015C80000439A4540D9E31808F1FF3004D29A4500
:1015D80002D9A8F102002344A3EB0A0389B2B3FBA2
:1015E800F9F809FB183308FB0EFE41EA03418E4562
:1015F8002CD9611808F1FF3304D28E4502D9A8F11D
:101608000203214443EA0040A1EB0E01A0FB02982B
:101618004145CE46434602D306D14D4504D2013852
:10162800B9EB020E68EB0403002EA7D0B5EB0E024F
:1016380061EB030101FA0CFC22FA07F3F9404CEACA
:101648000303C6E9003199E74046C5E74346D9E7B1
:101658002DE9F04390F8A53004460D4685B023B92E
:101668004FF07E50FFF7B6FA0546D4F884202E4B8B
:101678009A4212D12846FEF73FFF29A3D3E9002357
:10168800FFF722FA011E18BF012104F184000FF0B0
:10169800E7FB0120C4F8985005E0B4F89C30B3F596
:1016A800807F03D1002005B0BDE8F08304F1500924
:1016B800484627F0F3FF0028F4D01C492846FFF7D6
:1016C80093FBFFF793FD94F88080C3B294F89C6075
:1016D800276E206DB8F1000F0DD08DF80D30022364
:1016E8000122002100938DF80C6003ABB8474846EF
:1016F80044F05CF9CDE78DF80B600126414632468F
:101708008DF80C3000960DF10B03B8470096424651
:101718003146276E206D03ABE8E700BFAFF30080CA
:10172800AE47E17A14AEEF3FD848050800007F4382
:101738002DE9F04F044685B008466160062115463C
:1017480098469DF838709DF83CA01BF0B1F9A06050
:10175800067C16F0010602D07F4812F0FFFE9DF8C5
:10176800403008FB05F084F82A309DF844307D307D
:1017780084F828307E2390FBF3F0C0010430C4E9DC
:101788000458277360623DF048FD0622C4E9070645
:1017980072492046A66149F0D8F90222204602A9DA
:1017A800ADF8085049F0D1F90222204602A9ADF857
:1017B800088049F0CAF9F623032269462046ADF8A5
:1017C80000308DF8026049F0C0F97B1EDBB2082BAF
:1017D80005D840F25515DD4015F0010501D16048E6
:1017E800BBE7052F09D0072F06D0032F7AD1012395
:1017F80084F82930002502E02E4684F829604FF04D
:1018080000080026574F4FEA6810C0EB0020FEF78B
:1018180061FE0022544BFEF711FD32463B46FEF7AF
:10182800EDFFFFF75BF95FFA80FBC8F38200C0EBBE
:101838000020FEF74FFE00224C4BFEF7FFFC002273
:101848004B4BFEF7DBFFFFF749F95FFA80F908F029
:101858000300C0EB0020FEF73DFE0022424BFEF7DE
:10186800EDFC32463B46FEF7C9FFFFF737F9C0B239
:10187800002D61D08DF808008DF809B08DF80A9018
:101888000322204602A908F1010849F05EF9B8F1DF
:10189800800FB8D1BAF1000F1BD0364D20462A88E8
:1018A800AB78ADF8042001A903228DF8063049F081
:1018B8004CF90B222046304949F047F9D5F8030086
:1018C800EB7902900522204602A98DF80C3049F0E8
:1018D8003CF9204649F027F9A06949F048F905B0D4
:1018E800BDE8F08F092F84F8296083D10FF25809D9
:1018F800D9E90089354616A7D7E900672846FEF7D3
:10190800E9FD42464B46FEF799FC32463B46FEF758
:1019180075FFFFF7E3F8C0B28DF808008DF80900ED
:101928008DF80A000322204602A9FF3549F00DF977
:10193800B5F5FF4FE2D1ADE78DF808B08DF8099005
:101948008DF80A009CE700BF0000000000C04F406F
:101958000000000000C05F406FE205083FF705087F
:10196800CEDC0508000008400000F83F00000C40ED
:1019780000001C4097CF040846F705080000000047
:1019880030F0004201462DE9F84F034604D101200A
:10199800BDE8F84F33F036BD002803DABDE8F84F4C
:1019A80033F038BDB0F1FF4F03DBFFF715F9BDE8A1
:1019B800F88FB0F5000F35DA4FF09841FFF714FAB9
:1019C8006FF018020346C3F31604DE15764B4FF08A
:1019D8007E517F3E2344164403F4000006EBD356A1
:1019E80080F07E502043FFF7F5F804F10F026F4BAB
:1019F80005461340002B3ED10021FFF789FB98B123
:101A0800002E00F0C8803046FFF79AF9684905466D
:101A1800FFF7EAF9044667492846FFF7E5F9014662
:101A28002046C2E70022CEE75DA1D1E90001FFF719
:101A38007DF82946FFF7D8F901464FF07C50FFF7AB
:101A4800C9F8044629462846FFF7CEF9014620463C
:101A5800FFF7CAF904460EB921466FE03046FFF792
:101A68006FF907465249FFF7BFF95249064638460B
:101A7800FFF7BAF972E04FF08041DFF83CB1FFF7A9
:101A8800ABF801462846A344FFF762FA8146304680
:101A9800FFF756F9494680464846FFF7A5F901463B
:101AA8008246FFF7A1F945490746FFF79DF94449E2
:101AB800FFF792F83946FFF797F94249FFF78CF894
:101AC8003946FFF791F94049FFF786F85146FFF785
:101AD8008BF93E4982463846FFF786F93C49FFF7BD
:101AE8007BF83946FFF780F93A49FFF775F8394628
:101AF800FFF77AF901465046FFF76EF8C4F5571319
:101B0800074603F5227343EA0B03002B30DD4FF041
:101B18007C512846FFF768F92946FFF765F9014621
:101B280004463846FFF758F84946FFF75DF9074677
:101B380046B901462046FFF74DF801462846FFF70B
:101B480049F834E71A494046FFF74EF9194906465D
:101B58004046FFF749F93946FFF73EF80146204667
:101B6800FFF738F82946FFF735F801463046E6E72B
:101B780001462846FFF72EF84946FFF735F904468F
:101B8800002E3FF469AF0A494046FFF72DF909498D
:101B9800064640466CE7002009E700BFAFF3008027
:101BA800555555555555D53F20FB4A00F0FF7F0048
:101BB8008071313FD1F71737305CCFFF9788173ED8
:101BC80025333A3E2549923EABAA2A3F4FD01C3EC8
:101BD800298E633ECDCCCC3E31F000432DE9F04F49
:101BE800804687B00F4681460C460ED180F48009A6
:101BF8004FEA490919F5000F40F266823946404616
:101C0800FEF7EAFF07B0BDE8F08F20F00046B6F116
:101C1800FF4F02D8B3F1FF4F08D9B9F17E5FEDD17C
:101C280084F48004640014F5000FE5E700283246C8
:101C38003DDAB3F1974F1BD3B3F1FF4F3AD00225EA
:101C4800B4F17C5F4DD1B9F1000F80F29780B6F105
:101C5800FF4F28F0004040F04F82A6F17E562E43F9
:101C680040F0A080404607B0BDE8F04F33F0D2BB4B
:101C7800B3F17E5F2ED3D915C1F1960143FA01F570
:101C880005FA01F18B423BD1B3F17E5F4AD1002CBA
:101C980080F2938000214046FFF73AFA00284FD09F
:101CA8004FEAD97007B0BDE8F04F33F0ABBBB3F1E2
:101CB800FF4F3CD1B6F17E5F00F0068204D9002CBC
:101CC800C0F2058238469DE7002C80F2008207F1B9
:101CD800004097E7B1F1804F38D0B1F17C5F53D025
:101CE800002529F0404128F00040B1F17E5F3BD14A
:101CF800002C32DA01464FF07E50FFF729F92CE02C
:101D0800B3F17E5FC3D00025B4F1804FE9D1B6F1BD
:101D1800BF4F1DD2B6F1D05F24D941464046FFF7E8
:101D280063F86FE705F00105C5F10205ECE7B3F1CB
:101D38007E5FACD0B1F1804F4FF00005E7D07FE770
:101D480041464FF07E50FFF703F95BE70025DEE7D9
:101D5800B6F1FF4F28F0004031D1B9F1000FBFF6BE
:101D680051AF7AE728F000404EBB002C22DAB9F1D7
:101D7800000F1DDA6B1E5842584193E7404607B0E2
:101D8800BDE8F04F4AF05DBDB6F1FF4F20F00040CE
:101D98003FF438AFB6F17E5F3FF464AF002E3FF4F6
:101DA80031AF5FE7012D7FF42DAF00F1004029E747
:101DB800304677E7012D7FF425AF404622E74FEA0A
:101DC800D9710139029129433FF44CAFB3F19A4FCD
:101DD80040F29F81604B9E4207D8002C0ADA00200F
:101DE80007B0BDE8F04F33F005BB5C4B9E4207D906
:101DF800002CF4DC002007B0BDE8F04F4AF083BDAA
:101E08004FF07E51FEF7E6FE06465549FEF7ECFF19
:101E1800544980463046FEF7E7FF81464CA1D1E998
:101E28000001FEF783FE82464FF07A513046FEF7F6
:101E3800DBFF01465046FEF7CDFE3146FEF7D4FFE4
:101E480001464FF07C50FEF7C5FE824631463046CB
:101E5800FEF7CAFF01465046FEF7C6FF4249FEF7A5
:101E6800C3FF01464846FEF7B5FE01460646404612
:101E7800FEF7B2FE20F47F6B41462BF00F0B58465D
:101E8800FEF7A8FE24F47F6401463046FEF7A2FE62
:101E9800013D029B24F00F04064638461D432146A7
:101EA80014BF4FF07E55314DFEF794FE5946FEF7AC
:101EB8009BFF804639463046FEF796FF014640466E
:101EC800FEF78AFE064621465846FEF78DFF014674
:101ED80007463046FEF780FE00280446804620F07C
:101EE800004320DDB3F1864F0BD900212846FFF7C8
:101EF80019F9003818BF012072E7002114E1012206
:101F080027E139D11A493046FEF766FE814639463F
:101F18002046FEF75FFE01464846FFF721F90028F4
:101F2800E3D186232DE0134A934207D9002128469E
:101F3800FFF7F8F8003818BF01205CE71CD13946D4
:101F4800FEF748FE3146FFF701F90028E9D0EDE732
:101F5800E13D55555555D53FF3FF7F3F0700803F7D
:101F680000AAB83F70A5EC363BAAB83F000080BF76
:101F78003CAA383300001643B3F17C5F40F2A080DE
:101F8800DB157E3B4FF400045249B8F1000F44FAC8
:101F980003F438464444C4F3C753A3F17F0341FA1A
:101FA80003F1C3F1170301EA0401C4F3160444F46E
:101FB800000444FA03F4B8BF6442FEF70BFE074678
:101FC80031463846FEF708FE20F47F68424928F07B
:101FD8000F084046FEF708FF394681464046FEF79F
:101FE800F9FD01463046FEF7F5FD3C49FEF7FCFEDB
:101FF80006463B494046FEF7F7FE01463046FEF7E7
:10200800EBFD074601464846FEF7E6FD494606460B
:10201800FEF7E0FD01463846FEF7DCFD3146804616
:102028003046FEF7E1FE2F490746FEF7DDFE2E4952
:10203800FEF7D0FD3946FEF7D7FE2C49FEF7CCFD5A
:102048003946FEF7D1FE2A49FEF7C4FD3946FEF7A8
:10205800CBFE2849FEF7C0FD3946FEF7C5FE01460E
:102068003046FEF7B7FD074601463046FEF7BCFE90
:1020780081464FF080413846FEF7ACFD01464846A0
:10208800FEF766FF414607463046FEF7ADFE41467D
:10209800FEF7A2FD01463846FEF79CFD3146FEF7E5
:1020A80099FD01464FF07E50FEF794FD00EBC453B6
:1020B800B3F5000F06DA214633F03EF929462EE63D
:1020C80000247DE71846F9E74FF07E509AE5002096
:1020D80098E500BF000080FF0072313F1872313F61
:1020E8008CBEBF354CBB31330EEADD3555B38A386B
:1020F800610B363BABAA2A3EB6F17E5F3FF4ADAD2D
:10210800002E3FF457AE002D3FF4ACAD002302255E
:10211800029319F0FF4F7FF4F0AE4FF09741FEF7AE
:1021280063FE6FF017010246D315C2F316027F3B18
:1021380042F07E560B4403937E4B9A4208DD7E4B59
:102148009A427FF7DCAE039BA6F5000601330393A2
:1021580000227A4B30460492B24653F822B05946D0
:10216800FEF738FD314681465846FEF735FD0146F3
:102178004FF07E50FEF7ECFE014605904846FEF70C
:1021880033FE6F49019001EA6606019B049A46F006
:10219800005623F47F6806F5800628F00F0806EB42
:1021A800425641463046FEF71FFE01464846FEF7B6
:1021B80011FD594681463046FEF70CFD0146504652
:1021C800FEF708FD4146FEF70FFE01464846FEF7BA
:1021D80001FD059B1946FEF707FE0199834608464F
:1021E800FEF702FE57490646FEF7FEFD5649FEF782
:1021F800F3FC3146FEF7F8FD5449FEF7EDFC314695
:10220800FEF7F2FD5249FEF7E7FC3146FEF7ECFD1A
:102218005049FEF7E1FC3146FEF7E6FD4E49FEF770
:10222800DBFC814631463046FEF7DEFD0146484676
:10223800FEF7DAFD414606460198FEF7CDFC594601
:10224800FEF7D2FD3146FEF7C7FC414681464046BF
:10225800FEF7CAFD41498246FEF7BEFC4946FEF735
:10226800BBFC20F47F66414626F00F063046FEF799
:10227800BBFD3A4980463046FEF7ACFC5146FEF7B6
:10228800A9FC01464846FEF7A5FC0199FEF7ACFDFE
:10229800814631465846FEF7A7FD01464846FEF7F7
:1022A8009BFC824601464046FEF796FC20F47F667A
:1022B8002B4926F00F063046FEF796FD414681462B
:1022C8003046FEF787FC01465046FEF783FC254959
:1022D800FEF78AFD804624493046FEF785FD014613
:1022E8004046FEF779FC049A204B019253F82210DD
:1022F800FEF772FC06460398FEF722FD1C4B019A76
:1023080080463146484653F822A0FEF765FC514600
:10231800FEF762FC4146FEF75FFC20F47F6B414606
:102328002BF00F0B5846FEF755FC5146FEF752FCB2
:102338004946A5E571C41C00D6B35D00CC710508FB
:1023480000F0FFDF42F1533E55326C3E05A38B3E51
:10235800ABAAAA3EB76DDB3E9A99193F00004040F0
:102368000040763F4F38763FC623F6B8BC71050863
:10237800C47105082DE9F04F91B0009302F00403F1
:102388000293C2F3C2030133840705460E46DDF803
:1023980068800392059340F0BB81041D30B1072982
:1023A80009D86FF01B0011B0BDE8F08F01F00706E7
:1023B8003444C6F10806009B4FF000094FF0040AA8
:1023C800591E4FF0FF334F460193CB465346CDF885
:1023D80010900DB1009A22600598002800F3E8805B
:1023E8009848009A824203D397488242C0F0E0801E
:1023F800039AA4EB050E92074FEA9E0000F10381B1
:102408000F2F00F2B180002D00F0058107F1400286
:102418000DEB020C019A0CF8200C0CF8102C049807
:1024280001300490E7E07A285DD84B280ED8472879
:1024380059D829282DD8252852D054D820287AD0E0
:102448002338D0F1000B4BEB000B74E04C382E28EE
:1024580049D8DFE800F070484848484848484848A4
:1024680048484B484848484848484859484B4B59B9
:102478005959704B6D487048184B184848827F4B23
:1024880048484B487F0000204FF0000B4FF0040AEB
:1024980038E001222A38C0B202FA00F010EA0E0F22
:1024A80049D110F0625C2FD110EA020B43D060468C
:1024B800013C5444B4FBFAF40AFB04F4002D61D047
:1024C800A3EB050CA444B4453FF66BAF002868D1D4
:1024D800042B47D158F8043B2360042304342AE032
:1024E800019A013A01924FF0000B24E011F8010C17
:1024F8006C2834D1002011F8023C83466C2BC5D1DE
:102508004FF0080A5346D3E708F1070828F00708F0
:10251800073424F00704F8E802AB35B106982044E4
:10252800B0423FF63EAFC4E900AB4FF0000B0834B1
:102538004FF0080A534611F8010F002878D0BBF174
:10254800000F7FF470AF2528F5D14FF0010B019BE8
:10255800013301934FF0040AECE7584694E7002052
:102568008346A5E7082B02D06FF015001BE708F19A
:10257800070828F00708F8E80223C4E9002308231D
:102588000834D8E768B9042B02D108F10408A4E795
:10259800082BE9D108F1070828F0070808F108080E
:1025A800EDE7059A013A059258F8042B009210E7D6
:1025B800039A900720D54FF0010CA4EB050E4FEAC3
:1025C8009E00BEF5007FCFD20F2FCDD8F5B107F111
:1025D80040020DEB020E019AC0B20EF8200C0EF864
:1025E800102CBCF1000F3FF41AAF60F07F000EF81A
:1025F800200C09F101090137C5F108024FF6DA7E0E
:102608000434069297E74FF0000CDAE7BCF1000FAC
:1026180001D00136EFE7029802360028EBD1009886
:10262800CDE90631FEF7BEFEDDE906310644E2E7F4
:10263800631BB3F5806F97D245B9A6F10804E0187B
:10264800B1E600BF34C90408E0FC0508029A9B08FB
:1026580028602B709DF81030C2B1EB7085F802909D
:10266800B9F1000F05D0002208A8C5F1010C974266
:102678000ED14FF0000AC5F101030DF120080193B6
:102688000DF1300B574512D1601B8CE66B70E5E7F6
:1026980010F8013B190608D50CEB040EB64503F0FB
:1026A8007F033FF67EAE04F8013B0132DFE7B9F164
:1026B800000F03D098F90020002A17DB029BD3B142
:1026C8001AF80B2004F8012B0022019B181910445A
:1026D800B0423FF666AE98F80000009904F8010B86
:1026E8002046039249F0CEFF039A14440AF1010AE6
:1026F80008F10108C6E798F8002055F82230009341
:10270800029B009845F82230FEF74CFE421CDCE79D
:102718006FF00D0047E600BF2DE9F04F97B000AF0E
:10272800D7F880B03B62CBF3C0030446894690F8E3
:1027380002A0FA62BB6141B9457800780AEB8000D3
:1027480020444D4517D8A0EB0409E378FB61BAF1A2
:10275800000F02D01BF0010F16D1FB6953BBFB6AB7
:102768001BB1494620463A6A98474D4628465C3789
:10277800BD46BDE8F08F461C3046FEF713FE01301B
:10278800304409F10109DCE7626823787A62FA6A61
:102798009900796104EB8301002A40F001810E461B
:1027A8004FF000084D4601EB0A094E454CD101EBAC
:1027B8000A0610E01BF0020FD1D023789A007A6144
:1027C800626804EB83017A62FA6A002A77D14D467F
:1027D800904601EB0A061BF0050F0CBF02230123EC
:1027E800FB62FB6906EB430A0BF00203BB6256452A
:1027F800BCD016F8021B16F8013C54F82390994BEC
:10280800994502D3984B994536D3BB69002B40D0E4
:10281800786A33F073FE00283BD0E9468AB06A46EE
:10282800924B53617B6AC2E906314FF400731384FB
:102838008F4B42F8103F00234FF412518D4800F09F
:102848009DFC023DCD46D2E716F8013BF96254F8EB
:102858002300FEF7A7FDD7F88430F96A01304BB1A1
:10286800D7F8883098453EBFD7F8843023F8180049
:1028780008F10108054498E7BB6923B1786A33F089
:102888003DFE0028C9D11BF0010F05D1FB6AED1AE6
:10289800ADE7BB6A002BAAD04846FEF783FDD7F800
:1028A800843053B1D7F8883098453FBFD7F8842093
:1028B800431C22F8183008F10108054497E7BAF1DB
:1028C800000F73D01BF0040673D0D046002607F122
:1028D800480052463B61B96249F0D4FEB96A3B6987
:1028E80001EB0A02BA62FA69F9695200FA60BA6A37
:1028F80002EB41023A610BF00202BA603A69B96A26
:102908008A4258D162781BF0020F18BF00217A6200
:1029180008BF4FEA5801B2181BF0010FD2B240F0BD
:102928009F801BF0040F14BF40460020BB616270FB
:10293800A070E17020463A6A7969FB6A9847051EDB
:10294800FFF614AFBB69414623707B6A3A6A63702D
:10295800FB6984F802A0E37007F14800FB6A984716
:10296800B0F10008C0F2BA807B69A9EB0A01C91A64
:10297800FB683A6AC91AD7E90A0398470028C0F2DF
:10298800AF804FF0000BA84408EB000507F1380AA8
:10299800B34571D300213A6A0846FB6A9847E5E6D1
:1029A80056464FF0000807F1380092E75646D046E1
:1029B80096E7B04694E7BA6A12F8021B12F8015C6F
:1029C800BA6254F82500274A904202D3264A904218
:1029D8001ED3BA6932B1786A7B6033F08FFD7B68A9
:1029E80000288BD1BA6802BB08F1280207F1300C25
:1029F80008F10100944407F1580208F1020852FA5C
:102A080080F00CF8101C5FFA88F800F8105C75E785
:102A1800BA693AB1786A7B6033F070FD7B68002848
:102A28007FF46CAF1BF0010F09D006F1280207F103
:102A38003000711C161806F8205CCEB25EE71BF059
:102A4800040F3FF45BAF08F1280207F1300008F1EA
:102A5800010102EB000808F8105C5FFA81F84DE705
:102A6800002063E734C90408E0FC0508C87B0508B2
:102A78000400000144CE04081BF80A3054F82390DF
:102A880087F83730D7F884302BB3D7F888309B4590
:102A980021D2D7F8843033F81B8001213A6AFB6AC7
:102AA80007F13700984700281ADB0544B8F1000FF2
:102AB80006D14846FEF776FC00F101081FFA88F8AF
:102AC800414648463A6AFB6A9847002808DB0544AD
:102AD8000BF1010B5CE74FF00008DEE7454645E6E1
:102AE800054643E6014B1860704700BF800100208F
:102AF80080B505460E46174698460BF007F903467B
:102B080001F050FB0446DFF81890424649F80030BF
:102B180039463046A84754F8090001F017FA00BFB3
:102B280008000000044608B5EFF31183102383F36F
:102B38001288BFF36F8F36F084FF204601F0F4F956
:102B4800024833F002FD34F082FAFCE77C7C050889
:102B5800034A0020536823F002035360704700BF04
:102B6800004004E010B5EFF31184102383F31288BA
:102B7800BFF36F8F084803683BB9084A916A41F070
:102B880001019162916AC907FCD50133036084F39E
:102B98001188BFF36F8F10BDEC3200200008024689
:102BA80010B5EFF31184102383F31288BFF36F8FEE
:102BB80011490B68A3B90122104BD3E8EF1F002974
:102BC80003D1C3E8E02F0028F7D104D102210C4A31
:102BD8000C4834F07DF884F31188BFF36F8F10BD73
:102BE800012B08BF084803F1FF3302BF826A22F0B5
:102BF800010282620B60EEE7EC320020E83200202E
:102C0800B07C0508ECCE04080008024607B505F0BC
:102C180067FD0E4B0E4A1A600E4BD3F8942042F013
:102C28000402C3F89420D3F8943003F0040301930A
:102C3800019B094BDA6A42F00102DA629A6822F0D3
:102C480002029A6003B05DF804FB00BF3006002062
:102C580000093D00000C0246000802462DE9F04735
:102C6800044607464FF00109DFF8508014B938468A
:102C7800BDE8F08794FAA4F5B5FA85F509FA05F3E5
:102C88002E0108EB05156FEA030A24EA03042B7BDF
:102C9800002BEBD058F806301B694BB946447368D3
:102CA80002222846196807EA0A0733F0A1FFDDE780
:102CB800284698470028D9D1F0E700BF7CCF040800
:102CC80030B5002289B00F490F4838F0E5F80022E6
:102CD80000230024CDE906230E230C4DCDE903344F
:102CE8004FF440722846CDE90144094B0949009444
:102CF8000AF042FD0849284637F01CFF204609B073
:102D080030BD00BF252D0008282600208021002086
:102D180029300008C0470020F17C050801480AF066
:102D280089BA00BF341000202DE9F04780462048BA
:102D38000F4633F039FF0646002832D000252846D2
:102D4800BDE8F087237B83B12368DB680BB120469D
:102D58009847636883F8069023681B69CBB9636852
:102D680002222046196833F043FF013610345445D7
:102D7800E8D3B8F1000FE2D0002DDFD02846FFF7E6
:102D88006DFF0546002FF7D00021642037F086FF3D
:102D9800F2E7204698470028E1D009FA06F31D43D8
:102DA800E3E705464FF00109024CDFF80CA0DEE727
:102DB800003300207CCF04088CCF0408014B53F863
:102DC80020007047BCCF040808B5034608462BB15D
:102DD800044A136000F068FC002008BD6FF015007D
:102DE800FBE700BF8401002010B5044C237813B919
:102DF80003480AF01FFA0123237010BD3A3F002050
:102E08003410002010B50446094833F0CDFE3CB11B
:102E1800084BD3E8EF1F0139C3E8E21F002AF8D1B5
:102E2800054838F045F8BDE8104004480AF002BAF1
:102E3800F8320020FC320020282600203410002020
:102E480000200146034BD3E8EF0FC3E8E21F002A36
:102E5800F9D17047F832002070B5FFF7F1FF054649
:102E6800074C084EB44200D370BD63685B792BB140
:102E780023685B6813B12946204698471034F1E768
:102E88007CCF04088CCF040810B5044C04492046B4
:102E980033F06DFC034B1C6010BD00BF4C0F0020CD
:102EA800A8CF0408F032002000230D4A10B5137093
:102EB8000C4A4FF47A7113600B4A0C481360FFF701
:102EC80083FFFFF7E1FF0A4B0A4918468B4200D3FC
:102ED80010BD1A1A5C681211013222711033F5E71D
:102EE8003B3F0020F8320020FC320020C36B03086F
:102EF8007CCF04088CCF0408014600220023014837
:102F080033F056BC4C0F0020014833F0EFBC00BF33
:102F18004C0F0020024B0146186833F042BD00BF39
:102F2800F0320020014833F077BD00BF4C0F00207D
:102F380070B5244B1878002842D0FFF7E5FF054606
:102F480000283AD1204B214C1B68002B12DD37F0AA
:102F58005BFF0A220023FEF7B9F9D4E90032C01A50
:102F680040F2E93361EB0201984271F1000101D3AB
:102F7800FFF772FFD4E9003213F57A7342F10002C9
:102F8800C4E90032BDE87040FFF7CCBF63685B79E5
:102F980023B12368294620461B6898471034B44259
:102FA800F4D32846FFF7B6FF094BD3E8EF1F0139E2
:102FB800C3E8E21F002AC5D0F7E7064C064EEEE745
:102FC80070BD00BF3A3F0020F832002020260020C4
:102FD800FC3200207CCF04088CCF040870B50D4D5E
:102FE800297861B90120FFF79FFE0B4C0B4EB442C4
:102FF80006D3FFF79DFF0028FBD101232B7070BD7E
:1030080063685B791BB1236820469B689847103436
:10301800EDE700BF3B3F00207CCF04088CCF0408BD
:1030280000212DE9F0470846FFF77EFE044658B315
:103038004FF4FA784FF0000901F0B4F81B4B1C4A22
:103048001B58136033B11B4B1B68092B02DD1A4850
:103058000AF0F0F80025194FDFF85CA044B12046CB
:10306800FFF7FCFD044618B94FF0FF384FF0FF3961
:10307800FFF75EFF064628B9B5B942464B465046AB
:103088000AF012F93546E9E74FF0FF384FF0FF39FB
:10309800D2E72B689B691BB1002228461146984746
:1030A8001035BD42F5D3E8E7054DFAE70800000002
:1030B800F4320020FC320020341000208CCF0408A9
:1030C8007CCF040813B5184833F06EFD174B1B78F6
:1030D80073B1EFF31184102383F31288BFF36F8F5A
:1030E800FFF726FF84F31188BFF36F8F02B010BD7E
:1030F8000F4B1B68002BF9D050B9002200230D4854
:10310800CDE9002342F2107200230BF00FF9EDE72E
:103118000928EBD1074837F0CBFE074802B0BDE8D5
:1031280010400AF087B800BFFC3200203B3F002067
:10313800F4320020282600203410002010B5064B59
:1031480004461B6898472146A060044833F0AFFB4B
:10315800BDE81040FFF7B6BF840100204C0F0020E7
:10316800044A054B9B1AB1EBD30F34BF52F8310018
:103178000020704734CE04087CCF04082DE9F04FB6
:103188008FB0C1F34A2804AF0D469146B8607B6002
:103198000C0DB8F1000F63D000264FF0040B4FF070
:1031A8000A0A07F11403C7F80C80C7E907667E62AC
:1031B8000193CDF808B0CDF800A007F11C03324602
:1031C8004846F968FFF7A8FAB0F5006F03461CD324
:1031D8006C468AB0D9F8041004AB26481A46C3E9ED
:1031E800050140F2FF71D9614FF400711984224B37
:1031F80042F8103F4FF4125133462048FFF7BEFF04
:10320800A5462C37BD46BDE8F08FC0F30A0804F187
:103218001700184420F0070080083B60FFF76CFE99
:1032280068F35325044690B13B6800F11001C7E9E3
:10323800083607F11403F961CDE900A3CDF808B009
:1032480048460F4AF96807F11C03FFF765FA68F367
:1032580053252A4620467B68B96833F0E9FCD0E755
:1032680004F1170020F007008008FFF745FE044628
:10327800EDE700BF027D0508040000019CCE0408AC
:103288000B6C03082DE9F04F87B00446DDE9105AAE
:10329800DDE91279934698460391BFB13B46524601
:1032A80010210020CDF80090CDF81490FFF762F8B7
:1032B800B0F5006F06460AD340F2FF730221174AA1
:1032C800174807B0BDE8F04F33F00BBD3E4605F197
:1032D8001700304420F007008008FFF70DFE04F0C7
:1032E80007040BF0070BE40044EA8B1444EA462475
:1032F80044EA0554054640B13FB13B465246314683
:10330800CDF800901030FFF735F84346224628469E
:10331800039907B0BDE8F04F33F08ABC417D05083A
:103328009CCE0408406820B1034BC01A40F3CF007C
:1033380070474FF0FF30704734CE04080EB403B521
:1033480003AB53F8042B01460448019301F062F9DA
:1033580002B05DF804EB03B0704700BF4D6D030881
:10336800CA0605D48B064CBF02490349FFF7E6BFDE
:10337800704700BF6ED90508579A05082DE9F04F28
:1033880089B09B46149B9DF84CA00693159B044658
:103398000593169B0D469046179E0493BAF1000FAD
:1033A80000F09D8006F48073079333F01FFC06F04D
:1033B8000209024600283ED020469149FFF7BEFF89
:1033C8000746B9F1000F08D016F0440F35D12A4648
:1033D80020468C49FFF7B2FF074406F0010353B1BA
:1033E800894B204653F82A20884B8949002A08BF70
:1033F8001A46FFF7A3FF06F48073002B49D006F0A6
:103408000803002B63D1B8F1000F66D0424620466E
:103418008049FFF793FF0546069B3D44002B6DD17D
:10342800049B002B73D1F30700F1E480314620465A
:10343800FFF796FFD8E00746C3E7774B18680028E0
:10344800CAD0764B4FF47A791B684FF03C0CB5FB29
:10345800F3F5B5FBF0F14FF4616300FB115509FB7F
:1034680005F5B1FBF3F2B5FBF0FE03FB121100FB0F
:103478001E55B1FBFCF309FB05F5B5FBF0F50CFB9C
:10348800131120460091CDE901E56549FFF756FF84
:10349800A2E706F00803EBB1624B204653F82A2056
:1034A8006149FFF74BFF0546B8F1000F05D04246CA
:1034B80020465849FFF742FF0544BBF1000FABD047
:1034C8005A4620465949FFF739FF0544A4E74FF00B
:1034D800000BE1E706F00805E6E745469CE7BBF187
:1034E800010F069B06D1002B64D1049B002B7BD0D7
:1034F80000250CE0002BF8D04D485CE04D48069BB9
:1035080022464D4932F0C9FF049B002B68D0DFF8F2
:103518002C81DFF82C91049F3146102F204628BFBC
:1035280010274FF0000BFFF71BFF5D4545DC059B9F
:10353800494620461A78FFF701FF4FF0010B1BF0B0
:10354800070F03D141462046FFF7F8FE5F453BD9F8
:10355800059B4946204613F80B20FFF7EFFE0BF1B9
:10356800010BBBF1100FEAD14FF0000B2046354993
:10357800FFF7E4FE5A46059B20469A5CA2F120011B
:103588005F2928BF2E223049FFF7D8FE0BF1010B27
:10359800BBF1100F1DD01BF0070F03D14146204689
:1035A800FFF7CCFE5F455A46E5D841462046FFF76F
:1035B800C5FEEBE71F485546A1E741462046FFF701
:1035C800BDFE0BF1010BB0E720462049FFF7B6FE20
:1035D800C5E7059B3B440593049BDB1B04939AD1E9
:1035E800BAF1000F7FF41FAF204609B0BDE8F04FD5
:1035F80033F09BBB2046054A0549FFF79FFE15E7B8
:103608007E7D0508827D0508CCCF0408797D0508F4
:1036180054D90508A77D0508083300200433002085
:103628008B7D0508E0CF0408AB7D0508B17D050852
:103638007B6D03084D6D03081D46000811F305084E
:10364800B67D0508BC7D050867A205080FF30508C7
:1036580042F20F7373B58B4228BF0B4605680446C8
:10366800052168460D4A30F0E5F9064663682846A4
:103678000B225B680A4933F04AFB636832466946A5
:1036880028465B6833F043FB63681B2228465B6867
:10369800044933F03CFB02B070BD00BFB59105088A
:1036A800DA7D0508BE7D050800210123064A9042FF
:1036B80006D8064A01B901231360054B1860704704
:1036C800012140085B00F2E740420F00043300206C
:1036D80008330020F8B50D460446064F4618B44294
:1036E80001D12846F8BD14F8011BBB6801485B6886
:1036F8009847F4E720CC0408014B0360002070478A
:1037080028D004082DE9F34205460E4600244FF060
:103718001409084B084F1B680193019BA34202DC64
:1037280002B0BDE8F0823868314609FB0400A847BA
:103738000134F2E728D004089001002070B5104B3E
:103748000D461C68B4B10F4B196800238B4202DB8D
:103758006FF0010070BD224612F8146B864202D049
:1037680014460133F2E7E06836F055FF28B100202F
:103778002C60EFE76FF00C00ECE76FF01200E9E760
:103788009001002028D0040810B5436888B002933F
:1037980083680C46CDE9033200230A68C068CDE986
:1037A8000623054901AA059335F05BFA079808B97D
:1037B800059B236008B010BD156F03082DE9F84379
:1037C8000646FDF7EFFD0546EFF31188102383F356
:1037D8001288BFF36F8F114B1C68D3F804909C427A
:1037E80008BF002434B988F31188BFF36F8F2046CF
:1037F800BDE8F883A7683846FDF7D4FDA84206D18E
:103808002A463946304648F089FF0028EBD04C4517
:1038180001D02468E6E70024E5E700BF9401002012
:103828002DE9F0410E461546FFF7C8FF044628B3B8
:10383800C3681BB35F690FB3062E07D0072E20D0CD
:103848002A4631463B46BDE8F0411847838A3BB9D2
:103858002A463146B84750B9A38A0133A38206E005
:103868004FF6FF72934204D00133A3820020BDE8D3
:10387800F0810121114A124833F02AFA6FF015003D
:10388800F5E745B12A7832B10022828231462A46CC
:103898005B699847EAE7A38A012B08D12A460721E2
:1038A8002046B8470028E2D1A38A013BD6E70BB1EE
:1038B800013BDAE70221034ADDE700BF387E05084D
:1038C80054CE04085A7E050810B5044608B180682D
:1038D80038B9104A1048012133F0FAF96FF0150091
:1038E80010BDFFF76BFF08B10C4AF3E7A082EFF3B6
:1038F8001181102383F31288BFF36F8F084B5A6826
:10390800C4E9003214605C6081F31188BFF36F8FE3
:10391800E6E700BF787E050854CE0408917E0508C6
:103928009401002008B50348034A0021121A33F015
:1039380064FB08BD40120020B4430020074808B5C6
:10394800074A0849121A33F05AFBBDE808400648EE
:10395800064A0749121A33F052BB00BF0000002084
:1039680018120020E0FC05080000002000000020DC
:10397800E0FC05082DE9F04706460C4600AF002993
:1039880036D0D1E90012E9468AB06D46A3684FF0F7
:10399800050AA8461F48C5E90723C5E9050148F8EF
:1039A80010AF002342464FF421511B48FFF7E6FBB6
:1039B800D4E90312CD466369AD461848C5E9072323
:1039C800C5E90501C5F810A0002342464FF421516E
:1039D8001148FFF7D3FBCD46E3690121104A0E4891
:1039E80033F07FF9A36901210E4A0B4833F079F9C6
:1039F800012E07D1EFF305830B4A31460648103BE9
:103A080033F06FF92146304609F062F8BD46BDE84B
:103A1800F08700BFC07E0508CCCE0408EF7E0508FD
:103A28001E7F05082D7F05085B7F050830BFFFF75F
:103A3800FDBF00BF2DE9F04105460B4EDFF82C8095
:103A4800324606EB0807CC1B2046094948F01AFE07
:103A5800A01942460021083C48F03BFEC5F89040BA
:103A680007F10800BDE8F081000000000800000030
:103A78008CCF0408054B5A699B689A421FBF044AB9
:103A8800536843F080535360704700BF4C370020A1
:103A980000ED00E070B52A4C06460D4629482A4933
:103AA80033F0BAFAA36ADB0647D52648274933F02C
:103AB800B3FA1120A36A1C0704D52248244933F01D
:103AC800ABFA12201E4CA36A990712D521491D484A
:103AD80033F0A2FA636BA26A120609D501211E4AC5
:103AE800184833F0FEF81EB1A36A23F08003A362DE
:103AF8001320134CA36ADE0704D51248174933F084
:103B08008BFA1420A36A9C0604D50E48144933F096
:103B180083FA15200A4B9A6AD10658BF9A6A9A6A9C
:103B2800920642BF5A6A22F400525A629A6A42F0D6
:103B3800FF029A6200232B7070BD1020BAE700BF05
:103B480000ED00E0CCCE04086E7F0508847F0508F0
:103B5800B77F0508CA7F0508E27F0508F87F0508D2
:103B68001780050810B5244C2449254833F054FA29
:103B7800A36A99013ED52248224933F04DFA1E2006
:103B8800A36ADA0104D51E481F4933F045FA1F20FD
:103B9800194CA36ADB0204D519481C4933F03CFAD6
:103BA8000220A36A1C0304D51548194933F034FAD6
:103BB8002120114CA36A590304D51148154933F043
:103BC8002BFA2220A36A9A0304D50D48124933F030
:103BD80023FA2320084CA36ADB0304D508480F49BD
:103BE80033F01AFA2420A36A6FEA03436FEA1343F7
:103BF800A36210BD1D20C3E700ED00E04680050864
:103C0800CCCE04085E800508718005088B80050805
:103C1800B5800508D3800508F880050812810508D5
:103C280070B5294C06460D462848294933F0F4F961
:103C3800A36AD9043CD52548264933F0EDF9172065
:103C4800A36A1A0504D52148234933F0E5F9182059
:103C58001D4CA36A9B0512D51C48204933F0DCF99A
:103C6800A36BA26A100409D501211D4A174833F035
:103C780038F81EB1A36A23F40043A3621920124C3A
:103C8800A36A590504D51148164933F0C5F91A2015
:103C9800A36ADA050ED50D48134933F0BDF91B2088
:103CA800094A936A43F47F43936200232B7070BDE3
:103CB8001620C5E7A36A9B04F2D504480B4933F0E4
:103CC800ABF91C20ECE700BF00ED00E0CCCE040807
:103CD8003D81050853810508B77F050864810508FB
:103CE8007D81050892810508AD81050817800508C2
:103CF8002DE9F0418AB0654B0446D3F804800026CC
:103D080000AFC8F3080586F31188BFF36F8F02F080
:103D18007F43B3F17F4F07D102F00C03082B12D178
:103D28005B495C4833F078F9002634460023FB7180
:103D3800EB1E092B00F28980DFE803F00A7F827B03
:103D480087878787878510074CBF0C460126EDE7D4
:103D58005149504833F060F900234C4DFB71EB6A30
:103D68009A0705D54D494B4833F056F9002331E001
:103D7800EB6A002B01DA4A49F5E7EB6A5B00F5D5F7
:103D88004849444833F048F96B69A26943F48073A1
:103D98006B61BFF34F8FBFF36F8F6B6932F8022CE3
:103DA80023F480736B61BFF34F8FBFF36F8F4DF6B2
:103DB80002739A4207D0AB6ADBB26BB30120F91DDC
:103DC800FFF768FE37E023680121374A314832F0AF
:103DD80088FF2368FA79DAB907F1080504F1200C9D
:103DE8002A4620686168083403C264451546F7D13D
:103DF8007A6A002E45D0C2F3080121B96FEA52222F
:103E08006FEA42227A62184607F10801FFF7B2FD0D
:103E18002837BD46BDE8F081AB6A13F47F4F04D064
:103E28000120F91DFFF7FCFE05E0AB6AB3F5803F02
:103E38009CD3FFF797FE0346CCE70020F91DBFE7A8
:103E48000020F91DEEE719498DE7194A18F4F87FA3
:103E5800E8468AB0174B18BF13466A461649103D04
:103E6800C2E905134FF400731384144BD56142F86B
:103E7800103F00234FF411510648FFF77FF9C5465C
:103E880074E722F4FF7222F00102BBE700ED00E0C4
:103E9800F3810508CCCE04081E8205083582050882
:103EA8005682050864820508838205089F820508F2
:103EB800DA810508C5810508C382050804000001E8
:103EC800064B5A6942F010025A615A6942F48062FC
:103ED8005A615A6922F008025A61704700ED00E001
:103EE800EFF30880EFF3098101B57246FFF700FF91
:103EF80001BD00BF0A4880F30888102080F31188AC
:103F080008484FF40061401880F30988EFF31480E3
:103F18000221084380F31488BFF36F8F00F0C4F8C0
:103F2800E0BE0020C0560020BFF34F8F0549064B66
:103F3800CA6802F4E0621343CB60BFF34F8F00BF3F
:103F4800FDE700BF00ED00E00400FA05084B9B68A0
:103F580083420BD1EFF3058343B1064B5A6842F015
:103F680080525A605A6A22F400425A6209F0D4BE5A
:103F78004C37002000ED00E016498A684FF0300009
:103F88001044EFF3098C80E8F01F102080F31288AA
:103F9800BFF36F8F104F4FF000664A698A603E602A
:103FA800D2F890000D4C2060D2F894000023C2F89B
:103FB800943080F3118802F1300090E8F01F8CF300
:103FC800098802F1000004B533F032F8BDE8044076
:103FD800704700004C37002004ED00E03833002023
:103FE8001EF0040F0CBFEFF30880EFF3098081691E
:103FF80011F8021C0229FFD001B5724633F001F80E
:1040080001BD00BF0028ACBF00F16040064B4FEA7D
:104018000111C9B2ABBF00F5614000F00F0080F894
:1040280000131954704700BF14ED00E040B2002897
:1040380007DB01234109034A00F01F00834042F8CF
:104048002130704700E100E040B200280CDB01227B
:104058000649430900F01F008240203341F823201D
:10406800BFF34F8FBFF36F8F704700BF00E100E0D1
:10407800054B420953F82220012300F01F0003FAE0
:1040880000F01040704700BF00E100E0044B054A13
:1040980023F07F039360BFF34F8FBFF36F8F704799
:1040A8000000000800ED00E008B5FFF7EFFF0B4A3D
:1040B800D2F8883023F47003C2F88830EFF3148301
:1040C80023F0040383F31488BFF36F8FFFF72AFCF0
:1040D800FFF734FC00F048F808F01AFE00ED00E0A5
:1040E80042F8203C009B0B4942F81C3C019B21F004
:1040F800010142F8183C029B42F8081C42F8143CA3
:104108004FF0807342F8043C0023203A0265C0F85F
:1041180094307047F92A000800B50E4B1546986090
:10412800D0F890200C4B0E461A60D0F8803083F3FC
:104138000B882C4686F309880020044B98472046B4
:10414800002100220023024C204700004970030888
:10415800F92A00084C370020383300201022014B80
:104168001A61704700ED00E0002310210348C218CF
:1041780001337D2B82F80013F9D1704700E100E08C
:1041880008B5EFF30583064A103B02EBC30152F86A
:10419800330049688847BDE80840FFF76BBC00BF9B
:1041A800340B0020014800687047000038330020B5
:1041B8001FB5094C094A23460121094800F012F9A4
:1041C80000230393074B0121E41A01A801930294E9
:1041D80000F012F904B010BD00000C20000000200F
:1041E8007CD004084012002010B50C7A0B6804F04B
:1041F8001F0223F01F031A43CB68640923F01F032F
:10420800054943EA440343F00103C1F89800C1F8A3
:104218009C20C1F8A03010BD00ED00E010B50A4B9D
:10422800D3F89030C3F30723013B984208D9012102
:104238000346064A064832F054FD6FF0150010BDDB
:10424800FFF7D2FFFBE700BF00ED00E0DA820508C8
:10425800B4CE04082DE9F04F8946144606464FF0BF
:104268000008514D85B0C84527DAD6F804A0BAF140
:10427800000F44D0BAF11F0F17D91AF01F0F14D12D
:10428800D6F800B01BF01F0F0FD1584632F0ECFEE5
:1042980007460AEB0B00013832F0E6FE874210D0E1
:1042A8006FF01507414A3B4601E04346404A012169
:1042B800404832F016FD6FF01504204605B0BDE801
:1042C800F08F17F1160FEDD0BC42EBDDC5F89870F2
:1042D800D5F89C10C5F89870D5F8A03021F01F01CA
:1042E80043F01F0BD6E900321A44994202F1FF3A13
:1042F8001DD1D34507D13146F8B232F0BEFE08F1E0
:1043080001080C36AFE73146C5F89870D5F89C30EF
:1043180022F01F0203F01F031343C5F89C30E0B2DC
:1043280032F0ABFE10F1160FC5D0441CE7E7C5F814
:104338009870D5F8A020013B23F01F0302F01F025C
:104348001343D3453146E0B2C5F8A030E8D032F087
:1043580094FE10F1160FAED0C5F89870D5F89C20D1
:104368009DF808300BF1FF3B62F304038DF8083029
:10437800D5F8A0309DF808205B0863F347128DF844
:104388000820D6E900321344009323F01F035B444E
:10439800A3EB0A03013023F01F036946C0B203935D
:1043A800FFF73CFFBEE700BF00ED00E026830508ED
:1043B80000830508B4CE04080522044BC3F89420F2
:1043C800BFF34F8FBFF36F8F704700BF00ED00E062
:1043D800BFF35F8F0022024BC3F89420704700BFE1
:1043E80000ED00E010B5034C2278FFF733FF207092
:1043F80010BD00BF3D3F00202DE9F74F294D8A46EB
:1044080006464FF00008AB46274FD0451BDAD6F8D2
:104418000490B9F1000F3FD031680846019132F09D
:1044280023FE0199044609EB0100013832F01CFE15
:1044380084424FF014021D4B08D002FB08F36FF0C2
:1044480015024BF8032003B0BDE8F08F14F1160FE6
:104458002C60F8D01978A142F5DD02FB08B0C7F846
:104468009840C7F89840D7F89C4000F10801007BB5
:1044780064F304000871D7F8A0000C79400860F3D1
:1044880047140C71D7F89C1021F01F016960D7F808
:10449800A01021F01F01296108F1010814350C361C
:1044A800B3E700BF3C33002000ED00E03D3F0020B3
:1044B800F0B55349534CD1F890302568C3F307231E
:1044C8009D4287B000F299800020FFF781FF4E4B94
:1044D800C1F8C030854216D14C4C01A82570FFF7B1
:1044E8000BF9002506464A4FAE4213D10020237827
:1044F8004349D1F89020C2F30722934277DBFFF7B4
:104508005BFF002046E0616801EB0011FFF76CFEDD
:104518000130DFE70199280101EB0513DA683A4019
:10452800B2F1807F52D00AD8B2F5001F34D0B2F56C
:10453800800F3ED0B2F5801F12D00135D4E7B2F11A
:10454800006F43D0B2F1805FF7D15A689B68095871
:10455800013B22F01F00034423F01F03012032E037
:104568005A689B680958013B22F01F000344012048
:10457800844623F01F0340EA4C10CDE902218DF850
:10458800100002A920780593FFF748FE00282ADAD0
:104598006FF0150007B0F0BD5A689B680958013BD9
:1045A80022F01F0003444FF0020C012023F01F03E8
:1045B800E1E75A689B680958013B22F01F00034451
:1045C800022023F01F034FF0000CD4E75A689B68C1
:1045D8000958013B22F01F0003444FF0030C01204F
:1045E80023F01F03C7E7237801332370A5E7C1F839
:1045F8009830C1F8A00001337BE74FF0FF30C9E7DE
:1046080000ED00E088D00408AAFF44003D3F0020E8
:104618000000F0FFF0B587B007460E4614460021AB
:10462800102268461D4648F054F802238DF80230DF
:10463800054B2A4621466846CDE9047601932FF0BA
:10464800FFFA07B0F0BD00BFBB70030808B5024B06
:104658001B689847002008BD50330020034B044ACC
:104668001860937843F0020393707047503300202A
:104678009C01002008B5054831F067FF002383F34B
:104688001188BFF36F8F0423184602DF588305088B
:1046980008B50649064821F00701C1F1005202F5A4
:1046A800402231F0A2FE002008BD00BF3FD7002005
:1046B800543300204FF0FF324FF0FF33014808F029
:1046C800C3BC00BFAC010020014808F031BD00BFE9
:1046D800AC01002038B50546FFF7ECFF2A46082153
:1046E800074831F0CEFD044628B925B1FFF75AFD39
:1046F8000C22044B1A50FFF7E7FF204638BD00BFD5
:10470800543300200C00000038B504460D46FFF76E
:10471800D1FF21462B460822074831F02EFE0446D9
:1047280028B925B1FFF73EFD0C22044B1A50FFF7BC
:10473800CBFF204638BD00BF543300200C000000DA
:1047480010B50446FFF7B6FF2146034831F038FD9F
:10475800BDE81040FFF7B8BF5433002070B5416979
:104768000446867A0A4D59B1437ADB0706D42C23CE
:1047780003FB06535B6A1B689B68984700236361C9
:104788002C20214606FB0050BDE8704036F037B9B2
:10479800881000202C22024B02FB0030704700BF1B
:1047A800881000202C21827A054B01FB02339A6A7B
:1047B8001B7F801A1B3323F00303B0FBF3F0704711
:1047C8008810002038B52C24827A064B04FB02336B
:1047D8005B6AD3E901240C601568FFF7E3FF04FB6B
:1047E800005038BD881000202DE9F04385B00546FB
:1047F800684690461C46039136F008FBDDE90067E1
:10480800EFF31189102383F31288BFF36F8F6B8B3B
:10481800002B41D02A8B9A4225D900220023284612
:1048280008F0D6FC0446F0B189F31188BFF36F8F06
:10483800039B002B41D032463B46684636F00BFBC3
:104848002C21A27A254B204601FB02335B6A03A97F
:104858001B681D68DDE90023A847606170BB20461E
:10486800FFF77CFF24E0698B4B1E6B8389F311886B
:10487800BFF36F8F2B7F2A8BAC6A1B3323F00303A4
:10488800521A02FB0344154B154AEB1A9B1053436B
:10489800A3722B7FE372CBE789F31188BFF36F8F85
:1048A80023464246284608F093FC04460028BFD118
:1048B8000024204605B0BDE8F0836361012300258C
:1048C8002381039B29466382E27A656004F118001C
:1048D80047F0FFFE63692582E360EAE7881000205D
:1048E800A38B2EBA70B52C250C4C00B970BD037A79
:1048F8004668002BFAD0013BDBB20372002BF5D1DE
:10490800C3604360837A05FB03431B6A13B198476E
:104918003046EAE7FFF722FFFAE700BF88100020D9
:10492800F7B506460D461446124F384635F073FE65
:10493800E0B1BB68314638461B68AAB298470028E0
:1049480002DB002003B0F0BD002CFBD1AC42F8D252
:104958002F1B042F28BF042706F0B4F83A4601900D
:1049680001A9301947F08EFE3C44EFE76FF01200C2
:10497800E8E700BFCCCB040838B5044609F0BCF81A
:10498800204632F022FCA069C8B194F87030DB07E9
:104998000DD50221144A154832F015FC6FF0770541
:1049A800201D32F019FC09F0BBF8284638BD35F057
:1049B80032FE38B901210E4A0C4832F004FC6FF07F
:1049C8001205EDE7204601F02FF805460028E7D14B
:1049D80028220146A01847F07CFE94F8703043F076
:1049E800010384F87030DBE7788305084CCF0408AE
:1049F800A283050838B5054609F07EF8284632F046
:104A0800E4FB95F87030DA070DD40221184A1948EA
:104A180032F0D9FB4FF0FF34281D32F0DDFB09F0EE
:104A28007FF8204638BD9B0707D50221124A114856
:104A380032F0C9FB6FF07704EEE7A86933F0E2FDC6
:104A4800044628B101210D4A0A4832F0BCFBE3E7CD
:104A5800284632F04BFD044618B1A86933F0FBFD37
:104A6800DAE795F8703043F0020385F87030D3E741
:104A7800C58305084CCF0408EB8305081184050895
:104A880038B590F8703004469B0708D40221144AC0
:104A9800144832F098FB6FF07705284638BD32F09D
:104AA80094FB0021204601F05DF920B101210E4A56
:104AB8000C4832F088FBA06933F0CDFD054620B1E3
:104AC80001210A4A074832F07EFB94F87030201D15
:104AD8006FF3410384F8703032F07EFBDDE700BFEE
:104AE8002D8405084CCF04085484050872840508F1
:104AF8002DE9F04385B00746884614461E4632F035
:104B08006DFB05468EB1384632F06DFB012809D0A1
:104B1800FFF748FB6FF08502334B1A50002005B0B1
:104B2800BDE8F083B5FA85F56D09013429463846A4
:104B3800E2B232F0F7FC814630B9012123462B4A14
:104B48002B4832F0CEF8E3E744684EB1206861683C
:104B580001AB03C3227A01AC1A7007238DF8053024
:104B680008F10C06304632F01DFB2278824203D948
:104B7800304632F017FB02462146304632F0F0FA52
:104B8800D9F80C90B9F1000F09D1B8F81010FB8DC5
:104B98009942C3D93046C91A32F0FDFABEE7D9F8AE
:104BA800040083681B6B13B9D9F80090EAE729461B
:104BB80098470028F8D0041F54F8043F002BF3D07E
:104BC8001B78002BF0D0304632F0ECFA23681A78C4
:104BD800824203D9304632F0E5FA82B23046216883
:104BE80032F0BEFAE8E700BF0C000000A284050816
:104BF8002CCF04082DE9F04190F82830044603F042
:104C08001F03012B0F4600F128061BD0022B05D0ED
:104C180043BB90F8291032F0F2FC03E0818DC9B251
:104C280001F0FCF90546E8B1304632F00EFC0246C8
:104C380068688368A2B99B684BB13A463146BDE8BB
:104C4800F0411847818DC9B232F0C0FCEAE76FF035
:104C58008503FFF7A7FA0F4A13500020BDE8F0813B
:104C6800DB68E9E7204694F8291032F003FB024696
:104C78000028ECD0304632F0E8FB40B91369002B2D
:104C8800E5D03A463146204698470346E1E7D368DF
:104C9800F5E700BF0C0000002DE9F04F95B00D4678
:104CA800097E02AF00F1280331F0800804469146DE
:104CB800BB600BD00121A74AA74832F0DCFB6FF09C
:104CC800040840464C37BD46BDE8F08F6B7E03F0C4
:104CD8000102B9F1000F17D019F10C0F14D0B2B9B5
:104CE80019F1710F03D12846FFF7FCFDE9E79B4A4C
:104CF8000B4699480121CDF8009031F0FCFF284679
:104D0800FFF7F0FDC846DCE7002A00F0B28400296E
:104D180040F072842B8A072B0FD9EA681368A362C4
:104D28005368E362D5F804A0E28DBAF1000F17D1F9
:104D38008B4A0121884832F09EFB0121894A864826
:104D480032F099FB2846FFF7CDFDB86832F07DFBBD
:104D58000346A069002B00F0A384802100F0A9BCC1
:104D680004F1280032F071FBE0B99AF8193032B139
:104D780098071DD46E4688B002AA7B4B05E05E07F3
:104D880016D46E4688B002AA784BC2E9053A0323C6
:104D980042F8103F70480B464FF4C251FEF7EEF947
:104DA800B546CAE70AB9724AC3E79AF81930DFE785
:104DB8002946002032F0BCF9054628B9684A012185
:104DC800654832F058FBC0E7FFF7ECF9002394F888
:104DD8002820684E12F0600F8351C2F3411307D0A8
:104DE800032B40F0E981FFF7DDF96FF085033EE022
:104DF80004F1280032F029FB94F82930002840F00B
:104E08007781013B0A2BEED801A151F823F000BFAE
:104E1800DB4F0008EF4D00085F500008EF4D000819
:104E2800454E0008EF4D0008EF4D0008EF4D000813
:104E3800E94E0008EF4D00088D4F0008A069618D0C
:104E480003697F29D3F88030CDD8A28D002ACAD132
:104E5800E28D002AC7D194F82820D206C3D194F84D
:104E68003420022A05D1FFF79DF94FF0FF33335064
:104E780018E01A070BD5C9B232F01FFB804648B1BB
:104E8800638D01213C4A344831F02BFF2BE7012385
:104E980084F83D3094F83430012B1FD1638DEBB981
:104EA80084F83430FFF77EF93358002B7FF44AAF8B
:104EB8000123B868236332F0C8FA002840F08983D8
:104EC800E38D002B00F085832946002032F030F96D
:104ED8000546002840F07983284A70E70123DFE778
:104EE800204632F07BF9628D0146FF2A3FF67BAF00
:104EF800E38D002B7FF477AF94F82830DB067FF43E
:104F080072AF94F83430002BADD02AB12046D2B21B
:104F180032F02EFB0028A6D0618D94F83C308B42ED
:104F2800C0D02046C9B200F01DFF638D804630B165
:104F380001210090124A084831F0DDFED3E61A1E1E
:104F480014BF022301230521204684F8343032F0AF
:104F58007EFCA7E7C88405082CCF0408E984050867
:104F6800188505087B8505083A85050849850508DB
:104F78005A8505080C000000928505085C8605081E
:104F8800B485050894F8283003F01F03012B7FF43B
:104F98002AAFE38D002B7FF426AF628DFF2A3FF600
:104FA80022AFA18DFF293FF61EAF94F83430022BB3
:104FB8007FF459AF2046D2B2C9B232F089FB10F162
:104FC800020F804640F04B81FFF7ECF846F800806E
:104FD80068E7E38DA18D002B7FF405AF94F834309A
:104FE800002B3FF440AF012B10D100297FF43BAFD9
:104FF80012F01F020DD1638D012B7FF453AF94F88B
:1050080070306FF3C30384F870304BE712F01F025F
:1050180017D0022A7FF446AFB4F82A80B8F1000FFF
:105028007FF440AF5FFA81FA5146204601F05CF9FF
:105038000346FFF7B7F83350013306D14FF0FF3876
:1050480051E600297FF40FAFD5E742465146204686
:1050580032F001FA26E7E38DA18D002B7FF4C3AE71
:10506800638D5FFA81F8022B13D194F8283003F08E
:105078001F0358EA03037FF4B6AE0122A069090AA8
:1050880032F0FBF900287FF4AEAE012384F83D30FE
:1050980008E794F8340000283FF4E5AE01280DD164
:1050A80000297FF4E0AE12F01F020AD1012B7FF431
:1050B800F9AE94F8703043F00803A4E712F01F0229
:1050C80012D0022A7FF4EEAE002B7FF4EBAE4146FD
:1050D800204601F0E7F80346FFF764F83350013340
:1050E800ACD001224146B2E700297FF4BCAEDDE72F
:1050F8000A2B3FF678AE01A151F823F03151000890
:10510800EF4D0008EF4D0008EF4D0008EF4D000887
:10511800EF4D0008B1510008EF4D00086B5500082D
:10512800EF4D000899550008E38DA18D022B7FF4FF
:105138005AAE94F83430002B3FF495AE012B10D1C1
:1051480000297FF490AE12F01F020DD194F8703050
:105158004FEA930808F00208C3F3001348EA03086B
:1051680006E012F01F0210D0022A12D04FF00008F9
:1051780005F10C0A504632F015F8E38D98420ED22C
:10518800FFF710F86FF00B0371E600297FF46BAEA0
:10519800DCE72046C9B232F039FB8046E8E74146F1
:1051A800504631F0EEFF7DE694F82810628DC8066F
:1051B8004FEA1223D2B204D029462046FFF71AFD3F
:1051C8004CE0013B0E2B3FF60EAE01A151F823F047
:1051D800155200085B52000875520008EF4D000890
:1051E800EF4D0008CF53000871520008EF4D00083A
:1051F800EF4D0008EF4D0008EF4D0008EF4D000897
:10520800EF4D0008EF4D00086754000805F10C0841
:105218004046B4F82EA031F0C5FF82450AD2B4F852
:105228002EA0204631F0DAFF48B101287FF4DBAD2B
:10523800A16F05E0404631F0B5FF8246F1E7616FA6
:10524800002900F0DC800A78524528BF52464046C3
:1052580030E0002329462046FFF74AFC8046B8F193
:10526800000F7FF440AD1DE60123F3E7032120463C
:1052780032F03FF8824600283FF4B5AD32F0E0F84E
:10528800E38DF0B9BAF8142098463A85DAF8102078
:1052980005F10C0A128850467A8531F083FF804563
:1052A8000BD2E08D97F8282007F12801824228BF09
:1052B8000246504631F054FFF4E5504631F072FF93
:1052C800F0E79B4600233B759AF81530DAF808207A
:1052D8007B75C34B1340C34A934263D1102107F136
:1052E800180004F0F9F8002842DB07F12803102819
:1052F8009E4628BF1020DFF8F0C207F1180280454B
:1053080003F102033DD3800002303875C7F80CE082
:1053180005F10C0A504631F045FF97F81480D8453E
:1053280028BFD846404503D2504631F03BFF80465F
:10533800B8F1020FC34628BF4FF0020B50465A4639
:1053480007F1140131F00CFFA8EB0B08D7F80CB0EB
:105358004FEA58030BEB58025A452AD118F0010FAF
:105368003FF4A0AD5046FA68D15C31F002FF99E5F0
:1053780058307FF438AD01219C4A9D4832F07BF8C3
:1053880031E512F8011B08F101084FEA111A01F082
:105398000F011CF80AA01CF8011003F802AC03F86E
:1053A800011CACE79AF814303B75DAF81030FB6052
:1053B800AEE750461BF8011BC7E9002331F0E1FEB8
:1053C800D7E90023C8E7204631F008FFD4E91D8358
:1053D800002808BF98460023C7F82A30C7F82E309F
:1053E8000A2387F828300623204687F8293031F029
:1053F800FAFE01287FF4F7ACB8F1000F02D16FF084
:10540800150870E4B8F802307B8598F8043087F8FE
:105418002C3098F8053087F82D3098F8063087F842
:105428002E3098F8073087F82F3098F8113005F1AA
:105438000C0887F830304046B4F82EA031F0B2FEA0
:10544800824508D2E08D97F8282007F1280182428A
:1054580028BF0246FBE6404631F0A4FEF3E72046AB
:1054680031F0BCFE20B101287FF4BDACA36F00E091
:10547800636F002BC3D05B88B3F5007F7FF6B3ACB6
:105488005C4B04F15002BB62002387F82C3004F116
:105498005003FB60236D9A4260D105F10C0A504617
:1054A80031F080FEB7F82A80E38D984528BF9846EA
:1054B800404503D2504631F075FE804697F82820C3
:1054C8005046424528BF424607F1280131F048FEC0
:1054D800B8F1050F94BFA8EB0808A8F10508B8F1C2
:1054E800000F3FF4DFACD4F850B0FB689B453FF4A5
:1054F800D9ACBBF1000F3FF4D5AC9BF815300F2B9E
:1055080015D19BF814205046424528BF4246DBF887
:10551800101031F025FE9BF81430434594BFA8EBDA
:105528000308A8EB0808B8F1000F3FF4BBAC636DA3
:105538005B453FF4B7ACDBF800B0DAE75A7D0F2AD9
:1055480008D11A7D798D0A447A8597F82C20013282
:1055580087F82C20626D9A429FD01B68002BEDD1F2
:105568009BE794F8343094F83CA0002B3FF47BACD4
:10557800E38D012B7FF437AC05F10C08404631F080
:1055880011FEE38D9842FFF4FBAD51464046ECE630
:1055980094F8283003F01F03012B7FF464AC2046F5
:1055A80031F0D4FF00283FF45EACA38D4268FF2B96
:1055B8003FF619AC12799A42FFF415AC0F2B3FF65F
:1055C80012AC234493F83EA0D2E76B7E59077FF5CF
:1055D8007BAC2946204600F01DFE8046FFF771BBD4
:1055E80000FF02000003020079860508D785050838
:1055F8002CCF0408050F05005A077FF5A6AB8029B4
:105608007FF4A3AB2846FFF76DF9256B012D40D138
:1056180094F83D30002B3FF454AB94F82930052B17
:105628000CD1618DA069C9B231F047FF804628B11D
:10563800638D234A2946234831F053FB94F82930D7
:10564800032B11D1638D022B0ED1A18D00220D0ADF
:105658002946A06931F011FF804628B101212B4667
:10566800194A184831F03DFB002384F83D30FFF714
:1056780028BB5B077FF569AB0029C0D1236B012BE1
:105688003FF431AB0221114A0E4831F0F4FEFFF726
:105698002ABB02210E4A0B4831F0EDFEFFF711BB81
:1056A800E38D002B3FF459AB19F10C0118BF012110
:1056B800C90132F0DCFE002380462363FFF701BBFB
:1056C800928505082CCF04081A860508F98505086F
:1056D800388605080B7810B4062B14D10369D3F863
:1056E8009C20EFF31184102383F31288BFF36F8F8C
:1056F80000204B681860506A58B9C2E9083384F32F
:105708001188BFF36F8F00220023034810BC35F0C7
:105718007CB803605362F2E70410002030B589B00A
:10572800002200230024CDE906236FF007034FF47D
:105738008062CDE90334CDE90144154B1549009445
:10574800154808F019F81549134835F0F3F9144BC2
:1057580014498B4207D30020134B14498B420CD3B6
:10576800002009B030BD03F11402D2E8EF0FC2E8FF
:10577800E54F002DF9D11833EBE703F11402D2E815
:10578800EF4FC2E8E50F002DF9D11833E6E700BF67
:105798000D580008C04A002060260020C1A1050855
:1057A80088110020D0110020D011002018120020EC
:1057B80038B50D4631F0CAFE30B90121BDE8384090
:1057C8000E4A0F4831F084BAC46804B938BD2B7842
:1057D800032B07D0052B0CD0022B08D160688368F7
:1057E8009B6902E0606883685B6903B19847246835
:1057F800EBE760688368DB69F7E700BF9386050815
:105808003CCF04082DE9F047102684B0DFF8FC816E
:1058180000AF4FF0FF334FF0FF324046391D07F01D
:10582800AFFBFB681B69D3F89C40236A73B1EFF3A5
:10583800118386F31288BFF36F8FD4F820A0BAF1D2
:10584800000F1BD183F31188BFF36F8F3B79062BB1
:10585800DFD0072BDDD801A252F823F0FB5800084F
:10586800EF58000823590008015900085959000841
:10587800455900081B580008035A0008616ADAF8FD
:1058880000208A45226208BF626283F31188BFF351
:105898006F8F9AF8183051465D062046DAF81E20B8
:1058A8001ED1FFF7F9F905460028BED0E9468AB0AF
:1058B8006A469AF81830C2E9073A05235449C2E9FA
:1058C800051042F8103F00234FF421515148FDF7CD
:1058D80055FC2A46CD460721204631F0B8FFA4E7FB
:1058E80031F084FEDFE700220121204631F0AFFFCE
:1058F8008FE700221146F8E794F8703043F004036C
:1059080084F8703094F83430022B03D12046391DC6
:10591800FFF74EFF00220321E7E794F870306FF39A
:10592800820384F8703094F83430022B03D1204677
:10593800391DFFF73DFF00220221D6E794F83430E5
:10594800022B7FF466AF2046391DFFF731FF60E771
:1059580094F87030D4F818906FF3820384F870309C
:10596800D9F808A0D9F81030A033D3E8AF3F9A0788
:105978001BD54846DAF83C309847DAF8243000213D
:10598800484698470546DAF84030484698477DB17A
:10599800214A01211F4831F09BF9002204212046A9
:1059A80031F055FF2A4607219FE74FF0FF35EFE713
:1059B8002946204600F0D6F9054608B1174AE8E717
:1059C8008021204631F01FFF20B10121144A1148DF
:1059D80031F07EF9A06932F0FFFD0022831E5842A3
:1059E800584194F87030042123F0680343EA4013C7
:1059F80084F8342084F8703077E70121094A054893
:105A080031F066F90621BA686FE700BF041000207C
:105A1800C28605083CCF0408EC8605081A870508E5
:105A2800468705086387050838B5024605460C49C8
:105A3800806932F030FE044630B10121094A0A4833
:105A480031F046F9204638BD85F83C00284600F07C
:105A580047F904460028F5D0A86932F04BFEF1E773
:105A6800DD560008738705083CCF04082DE9F84384
:105A78004FF0010805460C4646462068002840D0ED
:105A880068F07F02D2B211465FFA88F731F034FD30
:105A9800E0B1D5F800901146484631F02DFD48B9DF
:105AA800134619480121194A31F01BF96FF0150006
:105AB800BDE8F88322F08002103206FA02F229EAE1
:105AC80002032B60236823EA020323603946206817
:105AD80031F012FD80B12A683946104631F00CFDCC
:105AE80008B94346DDE706FA08F122EA01022A600E
:105AF800236823EA0103236008F10108B8F1100FB5
:105B0800BBD10020D4E700BF64CF04089A870508FA
:105B18002DE9F04F00268FB05368CDE90621D468EF
:105B2800099002930C96039674B9039B029A093361
:105B38009BB293701B0AD370069B1671DC68002C0D
:105B480040F0BC80A146A3E0002560680D958368FD
:105B58001B6B002B00F0A38007999847002800F0E2
:105B68009E80C4E903553546071F57F8043F0BB11B
:105B78001A789AB9B54240F28F80E3680D9A1343B8
:105B8800E360606883689B6A002B00F08A8098470E
:105B98008146002800F088804E4A75E05A780B2A22
:105BA80008BF9D703B685A78042A10D1E2680D99A5
:105BB8000A43E260DA78002A59D101229D702369EC
:105BC800AA40134301352361EDB200230D93D7F8A2
:105BD800008098F80130052BC7D16FF012094FF0FB
:105BE800010B099B9B69089398F8051098F8042005
:105BF8000C9B42EA0122ADF82E2098F902205FFAA8
:105C08008BFA002AB8BF4AF0800A51461846049316
:105C180031F072FC90BB0D9B51461846059331F04C
:105C28006BFC58BB98F8063098F80320514600934F
:105C380008980DF12E0332F091FB8146F0B901234B
:105C48001AF0800F1EBF2AF0800110318B40049893
:105C5800059908BF03FA0AF3BDF82E201943184323
:105C6800CDE90C0188F802A0A8F804207DE76A1E97
:105C78009A700DA90CA8FFF7F9FEA6E70BF1010B26
:105C8800BBF1100FB0D1144A0121144831F020F8AB
:105C980048460FB0BDE8F08F6FF01509F3E73546B9
:105CA8006FE76FF0850977E76068079931F06EFC58
:105CB800039B2E4603442468039335E7E36804F105
:105CC8000C01A3600CA8FFF7D1FE81460028DFD1A4
:105CD800246834E7DB870508B787050864CF04081C
:105CE80070B5836905461B69426F93F88030C3F32A
:105CF8004113022B0CD0032B0CD0012B0CBF10230B
:105D08000823D3712E6E3EB9AE6DBEB9344611E08C
:105D18002023F6E74023F4E7324601212846FFF71F
:105D2800F7FE044640B173685B790B4A01210B48C2
:105D380030F0D7FF204670BD3668E4E732460021D0
:105D48002846FFF7E5FE044618B173685B79044AF4
:105D5800ECE73668D9E700BFFF87050864CF040879
:105D6800228805082DE9F04105460E4631F036FA3D
:105D780095F83C30804633B3284631F0E7FB0746B8
:105D8800F0B10146284631F051FC102204460021AA
:105D980005F13E0046F09DFC002385F83C30FF6885
:105DA8003FB984B119491A4831F0AFFB2046BDE824
:105DB800F081786883685B6A03B198473F68EFE7CA
:105DC8006FF03C04EEE71EB985F83C600024EDE76F
:105DD80032464146284631F0A5FB074690B10246B7
:105DE800284631F04DFC04460028DFD185F83C6098
:105DF800FC68002CEAD0606883681B6A03B1984786
:105E08002468F6E76FF03C04D0E700BF5484050827
:105E180024CF04082DE9F041054688461446576802
:105E280031F077FB95F87030D8070BD54F495048BB
:105E380031F06BFB6FF00F08281D31F071FB404605
:105E4800BDE8F081B8F1010F15D1284631F0CBF942
:105E580030B94849464831F058FB6FF08508EBE700
:105E6800FB7999061AD5AB691B69D3F880309A0774
:105E78000CD44149EEE7FB799B06F4D4B8F1000F46
:105E88000AD12B6E43BB05F158060BE0B8F1000FA1
:105E9800F7D0B8F1010F01D03849DBE7AB6D83B912
:105EA80005F1600600223368E3B96268B8F1000FB3
:105EB8003FD16B6F5B7C0133DBB253716A6F5374F4
:105EC80022E0A34206D12E49294831F01EFB6FF08B
:105ED8001508B1E71B68E2E7A34201D12949F3E7B6
:105EE8001B68CFE79C4221D12368CAB97268336026
:105EF800944200D173600023236063685B790221B8
:105F0800214A1B4830F0EDFEA16819B3284631F04C
:105F18000AFA8046D0B11D49154831F0F6FA8BE7E8
:105F2800136073689C4208BF7260E4E71A461B68F6
:105F3800BAE7B8F1010F02D001235371E4E7AB6F60
:105F48005B7C0133DBB25371AA6FB8E7A06831F00C
:105F580077FAB87100232360736823B9C6E900444F
:105F68004FF0000868E71C607460F9E7738805085B
:105F780024CF0408958805084F880508B3880508C4
:105F8800D3880508F08805080D8905082A890508B9
:105F9800F8B5054600AF21B301290BD1184C194EAD
:105FA8002AE0636828461968FBF7EAF9B0B11834A3
:105FB800B442F6D36C4688B06A46134BC2E905353D
:105FC8004FF400739383114B42F8103F00234FF4B2
:105FD800E2510F48FDF7D2F8A54600242046BD46F9
:105FE800F8BD0C4C0C4EE3E7636828461968FBF7CC
:105FF800C7F90028F2D01834B442F5D3DAE700BF65
:10600800D011002018120020618905080300000142
:1060180034CF040888110020D011002070B5012564
:1060280001F07F0311F0800F18BF10339D4090F8E6
:1060380034300446022B06D001210C4A0C4830F0BB
:1060480047FE002070BD90F83C6031F0C7F832463A
:106058000146204631F066FA0028F2D0C0680028D0
:10606800EFD083681D42EDD10068F8E77F89050805
:1060780034CF04082DE9F84305460846114616466C
:106088009846FFF785FF0446002843D0284631F09C
:1060980076FA95F87030DA0702D5204A012109E02E
:1060A800D4F8049004F11407D7E8AF3FDB070CD508
:1060B80002211B4A1B4830F00BFE6FF00F04281D0D
:1060C80007F036F82046BDE8F883D9F804301BB14C
:1060D800AB4201D0144AE1E742463146284631F046
:1060E80021FAA0B10023236003696BB9C0E9034416
:1060F800D7E8EF3F43F00103C7E8E23F002AF7D1B2
:106108000024C9F80450DAE71C600461F0E76FF076
:106118003C04D4E76FF01204D4E700BF7388050885
:10612800A489050834CF0408C68905082DE9F04F6D
:1061380083B000AF7B6097F830304C680E463B6008
:106148008146904631F04AF8A36801461B6B33B983
:106158006FF0150420460C37BD46BDE8F08F204689
:1061680098470028F4D00024051F06F10C0A55F8BA
:10617800041F09B10B782BB9002C0CBF6FF03C043D
:106188000024E7E74B78042B0ED1002C3CD18B7808
:106198007A689342EBD1CB783A689342E7D10B798E
:1061A800002BD7D00124E2E7052BE0D1002CDED06C
:1061B800B8F1010F91F802B009D0B8F1020FF1D18E
:1061C80052465946D9F8180031F0E8FA04E0524628
:1061D800D9F8180031F0C6FA04460028E2D06D4616
:1061E8008AB06A46F368C2E907B3062307495062D2
:1061F800C2E9051842F8103F00234FF44151044802
:10620800FCF7BCFFAD46A5E70024A3E7068A05080E
:106218005CCF04082DE9F0410B7E05465E060C466E
:1062280038D119062DD531F019F840B11B48012194
:106238001B4A30F04DFD4FF0FF30BDE8F081284695
:10624800D5F87480268AEF8D30F0C8FFF8B1421E69
:10625800534253419B01228A9AB1BE42324628BF1B
:106268003A46E98D91420CD9B2FBF3F103FB1122B6
:106278003AB994F91830002BBEBF637E43F0080387
:1062880063762146A869BDE8F04132F04CB998F828
:106298000730E0E76FF01500CFE700BF54CF0408E0
:1062A800428A050870B5064680690C4632F0DFF868
:1062B800054638B102212346094A0A4830F011FD43
:1062C800284670BD012214F0800F18BF24F0800406
:1062D800B36B18BF1034A2401A43B263F0E700BF93
:1062E800568A050854CF040870B5054680690E46DD
:1062F80032F0E8F8044638B102213346054A064828
:1063080030F0EFFC204670BD314605F1380031F021
:106318001BFAF7E76D8A050854CF040870B50646DE
:10632800EFF31181102282F31288BFF36F8F1D4C97
:10633800236881F31188BFF36F8F5B6893F870301F
:10634800DB0705D4BDE870400A22002307F0B8B97E
:10635800EFF3118382F31288BFF36F8F256865B955
:1063680083F31188BFF36F8F2368D3B13046BDE83C
:1063780070400022002307F06FB961682A688D42D7
:1063880008BF6260226083F31188BFF36F8F68686B
:1063980005F10801C36998472946034834F0D2F942
:1063A800E2E770BD60330020900F002030B585B063
:1063B8006C46054684E8060000230022144803A919
:1063C80006F040FD0246E8B994E80300039B5D60CF
:1063D800083383E80300EFF31180102383F3128856
:1063E800BFF36F8F039B1A600A4A516861B9C2E90B
:1063F800003380F31188BFF36F8F00220023064813
:1064080007F02AF905B030BD0B605360F1E700BF13
:10641800900F0020603300200000002038B54B7832
:106428000469202B4568206908D0222B19D0FDF774
:10643800B9FE6FF08502104B1A5010E0CB88072B7D
:10644800F5D1D3681A6842609A8802819B79837271
:1064580031F022FA22460821284631F006FA0020B7
:1064680038BD4B880921C3F34002838103F001033F
:10647800027643762246EFE70C00000008B5134683
:10648800026910694A78212A12D133B9FDF78AFEC8
:106498006FF00B02094B1A5008E0CA88011D072A41
:1064A80028BF072203F10C0030F05AFE002008BD77
:1064B800FDF778FE6FF08502004BECE70C0000005A
:1064C80038B5002405690E49EB6B05F14800C3E9AE
:1064D8000144DC606B6BC3E90144DC6034F018FBF9
:1064E80005F17800074934F0E7FA074905F1240077
:1064F80034F0E2FA284631F0CFF9204638BD00BF23
:106508001D660008C16700088D6800082DE9F34181
:10651800036906460D46D0F804801C690F7E002AE0
:1065280032D00B8A713238480BBF02210121374A19
:10653800374A00933B4630F0DEFB30462F7E31F081
:106548001FFA874204D1042104F1880031F099FA36
:1065580030462F7E31F022FA874204D1052104F11A
:10656800880031F08EFA30462F7E31F0FBF98742F1
:1065780003D104F18C0006F0BDFE2946404602B066
:10658800BDE8F04131F03CB931F0FAF9874214D155
:106598002A8AE968606B30F0A7FA28B1E3691BB171
:1065A80004F1240006F0E8FF04F18800042131F02A
:1065B80068FA04F1780006F0DFFF30462F7E31F0EC
:1065C800EDF9874215D1E3691BB104F1240006F007
:1065D800D3FF052104F1880031F053FAE36B5A899F
:1065E800DB889A4205D00022002304F1480007F016
:1065F80033F830462F7E31F0B5F98742BDD104F12A
:106608008C0006F017FEB8E71CCF0408978A050827
:10661800BB8A05082DE9F04750F8483C00F14006D0
:106628005B68074600213046D3F8008031F094F9C2
:10663800002854D00121304631F08EF900284ED17F
:10664800D6E8EF3F43F02002C6E8E12F0029F7D152
:106658009B0644D4404631F0A1F9002204460023A9
:10666800204830F032FD054650B93046052131F05A
:1066780008FA3846BDE8F0470A22002306F0ECBFC6
:106688008146047659F80C1F428A57F80C0C30F0F2
:106698004BFA04460146484630F05CFD54B1D8F840
:1066A800040031F0E5F9B4FBF0F303FB1044B4FA4D
:1066B80084F464092946404607F82D4C31F088F8DF
:1066C80068B10121084A094830F002FB2846FEF764
:1066D80009F93046BDE8F047052131F0D2B9BDE8E7
:1066E800F08700BF88100020DC8A05081CCF04084A
:1066F80038B503461B6940685D68AC68A37A84F8BE
:10670800223094F82D3084F82330696849B1237C0D
:106718003BB930F008FE30B10121054A054830F098
:10672800D7FA002038BD686830F08AFE2074F8E790
:10673800EE8A05081CCF040873B5102504698DF886
:106748000710EFF3118685F31288BFF36F8F0122CC
:10675800E06B0DF1070130F0C7F986F31188BFF33C
:106768006F8F012814D034F0DFF908B9A37EBBB9C4
:1067780001220E4BD3E8EF1F002903D1C3E8E02F15
:106788000028F7D104D10221094A0A4830F0A0FABA
:106798000A22002304F1480006F05EFF02B070BD33
:1067A80000210A2034F07AFACBE700BF68330020D2
:1067B800188B05081CCF040870B550F8782C00F128
:1067C80010045268034600212046156831F0C4F8C9
:1067D80000284DD00121204631F0BEF8002847D1CD
:1067E80053F8442C68689388918916695B1A9BB2A0
:1067F800F61A31F03DF9B0423AD8D4E8EF3F43F009
:106808001002C4E8E12F0029F7D1DB0606D5BDE860
:1068180070400221174A184830F05ABA284631F019
:10682800AFF8002206460023144830F04EFC044618
:10683800F0B10676686831F01BF9638A984203D292
:10684800686831F015F983B221462846638230F032
:10685800BFFF68B1284631F093F803460648012186
:10686800074A30F03EFA2046BDE87040FEF73AB8D5
:1068780070BD00BF378B05081CCF040888100020A6
:10688800578B050838B550F8243C04465B681A68ED
:1068980050F8083C33B9BDE838400121284A294856
:1068A80030F016BA002300F1640583828383022145
:1068B800284631F051F8B8B154E9023110699847C7
:1068C800637D1BB104F1540006F056FE05212846ED
:1068D80031F042F898B9637F6BB10022002304F1CC
:1068E800240006F0B9FE0AE00321284631F034F806
:1068F8000028E1D1E4E714F8093C002BEDD102218E
:10690800284631F029F838B123695A89DB889A4238
:1069180002D0204606F030FE0321284631F01CF84C
:1069280060B1A2699388918912695B1A9BB29A42F5
:1069380004D02046BDE8384006F01EBE38BD00BF72
:106948007C8B05081CCF0408D3B500260027044615
:10695800CDE90067054830F0BCFB28B1230658BFD5
:106968000023047658BF038202B0D0BDB4100020C3
:106978002DE9F04383B000234FF0010805691C4C52
:106988001C4E02AF28602B7785F8203005F12409CA
:10699800B442234601D3002019E095F82020103492
:1069A800CAB16C4688B01B6802AA1349C2E905132C
:1069B8004FF400739383114B42F8103F10480023A3
:1069C8004FF4E251FCF7DAFB6FF00B00A5460437F1
:1069D800BD46BDE8F08385F8208054F8043C48465D
:1069E800009354F8101C54E9032331F0E8FACFE778
:1069F800F80E0608080F0608078C050803000001B2
:106A08006CCF04081FB500230190CDE902334FF085
:106A1800FF324FF0FF3301A9024833F0F6FE05B00C
:106A28005DF804FBD40F002008B54B78FF2B07D185
:106A38004B882BB9CB881BB9FFF7E4FF002008BDB2
:106A4800FDF7B0FB6FF08502014B1A50F6E700BF67
:106A58000C00000013B514464A780369FE2A14D1C5
:106A68004A8892B9CA8882B193F820300BB1013BA9
:106A7800DBB201220DF1070104F10C008DF807309B
:106A880030F06EFB002002B010BDFDF78BFB6FF0FD
:106A98008502014B1A50F5E70C0000001FB5CDE93F
:106AA800010103924FF0FF324FF0FF3301A9034871
:106AB80033F0ABFE002005B05DF804FBD40F0020D6
:106AC8002DE9F041044617460E46006831F002F9F8
:106AD80031463A468046FFF737FFD4F87B30054603
:106AE800DB1B0146C4F87B30206830F071FE88B1AA
:106AF8000B4A434601210B4830F0F3F83146204653
:106B080031F08EF92846FDF7EDFE2046BDE8F0414C
:106B180031F052B9A37F0133A377BDE8F08100BFFC
:106B2800578B05086CCF04082DE9F74F0446006819
:106B380031F0E5F8302706464FF02408E37F012BB3
:106B48001FD82368D3F810A0D3F804909AF86110DE
:106B580017FB01810AEB010B584631F056FA5946EA
:106B680002460190484631F0E0F89AF81F30054691
:106B780033B1019A5946121A484631F0D6F80546FB
:106B880015B903B0BDE8F08F204631F08BF82A46DE
:106B9800014681463046FFF7D7FE05460146206884
:106BA80030F016FE88B10B4A334601210A4830F00E
:106BB80098F82846FDF796FE4946204631F030F908
:106BC80003B0BDE8F04F31F0F7B8E37F0133E37766
:106BD800B4E700BF578B05086CCF04082DE9F04FC8
:106BE800DFF8EC9289B04FF0FF324FF0FF33B9482D
:106BF80005A906F0C5F9059E069D3469002D40F0EB
:106C08009080257704F1240694F820309D42C0F244
:106C1800828004F11803D3E8EF2F22F00202C3E8C0
:106C2800E12F0029F7D1D3E8EF1F21F00401C3E8D1
:106C3800E21F002AF7D104F11803D3E8AF3FDB07BE
:106C4800D1D5237F022B00F09581032B00F08E8194
:106C580053BBDDF814A0DAF81050EB7F23BB504685
:106C680031F04DF88046284631F01CF84FF4007298
:106C7800014606464046FFF767FE0746014650466E
:106C880030F0A6FD002800F06D8101214346924AAC
:106C9800924830F026F83846FDF724FE314628465B
:106CA80031F0BEF831F088F8A37F002B9BD1237F09
:106CB800012B40F08481302304F1630694F861507D
:106CC800304694F8621003FB054500F06BFA243552
:106CD800024631462369284600F082FA0646C4F87F
:106CE8008400284631F087F98046284631F088F933
:106CF8000746284631F089F9E26D3044002A40F011
:106D08004281002840F03A81284631F0A5F9003840
:106D180018BF012033E1304631F064F901353036CF
:106D280072E7079FD6F804A095F8188047B32B8A16
:106D380071376A48009308BF0221434616BF0121F4
:106D4800674A684A2FF0D7FF30462F7E30F0D7FFCA
:106D5800874240F0F680E37F5A1EE2776A680AB1FC
:106D6800023BE3772046696931F05AF86B6813B142
:106D7800596931F055F82946504630F041FD5AE737
:106D8800304630F0BCFF804540F09480237FD5F832
:106D98000C80B5F810B0002B49D1BBF11F0F42D1C0
:106DA800D8F800304B453ED1414604F1540308F170
:106DB8001C0251F8040B914243F8040BF9D10A88DC
:106DC8001A808A7842219A70552384F873305323A5
:106DD80084F8743084F87630A36DE26DC4F87730A7
:106DE8000023C4F8803094F86030C4F87B209A06F9
:106DF80084F875100FD194F8612094F820309A42E5
:106E080009D294F86230013B0F2B04D8012384F88F
:106E18007F30237798E7206830F067FF022384F8F3
:106E28007F300423F5E7204630F0C6FF8CE7032BBC
:106E38008AD1302394F8617003FB0747D4F8803077
:106E480024375B44C4F88030BBF1000F16D03846B5
:106E580031F0DBF890B141465A46384631F0E8F84F
:106E6800804628B902215B461F4A1C482FF039FF8B
:106E7800D4F87B30A3EB0803C4F87B30D4F8802027
:106E8800E36D9A420DD2384631F0BFF800287FF4FE
:106E98005BAFD4F88020E36D9A4202D2206830F0CC
:106EA8003AFF384631F0D8F8003818BF012084F886
:106EB8007F00B6E7304695F8188030F00BFF804524
:106EC8007FF442AF237F2A8A052B0FD127773BE730
:106ED80055534243D40F0020578B05086CCF040844
:106EE800978A0508BB8A05081E8C0508022B7FF4C3
:106EF8002BAF4FF03008D4F8803094F86170134409
:106F0800C4F8803023681969D3F804B091F8613067
:106F180008FB031124310846039131F076F80399F0
:106F28000246584630F001FF00287FF40DAFD4F830
:106F38007B3013B1206830F0D8FE08FB07402430BE
:106F4800B0E730462F7E30F0C5FE87427FF40AAFA7
:106F5800A37F5A1EA2776A68002A3FF403AF023B58
:106F6800A377FFE6EB7F0133EB779DE62046FFF73B
:106F7800DBFD99E6204630F063FF95E6022084F8B1
:106F88007F0004231AE094F9601040B900292068B2
:106F980002DA30F0AAFEB7E630F0BDFEB4E600290A
:106FA80014DA904202D8B8F1000F06D1206830F008
:106FB8009CFE022384F87F30E3E702232377237FB4
:106FC800022B0CD1204630F03BFF0CE6904200D853
:106FD8001FB9206830F09FFEEBE70323EEE7032B91
:106FE80003D12046FFF7A0FDFDE5042B7FF4FBADA0
:106FF800A37F2BB101211D4A1D482FF069FEF2E540
:10700800206830F067FE0746204630F04BFE054604
:10701800024604F1730304F17F0153F8040B8B4219
:1070280042F8040BF9D11B782946137038460D2213
:10703800FFF78AFC06460146206830F0C9FB78B1A4
:107048000C4A3B4601210A482FF04BFE3046FDF71B
:1070580049FC2946204630F0E3FE30F0ADFEC2E59B
:10706800A37F0133A37705232377BCE5448C050868
:107078006CCF0408578B0508802938B50D4614468F
:1070880021D083290DD019BB80235371832303207A
:10709800117193710023E07023706570A370043040
:1070A80038BD0223137101235371002393710A23FE
:1070B800D37108224168A01845F042FB064B0E2008
:1070C8001B882382E6E7044B02201B889380E1E7B4
:1070D8006FF08500E4E700BF10F305082DE9F041E3
:1070E8008769D0F82480BA4228BF3A46B2FBF8F53F
:1070F8000446C2692B4600682FF068FF064648B967
:10710800B7FBF8F7AF4207D0E3692B44E361606A45
:10711800684312E000250126002205212068FCF7BB
:107128007FFB60B10121094A09482FF0D1FDE369CD
:107138002B44E3610020074BA362BDE8F081E369BB
:107148002B44E361002EF5D1E1E700BF658C05080B
:107158006CCF04080203000C81420B4607B509D323
:1071680002210D4A0D482FF0BCFD6FF0150003B049
:107178005DF804FB6AB101391144814201D28B42A6
:1071880007D90221009305481346054A2FF0B3FD9D
:10719800EBE70020EBE700BF7C8C05086CCF040808
:1071A800938C05080C290346084616D11B78252B15
:1071B80012D009D8122B10D8084A42FA03F313F058
:1071C800010F08BF0620704703F0FD02282A03D0EC
:1071D8005A2B08BF0A2070470A207047F6FFFBFFAA
:1071E8002DE9F0411E4690F82C30062A23F00C03B6
:1071F80080F82C304FF00003C0E904338361044663
:1072080088460B7886B040F00C81D3B94D7915F0DB
:10721800040540F0168290F82C309B070AD402230C
:107228004FF468521D4684F8295084F82830002508
:1072380062853AE030F045FE0028F0D12B462A4618
:10724800F1E7032B35D14F7917F0040740F0F981A6
:1072580090F82C308DF8077043F0040380F82C3038
:107268007023ADF8043090F829300D7903F00F033E
:107278008DF806300A23122D28BF12258DF80B3001
:10728800438D2A465BBA304601A98DF808708DF8FF
:1072980009708DF80A700397ADF81030ADF81270C8
:1072A800ADF8147045F0EEF9A762284606B0BDE8BF
:1072B800F081122B4BD14B795F0700F1C28190F816
:1072C8002C3043F0040380F82C304B7813F002077D
:1072D80023D113F0010F8B7819D0B1F8035032463F
:1072E8001946FFF7C9FE6DBAADB2854206DAB8F89D
:1072F800030040BA80B200231A4613E03246204603
:1073080098F80210FFF7B8FE0028F4DA05E083B118
:107318000221AB4AAB482FF0E4FC022305274FF4C7
:1073280010520020054684F8283084F829706285B8
:10733800BBE7B1F80350314630F0F9FD6DBAADB294
:107348008542D4DB3146204630F0F1FDDCE71A2BCC
:1073580027D14D7915F0040540F0738190F82C3051
:1073680043F0040380F82C308B783F2B14D1CF786E
:1073780097B90D790323042D28BF042530462A46E2
:1073880001A9019345F07EF93A463B4684F8282046
:1073980084F82970638588E7022205274FF4105383
:1073A800F4E71B2B23D14D7915F0040540F04981F2
:1073B800097990F82C200809C2F340030AD18E07F6
:1073C80008D5C80711D402F00302032A00F03E8151
:1073D800002301E0002BF6D094F82C2063F341023F
:1073E80084F82C2000231A461DE70123F4E71E2BFE
:1073F80040F022814D7915F0040540F022810B7987
:1074080013F0030306D0012BECD190F82C3043F095
:10741800010303E090F82C3065F3000384F82C3066
:10742800E0E70A2A40F00881232B40D14B7A13F079
:10743800040340F00681ADF804308DF806300823C7
:1074480090F82C208DF8073042F0040280F82C20A8
:1074580030F037FD0028B5BF4FF0FF33022203227A
:10746800236A8DF80C20A8BF1BBA0293636A3046C2
:107478001BBAC3F307228DF80D30C3F307438DF809
:107488000F3094F82C308DF80E2043F0040384F864
:107498002C30B8F8075001A96DBAADB20C2D28BF31
:1074A8000C252A4645F0EEF80023A362FDE6252BBD
:1074B8002ED14F7A17F0040740F0C38090F82C3093
:1074C80043F00403990780F82C3006D402274FF4C0
:1074D8006853002584F828705AE730F0F2FC002839
:1074E800F4D1236A93B1013B1ABA22F07F421B06FA
:1074F80094F82C00616A1A4309BA40F0040084F831
:107508002C000023082532607160E3E71A46EFE794
:10751800282B2BD14D7A15F0040540F0928090F875
:107528002C30D1F8027043F004039A07B1F80760D1
:1075380080F82C307FF573AE30F0C3FC00287FF460
:107548006EAE76BA3FBAB6B232463946206AFFF70F
:1075580003FE20B1022305254FF4045263E61A4BBB
:10756800E7612361636A7343A36167E62A2B2FD11E
:107578004D7A15F0040564D190F82C30D1F80270DA
:1075880043F00803B1F8076080F82C309B077FF5BB
:1075980046AE30F096FC00287FF441AE76BA3FBA8A
:1075A800B6B232463946206AFFF7D6FD0028D1D157
:1075B800064BE7616361636A7343A36112E700BF27
:1075C800BD8C05086CCF0408997F0308E570000896
:1075D8005A2B31D14D7A15F0040532D190F82C3060
:1075E80043F0040380F82C308B783F2B19D1CF78E7
:1075F800E7B94FF4C063CDE90135B1F8075030461B
:107608006DBAADB2082D28BF082501A92A4645F054
:1076180039F800231A4684F8283084F829706285DE
:1076280043E6022305274FF41052F4E70223052707
:107638004FF410520025EEE70121074A07482FF0C2
:1076480050FB022305254FF41052ECE502230525D3
:1076580045F20232E7E500BFDA8C05086CCF040872
:1076680007B56B46084A92E8030083E80300074819
:107678008268126822B11946904703B05DF804FB8E
:107688006FF05700F9E700BF8CCF040844CA04081C
:107698001F2808B5034606D909480121094A2FF0D1
:1076A80020FB002008BD0120074A00FA03F3D16837
:1076B80033EA0101F6D01269934318BF0020F1E7BD
:1076C8005CCE0408F58C050800200246012100F074
:1076D8001F021F2808B501FA02F2034606D9064818
:1076E800064A2FF0FEFA6FF0150008BD044B002083
:1076F800DA601A61F9E700BF5CCE0408F58C05086A
:10770800002002462DE9F041054600264FF0010809
:107718000E4F6B78F4B2A34201D8BDE8F0812B7804
:107728001C442046FFF7B4FF68B12046FFF7CEFFA0
:1077380057F834303BB107EBC40204F01F0451681A
:1077480008FA04F098470136E3E700BF6C330020DD
:10775800014B1954704700BFCF0A0020034670B18F
:10776800B0FA80F2C2F11F02D2B206498856064A20
:10777800D2F880100B43C2F88030FCF757BCFF22C8
:10778800F3E700BFCF0A002000200246034AD2F8E0
:10779800803023EA0003C2F8803070470020024698
:1077A800032921D8DFE801F0020C10190F4B1A68E1
:1077B80022EA00021A605A6822EA00025A607047F8
:1077C8000A4B1A680243F5E7084B5A6802435A60A5
:1077D8001A6822EA00021A607047044B1A680243CA
:1077E8001A605A6810435860704700BF002002466C
:1077F80030B5B0B1B0FA80F3C3F11F03DBB20B4868
:1078080050F833408C4204D100EBC3056D689542B3
:1078180005D044B940F8331000EBC30042600020A3
:1078280030BDFF23EBE76FF00F00F9E76C33002062
:1078380060B1B0FA80F3C3F11F03DBB20021044A40
:1078480042F8331002EBC30251607047FF23F5E79B
:107858006C330020C300074AC0F38100183052F887
:10786800202003F018000F238340134023FA00F070
:10787800704700BF00200246F8B504690D4600AF06
:10788800A034D4E8AF3FC3F38003994217D1164A16
:10789800164B6E4688B0002908BF13466A4614493D
:1078A800C2E905134FF400739383124B42F8103F5B
:1078B80000234FF4E4511048FBF760FCB5464DB186
:1078C800D4E8EF3F43F00403C4E8E23F002AF7D1CD
:1078D800BD46F8BDD4E8EF3F23F00403C4E8E23F17
:1078E800002AF5D0F6E700BF5D8D0508558D05081F
:1078F800648D0508030000010CCF04082DE9F0474A
:107908000546894690461F46D0F808A030F0AAFCE4
:107918000446D0B1067FF3070AD590F820301848FE
:107928000121184A2FF0DDF96FF07700BDE8F087E4
:107938003B464246494630F055FC48B994F8203059
:107948000121114A0E482FF0CCF96FF01200EDE733
:107958009DF8203026F0060684F82180678484F894
:1079680024302677DAF81830214628469847B0FAA6
:1079780080F3227F5B0963F300022277D6E700BF1A
:107988000CCF0408768D0508908D050870B505465E
:10799800866830F067FC0446D8B1037FDB0709D45A
:1079A80090F820300C4801210C4A2FF09AF96FF01A
:1079B800770070BD0146F3692846984738B1237FA0
:1079C80003F00103227F63F300022277F1E7034605
:1079D800F8E76FF01200ECE70CCF0408B28D050849
:1079E8002DE9F3411746D0F808800546D8F83C3011
:1079F8000E4698470022002339460B48FCF7F4FE50
:107A0800044670B901213B46084A094800962FF000
:107A180072F92846D8F840309847204602B0BDE8A9
:107A2800F0810676F5E700BFE0100020CD8D05084F
:107A38000CCF040870B50D460C7E497E0669C9074F
:107A4800D6F88020D6F8A4301FD56CBBEA68D48855
:107A580043B1012B03D1D6F8A800FCF743FF00235C
:107A6800C6F8A430C6F8A85064B3EB681C78E409DB
:107A78000134D6F8A4309C4204D10221144A154896
:107A88002FF026F9C6F8A44070BD6CB9012B1BD0A5
:107A9800042B14D12B8A002BEBD002210E4A0D485F
:107AA8002FF016F90624E4E7052B0FD0022B04D19A
:107AB80082F0040303F00404DBE7032B06D0012162
:107AC800064AECE70324D4E70524D2E70024D0E7EC
:107AD800248E05080CCF0408F78D0508048E0508C8
:107AE80013B503690C46D3F8AC0091F8201032F0B6
:107AF800C0F894F8203048B101210090084A09489C
:107B08002FF0F9F86FF0040002B010BD5B0601D148
:107B18000020F9E7237F43F002032377F8E700BF4B
:107B28003B8E050814CF0408F8B503694768D3F8F5
:107B3800AC4091F9203091F82060002B01DB002047
:107B4800F8BD7306FBD0488CB7F84830C0F30A007C
:107B5800834293BF033303308308C3F38D03402B61
:107B680098BF5B00D4F8E8049D008AB9A84224BFF6
:107B7800401BC4F8E80491F820100022204601F0C8
:107B88007F0132F011F90028D9D06FF00400D7E74F
:107B9800BA68121AAA4207D20A4832460A4930F08D
:107BA800DAFE6FF00B00CBE720469AB206F07F01B1
:107BB80032F0FAF80028E8D1D4F8E8342B44C4F8B5
:107BC800E834BCE714CF0408628E0508F7B54668A8
:107BD80003697468D3F8AC5064009834A1B20746BE
:107BE800A400284632F0FFF8C5F8E8440124102222
:107BF8000021284632F0D8F8D5F8E8344033C5F8E3
:107C0800E83473689C420ED3284631F038FF0546A5
:107C180080B102461649174830F09DFE6FF0040403
:107C2800204603B0F0BDE1B20022284632F0BCF88D
:107C38000134E6E702460146009040233846FFF744
:107C48005DFE044628B12A460B490A4830F083FEF7
:107C5800E6E702460090402380213846FFF74EFEB3
:107C6800044608B18022EFE73069FCF7DFF9D7E76F
:107C7800858E050814CF04089A8E050838B5044681
:107C88000369D3F8AC5043681869FCF7DDF90021A3
:107C98002046FFF77BFE38B10C490D4830F060FEF6
:107CA8006FF00404204638BD20468021FFF76EFEA1
:107CB80004460028F0D1284631F0FEFE024600288E
:107CC800F0D00449024830F046FEE9E7B48E0508D2
:107CD80014CF0408D78E050838B503690546D3F8CC
:107CE800AC40204632F05AF8024630B10D490E48F1
:107CF80030F031FE6FF0040038BD0021142032F05E
:107D0800CDFF204632F04DF804460028F2D1014656
:107D18002846FFF7B1FD22460221284630F0FAFA3C
:107D28002046E9E7EB8E050814CF040870B503690F
:107D380045680446D3F8AC0031F08CFE024618B111
:107D48001A491B4830F007FE6668F069D8B14368E5
:107D580098470446B8B102461649154830F0FBFD6D
:107D6800002C19DB00F09CFC024618B1124910489F
:107D780030F0F1FD2869FCF77BF910B12869FCF7B0
:107D880063F9002070BD0D48716983685B6843B969
:107D98000B49074830F0E4FD0A49054830F0E0FD9A
:107DA800E0E798470028DDD0F2E700BF0C8F050810
:107DB80014CF0408228F0508758F050844CA0408E3
:107DC800408F05085C8F05082DE9F04103690646D8
:107DD800D3F8AC50476800F02FFC044638B102468F
:107DE8002D492E4830F0B7FD2046BDE8F081766871
:107DF8002B4896F84A307169012BD0F8088012D9BF
:107E0800D8F81830083153B92649244830F0A8FD6D
:107E18002549224830F0A4FD6FF00404E4E7224627
:107E280098470028F0D1D8F8003071690BB91F497C
:107E3800EBE71B48984704460028F8D1F06950B191
:107E480003689847064630B102461949134830F08E
:107E580082FD002EDCDB40F2E4420021284644F09B
:107E680038FC3B6828462B607B682B7140232B72BB
:107E78003B6B6B727B6BEB7102F0EEFE024620B13E
:107E88000C49064830F067FDC6E7284631F014FE75
:107E98000028A9D0C0E700BF938F050814CF0408B5
:107EA80044CA0408B08F05080A900508D28F05084F
:107EB800ED8F0508229005082DE9F04F06464FF092
:107EC80000084FF0280A4FF0400BD0F81090446893
:107ED800D9F8AC708BB06368434559D84FF00008A7
:107EE8004FF0280A4FF0400B6368434500F290803A
:107EF80099F8803023F06E0343F06A0389F88030E4
:107F0800636B2BB999F8803043F0010389F880300E
:107F180007F5B86108230422C7F8E46407F5B260DE
:107F280032F060FCD4E9101207F59E654FF00008A6
:107F38004FF000096FF0070301200027CDE9033057
:107F4800CDE906892846CDE901775D4B009605F015
:107F580013FC3168284632F0EDFDE368984739464E
:107F6800A06909AA31F032FA051E08DB099B3A46D6
:107F78001979186801F07CFC051E80F28480AB1C1E
:107F880000F081802A464F494F4830F0E4FC21E058
:107F98000AFB08F3E26B1A44917E41F040019176A6
:107FA800E26BB8F1000F19D1917E41F00101917691
:107FB800E26BA2F818B0E26B30461A4482F82080CF
:107FC800E16B194430F060F90546F0B13F493E488D
:107FD80030F0C6FC28460BB0BDE8F08F1A44917EFD
:107FE80041F004019176E26B1A44917E41F002015E
:107FF8009176E26B1A44917E41F008019176E26B2A
:10800800B4F848101A441183D5E708F1010862E76B
:108018000AFB08F3A26B1A44917E41F02001917685
:10802800A26BB8F1000F17D1917E41F00101917652
:10803800A26BA2F818B0A26B68F07F011A4482F80C
:108048002010A16B3046194430F01EF9054600286F
:10805800BCD108F1010847E71A44917E41F00401B8
:108068009176A26B1A44917E41F002019176A26B3F
:108078001A44917E41F008019176A26BB4F8481039
:108088001A441183D7E7A06A08B90025A2E7283463
:1080980032F0C1FA30B90E490B4830F061FC6FF08C
:1080A800150597E74FF4B011204630F0DFFB0028A4
:1080B800EBD00849044830F053FC6FF0040589E719
:1080C800B58100085290050814CF040836900508B9
:1080D800709005088C90050873B5D0F8AC60084618
:1080E8000C46154630F0C7F8B8B930466B8AEA68CE
:1080F80094F8201031F07DFD58B194F8203001211A
:108108000090074A07482EF0F6FD6FF0040002B011
:1081180070BD0121204630F0B2F80020F7E700BF1B
:10812800A990050814CF04082DE9F341036907460F
:1081380008460C461546D3F8AC8030F09CF878BB5E
:1081480094F820102B8A80291E46EA6802D1402B19
:1081580028BF402691199B1B2B82E9603346404675
:1081680094F8201031F06BFD054660B194F820308A
:10817800012100900B4A0C482EF0BDFD6FF0040061
:1081880002B0BDE8F0810121204630F078F894F87B
:108198002030802B04D11EB12946384630F08DFBA3
:1081A8000020EDE7CF90050814CF04082DE9F74F1C
:1081B8000369A04FD3F8AC50DFF87C824FF0FF3250
:1081C80001A94FF0FF3305F5B26004F0D9FE9DF820
:1081D8000410012900F0C78002294CD00029EDD1F4
:1081E800D5F8E44405F29C4A204630F03BF830F0DC
:1081F80066F808B1FCF776FB8021204630F032F8AB
:1082080030F05DF808B1FCF76DFB0822002120462C
:1082180030F0D2F9064620B93846884930F0A0FB3C
:10822800CCE730F067F80822514606F10C002EF032
:1082380097FF20463146FFF7FDFB204630F0F3FA62
:1082480068B1F3682046D98830F037FB10F10C0F7D
:108258000246B3D13146204630F068F8AEE72046F2
:1082680030F0E8FA18B1204630F091FAA6E7204637
:1082780030F0B3FAA2E79DF80590D5F8E46449F028
:10828800800B594630462FF0EDFF824600212FF033
:10829800F6FF504630F02AF8044600288ED019F030
:1082A8007F0F18D1038A73B3402B28BF4023C268BD
:1082B800594628461E4631F0C2FC024620B14146C6
:1082C800384630F048FB79E7238A9B1B2382E36812
:1082D8003344E36072E730F014F8814678BB5046C7
:1082E8002FF0E9FF4A462146304630F01FF8504645
:1082F8002FF0FCFF024600283FF460AF514630469D
:10830800FFF712FF5AE72FF0FCFFC0B950462FF0D5
:10831800D2FF304630F09CFAF8B12146304630F0B2
:108328007BFA30462146FFF785FB304630F089FA64
:1083380000283FF443AF2046FCF7D4FA3EE7204636
:108348002FF0E3FFE26800235946284631F077FC16
:10835800024600283FF432AFB1E7304630F07FFAEA
:108368000028DAD1DDE79DF80590D5F8E4644946A0
:108378003046BDF806B02FF075FF04462FF0B6FF63
:10838800824648B938464A462D4930F0E4FA514603
:1083980020462FF074FF11E759460C302EF0DAFE14
:1083A800B9F1000F3CD1304630F04BFAD8B1204635
:1083B8002FF081FF824601463046FFF73BFB5146CE
:1083C800304630F029FA002120462FF058FF204689
:1083D8002FF08CFF024600283FF4F0AE21463069AA
:1083E800FFF77AFEEAE6BAF81020D5F8EC349A429C
:1083F80009D2DAF80C1040230A44284694F82010D1
:1084080031F0F7FBDAE620462FF055FF82460146A9
:108418003046FFF70FFB5146304630F092F9D2E76D
:1084280020462FF048FF0022014630462FF07EFFFD
:10843800C9E700BF14CF040813910508F690050892
:1084480032910508F7B591F82150036905F0030545
:10845800D3F8AC706B1E022B4FF001020C4688BF9C
:108468000025FFF761FB064698B9628C2B46384613
:1084780094F82010C2F30A0231F054FB48B194F882
:10848800203001210090044A04482EF034FC6FF09B
:108498000406304603B0F0BD4B91050814CF04081C
:1084A80013B503690C46D3F8AC0031F028FB40B192
:1084B8000121009023460448044A2EF01CFC6FF06A
:1084C800040002B010BD00BF14CF04086E91050867
:1084D80037B5036905460C46D3F8AC0091F820106F
:1084E80031F059FB024630B92146284603B0BDE8B1
:1084F8003040FFF719BB94F8203001210090044A5E
:1085080004482EF0F8FB6FF0040003B030BD00BF44
:108518009491050814CF040873B5036905460C4601
:10852800D3F8AC0091F8201031F0DAFB58B194F888
:10853800203001210090154A15482EF0DCFB6FF021
:10854800040002B070BD237F60F341032377204607
:108558002FF0CCFE064608B90020F2E720462FF09F
:108568008AFE94F92030002B07DA0028F4D132462D
:1085780021462846FFF7D8FDEEE70028ECD0324622
:1085880021462869FFF7A8FDE6E700BFB89105086E
:1085980014CF040837B50D46044631F048FB0123D3
:1085A8008DF805508DF80430ADF806000022002340
:1085B80001A904F5B26032F028F918B1024903485C
:1085C80030F0CEF903B030BDDF91050814CF0408B0
:1085D800002307B5ADF8063002238DF805108DF895
:1085E80004300022002301A900F5B26032F00DF931
:1085F80018B10349034830F0B3F903B05DF804FB40
:10860800DF91050814CF0408002307B50193002261
:10861800002301A900F5B26032F0F7F8002803DA68
:108628000349044830F09CF903B05DF804FB00BF2F
:10863800DF91050814CF040838B54FF0FF324FF02A
:10864800FF33124804F030FE0446C0B9104D2B68C1
:108658005A1C2A6083B90F4BDA6802F44032B2F52B
:10866800003F0ED26FF0040401210B4A0B482EF094
:108678002FFB2B68013B2B60044804F0DBFD2046F0
:1086880038BD1A6942F080521A61F5E7641000207B
:10869800CC3500200008024612920508F4CE0408E2
:1086A80010B54FF0FF324FF0FF330A4804F0FCFDDD
:1086B800044660B9084A1368013B136023B9074AA6
:1086C800136923F080531361024804F0B3FD204678
:1086D80010BD00BF64100020CC3500200008024601
:1086E800074B1A6822F004021A605A68D207FCD4B1
:1086F8000222DA601A6842F001021A60704700BF6D
:1087080000040340044B1A6822F001021A601A6838
:10871800D207FCD4704700BF000403400D4A0E493D
:10872800936813F4000308D0936813F400030CD182
:10873800D2F8F42051F8230070479068000207D45B
:10874800D2F8F430C3F30333F4E793681B0FF1E76F
:108758009268EFE7000C0246BCD5040838B5394BDF
:108768000D4618680B881446C3F30B03112B31D838
:1087780013B96FF0850040E0013B102BF9D801A236
:1087880052F823F005880008D7870008D187000829
:108798007B8700087B870008278800081B8800085B
:1087A80021880008F7870008F7870008F78700087E
:1087B800F7870008F7870008F78700082B88000864
:1087C80005880008058800084FF4FA400FE04FF4C8
:1087D80000400CE0882B0AD003F67473C3F30B0334
:1087E8001C2BC6D8184A22FA03F3DB07C1D5206030
:1087F8002B68B3F5805F1ED2002038BDFFF78EFFCF
:108808004FF42023A0FB0303400B40EAC340400879
:10881800EDE7FFF783FFEAE70C4B1868E7E70C483A
:10882800E5E7FFF77BFF4FF42023A0FB0303400B92
:1088380040EAC340DBE7C3F313330133B0FBF3F083
:108848002060D9E73006002011011111BCD50408B9
:10885800006CDC0237B5A94CA94BE26902F00C02A6
:108868001341D80700F14581FFF758FF236AA54A4D
:1088780003F00F03D35C20FA03F5A34BDA6842F444
:108888004032DA60DA681104FCD5A048854201D28A
:1088980003F056F8994CD4F8943043F00403C4F824
:1088A8009430D4F8943003F004030093009BFAF753
:1088B80059F9D4F8F03023F0180343F01003C4F842
:1088C800F030D4F8F03043F00103C4F8F030D4F8B5
:1088D800F0309A07FBD5D4F8F03043F08003C4F8A1
:1088E800F030864CD4F8F0301B05FBD5FAF758F970
:1088F800A36843F40003A360A36823F0704343F024
:108908008043A360236843F040032360236843F057
:1089180008032360236843F001032360774B1A6838
:108928005407FCD5D3F8942050070BD4D3F89420DF
:1089380042F00402C3F89420D3F8943003F00403FF
:108948000193019B6D4CFAF70DF9D4F8F03043F020
:108958008063C4F8F030D4F8F0301901FBD5FAF789
:108968001FF9236843F480532360644B1A68920408
:10897800FCD5DA6902F00C020C2A1AD11A685405DF
:1089880007D41A6842F480721A605C4A1368580562
:10899800FCD55A4BDA6922F0030242F00102DA618F
:1089A800DA6902F00C02042AFAD11A6A22F00F02DC
:1089B8001A62524B1A6822F080721A609A6A22F080
:1089C800030242F001029A624F4AD16821F48021E1
:1089D800D160D46814F48044FBD19A6A474922F4E0
:1089E80070429A624A4B4B4A1B699342B6BF4A4A45
:1089F800102393FBF2F38A6A03EBD37322F47042D9
:108A08005B1042EA03338B623F4BDA6842F4802200
:108A1800DA60DA685104FCD5FFF780FE3F4AA0F51A
:108A28007413A3F51063934205D93D4B3A4A0344A6
:108A3800934260D20C24314B9A6A22F470629A6293
:108A48009A6A22F00C0222439A625A6B22F4FF724D
:108A580022F0010242F04F025A639A6A22F0100291
:108A68009A625A6B22F4FE0242F480325A639A6A7E
:108A780042F400329A625A6B22F0FE4242F080724F
:108A88005A639A6A42F480229A621A6842F08072A3
:108A98001A601A689201FCD5DA6A22F00302DA62D7
:108AA8001A6B22F003021A631A6A22F00F021A6282
:108AB8001A6A22F070021A621A6A22F4E0621A62D2
:108AC8005A6A22F070025A62DA6942F00302DA61E5
:108AD8000A4AD36903F00C030C2BFAD10B4CA542BC
:108AE80002D3204602F02CFF00200E4B1C6003B07E
:108AF80030BD0020BAE66FF02100F8E7000C02460E
:108B0800FEEFFFFF6C970508000802460068890918
:108B1800BCD504080020A10700127A0000093D0016
:108B2800FFED85FF30060020182808D8054BC34004
:108B380013F0010F14BF00206FF0850070476FF02D
:108B480085007047CE7E030108B5074831F063FD04
:108B580038B10648FBF782FD0448F9F7C3FF002047
:108B680008BD6FF01200FBE720CC0408798B0008E1
:108B78000A2838B50446074D04D1AB680D212846AC
:108B88005B689847AB6803485B68E1B29847204642
:108B980038BD00BF20CC0408064A11680B6823F0D2
:108BA80004030B605068044B196883685B6803B161
:108BB80018477047EC0400205805002010B5094BF1
:108BC800D3E90040084B196883681B6803B19847CC
:108BD800236843F004032360236843F008032360F9
:108BE80010BD00BFEC0400205805002008B5EFF3C5
:108BF8001181102383F31288BFF36F8F0120084B74
:108C080093F8482083F8480081F31188BFF36F8FE9
:108C180022B9FFF7D3FF5E20FBF708FA002008BD52
:108C2800EC040020F8B51646837890F803C0EFF3FB
:108C38001182102484F31288BFF36F8F077890F89D
:108C480001E0DB1B03EA0C039E4288BF9EB2BD19FC
:108C58000CEA05053C46057082F31188BFF36F8F57
:108C68008A198A421AD177450CD1EFF31182102163
:108C780081F31288BFF36F8F0178417082F31188F6
:108C8800BFF36F8F02799B1B9A4205D331F04CFFDB
:108C980060B1084804F070FC3046F8BD05196D79DC
:108CA800013401F8015B04EA0C04DAE7FFF79EFFE0
:108CB800F2E700BF240500202DE9F8430D461446CD
:108CC800124F07F1560807F1180914B92046BDE8F4
:108CD800F8834FF0FF324FF0FF33384604F0E4FAE0
:108CE800224629464046FFF79DFF064630B94FF019
:108CF800FF324FF0FF33484604F0D6FA3846A41B3B
:108D080004F098FAA4B23544DFE700BFF404002069
:108D180010B54368046933486060196883681B6844
:108D280003B19847012204F10800114631F075FE9D
:108D38000122002104F1200031F06FFE04F1380017
:108D4800294931F0B9FE072384F86130042384F8F7
:108D580062300F23002284F84C300C23114684F82B
:108D68005E2084F85F2084F8602084F8492084F825
:108D78004A2084F84B2084F84D305E202EF050F9BC
:108D88001A4B1B491B681A681C6922F07C4222F0A6
:108D98007F028A42D86806D14AF2B0218C4202D1B9
:108DA8001449884211D0196821EA0201124A0A437B
:108DB8001A604AF2B0221A610E4ADA601A6822F082
:108DC80080421A601A685200FCD41A6842F0040201
:108DD8001A601A6842F008021A60FFF707FF0020BD
:108DE80010BD00BF44CA0408B98B0308EC04002076
:108DF800000DF000BB7C0100000DF04010B51D4BCC
:108E080001461B68EFF31184102282F31288BFF326
:108E18006F8F5A68500605D45A68D2071DD46FF070
:108E28000A0015E01A6842F080421A601A6822F0B7
:108E380080421A600A221868400005D45868400623
:108E480002D458684007E7D5013AF4D16FF004001E
:108E580084F31188BFF36F8F10BD5A689207F5D459
:108E6800586810F04000F1D19B680B60002BEFD1DF
:108E7800D5E700BFEC0400202DE9F347D8070F46DB
:108E8800144605D42E48FFF7CDFE02B0BDE8F087A2
:108E9800002A37D0EFF31185102383F31288BFF32C
:108EA8006F8F5E20FBF7E4F806465E20FBF7CCF8F0
:108EB80085F31188BFF36F8FDFF88880FFF77EFE98
:108EC800D8F800305A68510714D45B685A0611D490
:108ED8004FF0804A2546DFF87090C9F888A1D8F885
:108EE80000305B68DB070FD4BFF34F8F20BF40BF54
:108EF80020BFF4E701A8FFF781FF0024E6B15E2058
:108F0800FBF794F82046C0E701A8FFF777FF002891
:108F1800C9F888A1E3DB6A1E291F019B17FA82F2B0
:108F280089B2013DADB202F801391B0A002DE5D026
:108F38008D42F6D10193D2E7FFF72EFEE2E700BF9C
:108F480035050020EC04002000E100E02DE9F7439E
:108F580001A8FFF753FF002844DB002104278846B7
:108F68000846264C019A94F84B3094F84CC094F873
:108F78004AE0A3EB0E053CEA05055FFA82F91ED12B
:108F880094F8600094F85F6094F86150861B35EAA5
:108F980006062AD109B184F84B30B8F1000F00D089
:108FA80001925E20FBF750F8FFF7F6FD002384F8E6
:108FB8004830134803B0BDE8F04304F03BB9E1186A
:108FC80081F84E90012101330CEA0303013F4FF071
:108FD80001084FEA1222CCD109B184F84B30019232
:108FE8000028E6D103B0BDE8F0832618013005401B
:108FF80086F86390012084F86050E7E7EC040020CD
:109008000C05002000487047F4D10408044BB3F85D
:10901800A0379B020B60002318464B60704700BFC7
:109028000000FA0B07B50346054A009105480121DF
:109038002DF061FE6FF0150003B05DF804FB00BF72
:109048006A9205086CCE040873B5064664220023AC
:10905800684631F0DBFEDDE9004533691B681A6AB2
:1090680012F0FA0212D01A6A02F0FA021A626FF0CB
:10907800040002B070BD22462B46684631F0EBFE74
:10908800DDE9003213430CBF0122002233691B685B
:10909800186A10F48030ECD0002AECD00A230121A1
:1090A800024A03482DF01DFEE1E700BF949205082F
:1090B8006CCE040870B5036906461D6849B1FFF710
:1090C800C3FF044650B13069043004F0B3F82046B9
:1090D80070BDAB6A002B06DB0024F8E7AB6A43F0EF
:1090E8000043AB62F8E7034BAB6003F18833AB6036
:1090F800F2E700BF2301674573B5012306460D4615
:1091080014462FF055FE50B90A482B4601210A4A49
:1091180000942DF0F0FD6FF0150002B070BD3CB169
:1091280022462946304602B0BDE870402FF0F2BD15
:109138002046F2E76CCE0408A8920508F7B51C464D
:1091480017460123224606460D462FF031FE50B938
:109158000B482B4601210B4A00942DF0CCFD6FF0F3
:10916800150003B0F0BD44B123463A4629463046BF
:1091780003B0BDE8F0402FF0F2BD2046F1E700BF94
:109188006CCE0408D39205082DE9F84F484B1746D2
:109198001B680D46834603F001080026FFF7B2FA64
:1091A800013FDFF81091DFF810A12F44AF420CD334
:1091B800DBF810301C68A36A002B0EDA01213F4A45
:1091C8003F482DF085FD6FF00406B8F1000F01D07F
:1091D800FFF786FA3046BDE8F88F5846FFF734FFA8
:1091E800061EF2DBDBF810301B681B6C9B021AD5DD
:1091F8004FF6FF71B9F8A020236C8A4203F480135C
:1092080007D1B5F5801F44D24BB1A36A43F400637C
:1092180008E0002AF5D0B5EB422F37D22BB9A36A64
:1092280023F40063A3626B0B09E0B5F5801FECD350
:10923800A36A23F40063A362A5F580135B0BA26AFB
:10924800584642F00202A262A26A22F47E72A26228
:10925800A26A42EAC303A362A36A43F48033A36207
:10926800A36AFFF7F1FEDBF8103006461B681B6C9B
:1092780013F4001FA36A14BF03EA0A0323F00203CE
:109288000028A362A1DB05F500558FE7B5F5801F1F
:1092980005D3002BCCD1A36A43F40063CBE70121AB
:1092A8002B46084A06482DF01CFD6FF015068CE782
:1092B800000403400007FA0BFDF7FFFF249305089D
:1092C80074CE0408319305082DE9F84F0024984618
:1092D800324B0D461F6806469146A346FFF712FA21
:1092E80007F0010705F10065D8450DD93369D3F8B2
:1092F80000A0DAF82830002B0CDA0121284A294886
:109308002DF0E6FC6FF004040FB1FFF7E9F92046F1
:10931800BDE8F88F3046FFF797FE041EF4DB2BF00C
:1093280003024A44111F0B460C3253F8040F00BBCA
:109338009342FAD1DAF8283043F00103CAF828300A
:10934800DAF828302B4651F8040F914243F8040B01
:10935800F9D13046FFF778FEDAF82830041E23F0FA
:109368000103CAF8283005F11005CDDB0BF1100B0D
:10937800BAE7284600230468013408D005F1784587
:109388000121094A07482B442DF0ABFCBAE7013309
:10939800042B00F10400EED1CCE700BF0004034029
:1093A8002493050874CE04084A93050830B5104C78
:1093B800104D0C60236813B12B68136030BD03692E
:1093C8001B68196C1B6C9B020FD54FF6FD700A4B7E
:1093D800B3F8A030591E89B281428CBF4FF4807314
:1093E800DB0823604FF40053636001232B60E4E73C
:1093F800D4350020D03500200007FA0B2DE9F843BA
:10940800D0F8049090460746D9F808000D461E4645
:109418002EF0B8FEB8F5001F044616D12846D9F834
:109428000840FEF717FA84420CD129462EF0AAFE0E
:109438000446FEF7ABF92046FEF7FAF9002120466C
:10944800FEF7AEF90020BDE8F883B8F5800F20D00C
:10945800B6F1806F19D0B6F1C06F18D0B6F1007FA1
:109468001AD102263A4620460E49FEF7C1F9B0B98C
:109478002846D9F808102EF08AFE20463146FEF715
:109488008FF92046FEF76AF9DCE70126EAE70326AA
:10949800E8E76FF08500D6E76FF01500D3E76FF0C7
:1094A8000F00D0E76390030808B5094A136943F031
:1094B80000531361416807480C3183681B681BB16E
:1094C800984700EAE07008BD6FF05700F9E700BF61
:1094D8000008024644CA04080C291FB528BF0C21FD
:1094E8000C460A4BD3F8082712BA0192D3F804277E
:1094F80012BA0292D3F800370A461BBA01A903939D
:1095080043F0C0F8204604B010BD00BF0000FA0BBD
:1095180008B50121034A04482DF0DAFB6FF0040076
:1095280008BD00BFF693050894CE040898B54268B4
:109538000369D26800AF83F8621029B9136823F46D
:1095480040131360BD4698BD6C468AB06A460368EE
:109558000848D161C2E905034FF400731384064B30
:1095680042F8103F00234FF411510448F9F706FE62
:10957800A546E7E7149405080400000194CE040802
:10958800F7B500224368044606691C480F46DD68A3
:10959800596883680192DB684BB90121184A194858
:1095A8002DF096FB6FF00404204603B0F0BD01AA2D
:1095B80098470028F1DB376306F118074FF0FF32B0
:1095C8004FF0FF33384603F06FFE2B68204623F038
:1095D80001032B6096F86210FFF7A8FF2046019957
:1095E80000F0A0F896F8613004461BB12B6843F0F0
:1095F80001032B60384603F01DFED5E744CA040872
:109608002894050894CE040870B504464668056990
:109618004FF0FF320021284631F0FFF93368204629
:109628009847002385F8603085F86230012205F1FB
:109638001800114631F0F1F9204600F03FF8316981
:10964800184B994222D015D8174B994220D0174B66
:10965800CB1A594259418900204641F01001FFF7C1
:109668008FFF041E18DA0121114A12482DF030FB31
:10967800204670BD104B99420CD003F5C31303F577
:10968800206399420CBF0A210021E5E70621E3E7A0
:109698000221E1E70821DFE70123002485F8603093
:1096A800E6E700BF40420F00A0860100801A0600CE
:1096B8005694050894CE040840E1330037B5456850
:1096C8000021686901AA2FF081FE041E07DB019BB7
:1096D80000221979186800F0CBF8041E08DA012175
:1096E80023460C4A0C482DF0FCFA204603B030BD46
:1096F8000A48696883681B683BB90121084A06481B
:109708002DF0E6FA6FF00404EFE7984704460028C6
:10971800EBD0F2E79494050884CE040844CA040800
:10972800B29405082DE9F74F4468036900200193B6
:10973800E369E568DFF81481DFF81491DFF814A114
:10974800DFF814B10093009B8342019B1A6B0DD183
:10975800C2F34202012A3BD0022A68D03F4A40485D
:1097680001212DF0B5FA6FF015001FE00C2303FB63
:1097780000F7D4F818C0DFF8ECE00CEB07067368C4
:1097880073451DD015D853451CD05B4514BF002325
:1097980001239B00C2F34202B2EB530F16D15CF8CF
:1097A80007308B4212D1B36800202B6103B0BDE8AB
:1097B800F08F434508D04B450CBF0A230023E9E747
:1097C8000623E7E70223E5E70823E3E70130BAE7E2
:1097D80041F25C2E4FF47A6C40F2E2474FF4FA768D
:1097E8000220214B421EB1FBF2F2B3FBF2F2BCFBAA
:1097F800F2F4013CFF2C23D8BEFBF2F808F1FF3845
:10980800B8F1FF0F1CD8B6FBF2F9B9F10F0F17D852
:10981800B7FBF2F2013A0F2A12D8023848EA094394
:1098280043EA007343EA025343EA0423BCE740F2E5
:10983800145E4FF4167C4FF4FA7740F27716CFE7B0
:1098480001301128CED1094A89E700BF40E1330031
:10985800404B4C00A0860100801A0600E2940508DF
:109868008CCE040840420F0000CA9A3B5D9505085B
:109878002DE9F047044600251D4F00EBC106B44210
:1098880001D1002014E02068C30600F01F0911D49C
:10989800656845F02005C0F3481AC0F3442019282C
:1098A80023D857F82080B8F1000F0DD16FF01200BF
:1098B800BDE8F087B9F1100F04D0B9F1110FEAD162
:1098C8006568E8E73025E6E7404630F0A4FE002862
:1098D800ECD04B462A4640460AF00F012FF0D3FB46
:1098E800002804F10804CADAE2E76FF01500DFE7A0
:1098F80040D3040843681B6803F1080252E8002FAC
:1099080042F0010203F1080040E800210029F3D1E8
:10991800174A93421ED002F1805293421AD0154A38
:10992800934217D002F18052934213D0124A9342C5
:1099380010D002F1805293420CD0104A934209D0C1
:1099480002F18052934205D00D4A934202D0B3F1FE
:10995800502F03D15A6842F040025A6053E8002F52
:1099680042F4807243E800210029F7D1704700BF14
:10997800003801400044004000480040004C0040CE
:109988000050004043681B6803F1080252E8002FAA
:1099980022F0010203F1080040E800210029F3D178
:1099A800174A93421ED002F1805293421AD0154AA8
:1099B800934217D002F18052934213D0124A934235
:1099C80010D002F1805293420CD0104A934209D031
:1099D80002F18052934205D00D4A934202D0B3F16E
:1099E800502F03D15A6822F040025A6053E8002FE2
:1099F80022F4807243E800210029F7D1704700BFA4
:109A0800003801400044004000480040004C00403D
:109A1800005000400129034608461AD002290BD0FD
:109A2800C9B91B680D4A934217D002F180529B1A9C
:109A380018BF0123180370471868084B98420AD0CA
:109A480003F18053984214BF4FF440504FF4005034
:109A58007047002070474FF40050704700240046BC
:109A680070B500261D46094B6C0833F812203346A2
:109A7800F7F72CFC090241EA1061000220182A4677
:109A8800334641F10001F7F721FC70BDA4750508C4
:109A98002DE9F04782B0436880460C461D6800AF48
:109AA800002944D0586819698368DB686BB13A1D8E
:109AB8009847061E0CDA0121354A36482DF008F978
:109AC80030460837BD46BDE8F0876FF05706F2E725
:109AD800314B9D4203D003F180539D4249D100266A
:109AE800D7F80490DFF8B4A0234648460021B2B264
:109AF800FFF7B6FFA0F5407050451BD90136102E70
:109B0800F2D16D468AB0D8F800306A462449D4614B
:109B1800C2E905134FF400731384224B42F8103F37
:109B280000234FF411511B48F9F728FBAD466FF09D
:109B38001506C5E7EB6A484623F00F033343EB628B
:109B4800194B33F8162000231946F7F7BFFB090213
:109B580041EA106163080002C01822464FF0000372
:109B680041F10001F7F7B2FBC0F31300E8600026EB
:109B7800A6E72B6823F400432B607B6803EB5403B0
:109B8800B3FBF4F30F2BBCD99BB2EB60EFE700BF3C
:109B98002894050804CF040800240046FFFC0F00A1
:109BA800A195050804000001A47505082DE9F843EE
:109BB80007460D7940683B69012D0E460468D3F8C5
:109BC800008017D0AB1ED3F1000949EB03094FEA17
:109BD80089297179FFF71EFFB2790346022A0CD052
:109BE800042A0ED0ADB1033D012D0CD86FF08500CD
:109BF800BDE8F8834FF4C069EBE73DB94FF08050FA
:109C080008E0002DF2D14FF4805003E0033D012D10
:109C1800ECD90020B3F5805F4ED0B3F5405F4DD04E
:109C2800002B0CBF012303239942DFD149462FF0B3
:109C380018FC8242DAD1F37953B3012B40D1224B7D
:109C48009C4225D003F180539C4221D01F4B9C425B
:109C58001ED003F180539C421AD01D4B9C4217D052
:109C680003F180539C4213D01A4B9C4210D003F14D
:109C780080539C420CD0184B9C4209D0B4F1502F11
:109C880006D0164B9C4203D003F180539C42ADD1C1
:109C98002368314623F00103384623602FF065FD21
:109CA8000028A3DB236843F00103236096E8030040
:109CB80088E8030000209BE70023B5E70223B3E709
:109CC800032BBCD092E700BF00380140004400409D
:109CD80000480040004C004000500040002400466E
:109CE8002DE9F04383B0466805467068316983689A
:109CF80000AF1B685BB90121724A73482CF0E8FF7A
:109D08006FF0570420460C37BD46BDE8F0839847EE
:109D1800044630BB0021706A3A1D2FF057FB041E21
:109D2800F0DB7B68002219791868FFF7A1FD041E93
:109D3800E8DBD5F804802B69D8F80040D3F8009008
:109D4800236823F001032360D8F8080030F063FC8F
:109D580078B901215D4A5C482CF0BAFF6FF0120413
:109D6800D0E70121574A58482CF0B2FF002CC9DB34
:109D7800D0E7D8E902018368DB6803B1984754E863
:109D8800003F43F00C0344E80032002AF7D149466B
:109D980028462FF0EAFC002802DA6FF01504B1E734
:109DA80098F818301BB1A36843F00803A36098F82B
:109DB80019301BB1636843F40043636098F81A30A4
:109DC8001BB1636843F48033636098F81B301BB1A0
:109DD800636843F40033636098F81C30002B5AD052
:109DE8003B4B9C423AD003F180539C4236D0394BCE
:109DF8009C4233D003F180539C422FD0364B9C4277
:109E08002CD003F180539C4228D0344B9C4225D05F
:109E180003F180539C4221D0314B9C421ED0B4F1B7
:109E2800502F1BD02F4B9C4218D003F180539C42DB
:109E380014D06C4688B06A462B682B49C2E90513D2
:109E48004FF400739383294B42F8103F00234FF4DB
:109E5800E2511D48F9F792F9A5469EE76B681A6822
:109E6800936843F480439360236898F81D2023F097
:109E7800787343EA42532360236898F81E2023F43A
:109E8800F81343EA0243236098F81F301BB1A36814
:109E980043F40043A36098F820301BB1236843F0D3
:109EA80000532360236843F001032360E3699A02A7
:109EB800FCD5E3695B02FCD52846B36A98470024C1
:109EC80020E700BFB895050804CF0408D895050811
:109ED800003801400044004000480040004C004069
:109EE8000050004000240046F395050803000001D7
:109EF80038B50B68054698882FF004FD04280C46F1
:109F080003468A6D1AD002280FD191F870100129E2
:109F180002D9A16E012911D8002A49D0E16D01B1F9
:109F2800118889B2298402250EE0012821D191F8EF
:109F38007010032918D9A16E032917D992B1E16DC0
:109F480001B1116829620425E26DB5FBF3F53AB158
:109F58009542294619D901211B4A1C482CF0B8FE04
:109F6800284638BD1146EDE7012902D9A16E01291D
:109F7800D2D8FAB1E16D01B11178C9B285F82010D3
:109F8800E26D0125002AEBD02946521AE2659AB9FA
:109F9800A26C04F14C010832A264E26C04F148009E
:109FA800013AE26404F15C022FF096FCA065D7E761
:109FB8001146B6E71146E0E7A26D002AD0D001FBB2
:109FC8000322A265CCE700BF50960508DCCE040842
:109FD80038B50B68054698882FF094FC04280C4681
:109FE800D1E91812034618D002280DD194F8700050
:109FF800012802D9E06E01280FD8288E80B209B155
:10A0080002B1088002250DE001281DD194F87000E6
:10A01800032814D9E06E032813D9286B09B102B1BB
:10A0280008600425626EB5FBF3F59AB1954229469E
:10A0380018D90121184A19482CF04AFE0AE00128CB
:10A0480002D9E06E0128D8D895F83000C0B229B1FD
:10A0580012B90125284638BD0870626E002AF8D06A
:10A0680001252946521A62667AB9226D04F1540113
:10A0780008322265626D04F15000013A626504F10C
:10A0880064022FF029FC2066E4E7226E002AE1D062
:10A0980001FB03222266DDE750960508DCCE0408A2
:10A0A80038B50446006903691BB94360083003F0FA
:10A0B800C1F8012160682FF06AFC002802DA10F16B
:10A0C800860F15D16568002128462FF060FC041E14
:10A0D8000CDB0948A96883681B6853B19847044694
:10A0E80020B10121054A06482CF0F2FD04EAE4708B
:10A0F80038BD6FF05704F4E744CA04086E960508A3
:10A10800DCCE04082DE9F04F87B081460E469B4609
:10A118009246046900AF32B92BB9002630461C3785
:10A12800BD46BDE8F08FB3889A042FD44FF0FF32B4
:10A138004FF0FF3304F1080003F0B6F8666000231F
:10A14800C4E90F3384F84430D9F81030D9F80480C2
:10A15800FB601B68D8F800509E4240F0B580B38879
:10A168001B0540F1AC81BAF1000F16D028464FF418
:10A17800C1212FF0A2FBB0882FF0C4FB0346DAF808
:10A188000020A264A2B1DAF8042011E02369002BB0
:10A19800CCD163689E42C9D1D1E728464FF4C0218B
:10A1A8002FF08BFBB0882FF0ADFB03460022A26492
:10A1B800E26404F14C0104F15C0204F14800FB6024
:10A1C8002FF08AFBFB68A065BBF1000F40F093817C
:10A1D800C4F850B00022626504F1540104F164022D
:10A1E80004F150002FF078FB00232066A3632A684F
:10A1F800EB6802F4006203F4C0231343FB6098F891
:10A208002130DB0728D5B288D9F80430D007BB60E5
:10A218001B6821D41968D86801F4006100F4C020D3
:10A228000143D9F8102040F07181D16D566E29B1E3
:10A23800002E00F069818E4228BF0E46002E56DBA4
:10A24800B968C969B142C0F06F81C2E91A665A6833
:10A25800120C120432435A60D9F804301B681A6889
:10A2680042F001021A60DA68510206D51A6842F40F
:10A2780000721A601A689205FCD5E36D1BB9666E08
:10A28800002E00F0F0812268D8F800609288D2078A
:10A2980040F150817269920740F15482002B00F01E
:10A2A800518221463046FFF723FE7369D80740F1F3
:10A2B8005F81236E002B00F05B81636E002B00F042
:10A2C8005781214630462EE2D8F81020B188022A5C
:10A2D800C1F3451312D0032A13D0012A2CD1043B11
:10A2E8001C2B8CBF002301237BB96FF0850600234C
:10A2F800636004F1080002F09DFF0FE7043B0C2B9C
:10A30800EFE7082B01D0102BEFD1080448BFEB680A
:10A31800A44842BF23F4601343F40023EB6083682E
:10A32800D8F80810DB686BB901219F4A9F482CF0C8
:10A33800CFFC6FF00406DAE701219D4A9B482CF018
:10A34800C7FCD2E707F1140298470028ECDB00228B
:10A358007B69316823FA02F0884218D90132092A48
:10A36800F8D16D468AB06A46D3611B0A1362052389
:10A378009048C2E9050142F8103F00234FF42151EB
:10A388008A48F8F7FBFEAD466FF01506AFE72B6875
:10A39800894923F001032B60AB6851F8222023F090
:10A3A80070431343AB6098F82130990700F190800F
:10A3B800B38813F0020FEB6814BF43F0007323F067
:10A3C8000073EB60B38813F0040FEB6814BF43F01D
:10A3D800807323F08073EB60B18811F4006104D0BE
:10A3E800BAF1000F7BD04FF4C12128462FF065FA4F
:10A3F800B38813F0100FEB6814BF43F4000323F481
:10A408000003EB60AB6823F48003AB60327DB38854
:10A418001AB998F82120520764D5D80706D4EB68F2
:10A42800D9005EBF2B6843F480532B60EB6823F0A0
:10A43800105343F08063EB60B388604913F0010F59
:10A44800EB6814BF23F4800343F48003EB60B28805
:10A45800AB68C2F34512043A51F8222023F01F03D7
:10A468001343AB60EB68D8F8182023F00F031343AD
:10A47800EB60EB68D8F8142023F0F00343EA0213EA
:10A48800EB6098F821304E49DA0741BFB38898F855
:10A498002020C3F34513073343BFDB085B00B2FB3F
:10A4A800F3F30123FA6882F87030AA68013B51F887
:10A4B800233022F4F0721343AB60FB681E60B0884F
:10A4C8002FF020FA0346BAF1000F7FF458AE6DE67C
:10A4D800D8F80020D36843F40043D36068E74FF40A
:10A4E800C02182E713F0010FEB6823F0105308BF77
:10A4F80043F000539FE7DBF800202265002A3FF471
:10A5080069AEDBF8042066E60E4697E6B1F5C12F82
:10A5180030460CBF51465946C7E900322FF015FAAC
:10A52800D7E90032064689E60121264A1F482CF061
:10A53800CFFB29E798F8213013F0010F3368F26850
:10A5480000F0E28003F4006302F4C022134354D104
:10A5580073695B0738D47369D8073BD5E36E002B62
:10A5680038D0214630462FF058FA73691B0758D463
:10A57800D8F80060736913F4787340F0E880FB68DA
:10A58800B3F5C12F7FF479AEE36D002B00F0FE80A8
:10A598002B68EA6803F4006302F4C0221343FB60EB
:10A5A8006BE600BF44CA0408B1960508DCCE04086F
:10A5B80089960508DD960508A8D4040848D5040836
:10A5C80028D504080C970508A36E002BC3D0E36EAA
:10A5D80073B9736973699A07C7D5A36E002BC4D082
:10A5E800E26E9342C1D1214630462FF002FABCE711
:10A5F800214630462FF0FDF9B3E7B3F5C12FE9D076
:10A608007269D10702D5E26E002AAAD1B3F5C02F2C
:10A61800ABD0DFE721463046FFF7DAFCE36E1B1AC2
:10A62800E366E36E002BF5D1E36D626E002B53D128
:10A63800C4E91A22002A9BD0B369304643F01003BC
:10A64800B361B36943F00803B3612FF0B5F9A26EA3
:10A65800D8F81C309A4246D901218E4A8E482CF0EF
:10A6680037FB6FF01506D9F80450D9F8108029681F
:10A678004B69D80700F1D380CB685A0240F1D280E9
:10A68800DFF8189208462FF052F9002800F0CA8027
:10A698000B68D80740F1C68095F82130DA070DD449
:10A6A800D8F800309B88C3F34513192B06D829FA2C
:10A6B80003F3DB0702D508462FF07EF90B68CA685A
:10A6C80003F4006302F4C0221343B3F5C02FD9D1B9
:10A6D80008462FF071F9D5E712B1934228BF134607
:10A6E800C4E91A33A8E7736821461B0C1B041343FB
:10A6F8007360336843F001033360336843F40073D5
:10A7080033602FF076F933E703F4006A02F4C023CC
:10A718004AEA030ABAF5C02F08D1D8F800004369FD
:10A72800D907FCD52146FFF753FC21E77369980741
:10A73800FCD521463046FFF7DBFBBAF5C12F3FF4C5
:10A7480017AFEAE7336923F002033361ADE56D46DD
:10A758008AB06A46524951615249C2E906134FF418
:10A7680000731384504B42F8103F00234FF41151EB
:10A778004948F8F703FD7369AD46590603D5B3692F
:10A7880043F04003B3616FF004066CE7636E002B7F
:10A798003FF4FEAE30462FF0CAF803460028F9D140
:10A7A800326822F00102326022689088C20712D40F
:10A7B8001A46D4F854C0624527D12FF0A3F893FB6A
:10A7C800F0F200FB12323ABBB3FBF0F37268120CE2
:10A7D8001204134373604FF4C02130462FF06DF814
:10A7E800336843F001033360F3685B027FF5D0AE52
:10A7F800336843F400733360336898053FF5C8AE97
:10A80800736919073FF5C4AEF6E7216D01EBC20184
:10A81800496801320B44CEE72B68EB6821E791F8D1
:10A82800303025E74B699B0542BF8B6943F40073C1
:10A838008B6195F821000B68C007CA6810D58B6931
:10A8480043F010038B618B6943F040038B618B6984
:10A8580043F008038B614B681B0C1B044B6007E03B
:10A8680003F4006302F4C0221343B3F5C02FF2D0FF
:10A87800D8F800309B88DB0402D408462FF09CF8F7
:10A8880094F84430002B3FF432AD002E3FF445AC31
:10A898002DE500BF0C970508DCCE04080002020273
:10A8A8003897050843970508040000014FF0E02396
:10A8B80010B50F499C691A6908689B690D4902F42B
:10A8C800803234B993B903464AB90A681044C01AA9
:10A8D80010BD002B08BF03460AB9A342F5D90A6880
:10A8E80002440A604FF0E0221269EEE70446F3E7FB
:10A8F80048370020443700201022094B002083F8F5
:10A9080023204FF47A52074B1A60074B43F67F62B5
:10A9180018604FF0E0235A61072298611A61704766
:10A9280000ED00E04837002044370020684620F05A
:10A9380007018D4619B5FFF7B9FF1149114B086892
:10A94800D3E90042001942F10002C3E900020023E2
:10A958000B604FF47A530C4AD2E90041001BB0FB5C
:10A96800F3F043431B1941F10001C2E9003103F040
:10A97800E5FBF9F77FF8BDE819408546704700BF49
:10A9880044370020882D0020802D00202DE9F0413B
:10A99800DFF8E08099B1421C0BD14FF0E022136937
:10A9A80023F0010313614FF07F43C8F80030BDE87E
:10A9B800F081D8F80060012807DC00270BE0431C71
:10A9C800D8F80060F7D140F21740B0F5836FA8BF00
:10A9D8004FF48360471EEFF31185102383F3128829
:10A9E800BFF36F8FFFF762FF4FF0E023224C9969A6
:10A9F800D4E9002380184FF0000243F10003C4E9B2
:10AA080000031E4B1A601E4B1A68831A2ED44FF48B
:10AA18007A5C0CFB073303F579533F33B3FBFCF740
:10AA2800131A0CFB0733B3F5806F38BF4FF48063FC
:10AA3800144A934228BF13464FF0E022C8F800306A
:10AA4800013B90695361002381429361A1EB0003AC
:10AA580038BF9B19D4E900125B1842F10002C4E91F
:10AA6800003285F31188BFF36F8FA0E74FF480633E
:10AA7800E2E700BF48370020882D00204437002037
:10AA8800802D0020809DFF0038B5EFF3118510233D
:10AA980083F31288BFF36F8F084B1C68084B1B6841
:10AAA800E41AFFF703FF85F31188BFF36F8F4FF4A4
:10AAB8007A532044B0FBF3F038BD00BF882D002046
:10AAC800802D002038B5EFF31185102383F3128809
:10AAD800BFF36F8F044B1C68FFF7E8FE85F31188FE
:10AAE800BFF36F8F204438BD882D00202DE9F04139
:10AAF8004B4AD369916A13F00C0342D00C2B52D104
:10AB080001F0030101293CD00024D369444EB36A03
:10AB1800B56A03F00308B06AB36BC0F30010C3F35F
:10AB2800CC035843F6F708F9C5F30325B8F1020F2B
:10AB3800074605F1010542D0B8F1030F3FD0706B0D
:10AB4800C0F30800F6F7F8F84FF0645106463846A7
:10AB5800F6F74AF901463046F6F73EF84FF07E51CF
:10AB6800F6F73AF806462046F6F7E6F80446284689
:10AB7800F6F7E2F801462046F6F7EAF901463046CC
:10AB88003AE09168090254BFD2F8F4209268254946
:10AB980054BFC2F30332120F51F8224063B10C2B99
:10ABA800B4D0002408E0D26902F00C02042A35D09F
:10ABB800082B1D4C18BF00242046BDE8F081706B9F
:10ABC800C0F30800F6F7B8F84FF064510446384669
:10ABD800F6F70AF901462046F5F7FEFF4FF07E51D9
:10ABE800F5F7FAFF04462846F6F7A6F801460F4897
:10ABF800F6F7AEF901462046F6F7F6F8084B044694
:10AC0800586BC0F306600130F6F796F80146204607
:10AC1800F6F79EF9F6F7EAFA0446CDE7024CCBE7D9
:10AC2800000C0246BCD504080024F4000024744B30
:10AC380008B5FFF75BFF054B054A1B6A03F00F03D6
:10AC4800D35CD840034B186008BD00BF000C024617
:10AC58006C97050830060020F7B5044610B390F845
:10AC68009534056803F0FF021BB980F894242EF090
:10AC7800EFFE032384F89534324B20689D4204BFCD
:10AC88000023A3712FF00BF9237C251D8DF80030CC
:10AC980095E80E0020682FF0BEF8014630B1022377
:10ACA80084F895340125284603B0F0BD20682FF0BC
:10ACB800FCF80028F3D101270246267904F1140391
:10ACC800C1B28E4203F1240321D800210A4604F5BB
:10ACD8001573C8B2864203F1240326D8237C8DF865
:10ACE800003095E80E00206800F00AFC05460028B0
:10ACF800D5D10123607484F89534237B012B02D1CC
:10AD080020462FF074F820682FF0DCFACBE723F800
:10AD18000A0C43E9072203F8237C03F8241C03F8F0
:10AD2800202C43F8142C0130CAE743E9072203F822
:10AD3800232C03F8240C03F8202C43F8142C01319D
:10AD4800C7E700BF000004422DE9F04F066889B04C
:10AD5800044630462FF0F2FA0390002840F06E8146
:10AD680020682FF0BDFA002800F06881D6F808386E
:10AD78002068C3F30D23C4F8D4342FF0B1FA870741
:10AD880048BF226806F5006542BF536903F0020315
:10AD9800536120682FF0A4FAC0062CD52268936965
:10ADA80023F010039361D6F82080C8F34343022BA5
:10ADB80008F00F0740F0458147F6F07318EA030FD3
:10ADC80014D0242303FB0747C8F30A194A46304620
:10ADD800D7F860122FF018FAD7F860324B44C7F84A
:10ADE8006032D7F868324B44C7F8683222689369F2
:10ADF80043F01003936120682FF072FA010300F109
:10AE0800328120682FF06CFA42030DD520682FF0AC
:10AE180073FA27464FF0000A049006F5106B049B5E
:10AE28002068002B40F0EA8120682FF059FA0028AA
:10AE380013DA6B6823F001036B6094F8CC34012BB0
:10AE480040F084820021204684F8CC142EF0E2FFE2
:10AE58002268536903F00043536120682FF040FAD9
:10AE680001050AD5AB68DA0702D520462DF0E8FDC2
:10AE78002268536903F40063536120682FF030FAA5
:10AE8800030115D52268536903F00063536194F8F0
:10AE9800CC34002B40F05E820121236884F8CC1466
:10AEA8005B6D2046C3F38303C4F8D0342EF0B2FFA1
:10AEB80020682FF015FAC70433D56B68102123F0EA
:10AEC80001036B6020682FF01EF84FF67F3106F5FE
:10AED800106322790398824200F24082EB6943F0C2
:10AEE8000113EB61E37B002B00F05682D5F8843028
:10AEF80043F00B03C5F884306B6C43F00B036B64B1
:10AF0800D6F8003804F29C4223F4FE63C6F80038F1
:10AF1800A179206800F0EEFC2268536903F480539D
:10AF2800536120682FF0DCF9800416D520682FF0D3
:10AF380009FA20682FF032F8E0712768FFF778FEE9
:10AF4800E2790146384600F06BFA20462DF040FDC4
:10AF58002268536903F40053536120682FF0C0F945
:10AF6800010707D520462DF089FD2268536903F0B3
:10AF78000803536120682FF0B3F9020600F1178225
:10AF880020682FF0ADF9C3020CD5A046012706F5BD
:10AF980012692379BB4200F228822268536903F4BC
:10AFA8008013536120682FF09BF9870229D5234627
:10AFB800012206F53261207990421DD993F87C72FE
:10AFC8000868012F40F02782002880F22482D4F8F4
:10AFD800D4C48CEA1040C00700F11D8283F87B724C
:10AFE800B06940F08000B0617069000600F113821A
:10AFF8006B6843F400736B602268536903F40013B1
:10B00800536120682FF06CF9410007D520462DF0D8
:10B018000BFD2268536903F08043536120682FF0C9
:10B028005FF942070AD523685D686B0702D5204699
:10B038002DF000FD226853682B43536009B0BDE82A
:10B04800F08F062B7FF4D2AE0822304604F29C41E2
:10B058002FF0DAF8242303FB0747D7F86832C8F340
:10B068000A184344C0E620682FF03EF9A24600279C
:10B07800049006F53068049B2068002B3FF4C1AEAD
:10B08800049BDB0765D55FFA87FB59462FF03CF92F
:10B0980010F0010F81461ED00123C8F8083020683F
:10B0A80094F806C000F5306303EB4713BCF1010FB9
:10B0B800016C9A687BD112F0080F07D0B44881421E
:10B0C80009D9120407D54FF4004203E012F0200F0B
:10B0D80048D020229A6019F0080F0FD00823C8F82A
:10B0E80008302368AA49186C03F5306303EB47134B
:10B0F80088429A6870D82046FDF786FA19F0100F32
:10B108001CBF1023C8F8083019F0020F14D0736957
:10B118001A0642BF6B6843F480636B609AF8573233
:10B12800012B06D10023594620468AF857322EF0C3
:10B13800E4FC0223C8F8083019F0200F1CBF2023B4
:10B14800C8F8083019F4005F1CBF4FF40053C8F862
:10B158000830049B01375B08049308F120080AF1C2
:10B16800240A88E712F0280FB5D1DFF824C2614518
:10B1780001D91204A7D41A69DAF87432C2F3120298
:10B188009B1ACAF868326FB9D4F864222AB9012127
:10B1980004F29C4200F0AEFB04E0D4F860221A44AA
:10B1A800C4F8602259462046FDF7F4F993E7DFF822
:10B1B800E4C1614506D1110485D49006F2D5202258
:10B1C8009A60EFE7002FEDD1D4F86432002BE9D173
:10B1D800394604F29C42DDE7110448BF4FF40042AF
:10B1E800204648BF9A60FDF70FFAA179012985D159
:10B1F800206804F29C4200F07DFB7FE7049BDB079C
:10B2080040F19B805FFA8AF3194607932FF085F87F
:10B2180010F0010F804620D001216B6B0AF00F025D
:10B2280001FA02F223EA02036B63CBF80810A17952
:10B2380001290DD1D7E9072313443B62BAF1000F66
:10B2480006D1636A23B9206804F29C4200F052FBDD
:10B2580020465FFA8AF1FDF7BBF918F0080F1CBF0A
:10B268000823CBF8083018F0100F1CBF1023CBF8B8
:10B27800083018F0400F1CBF4023CBF8083018F0F6
:10B28800020F10D0514630462EF03DFEFB7D012BBB
:10B2980006D100232046FB755FFA8AF12EF02EFCBA
:10B2A8000223CBF80830236818F0800F059344D0A8
:10B2B800D7E909329A4240D8A3EB0208FB699845BE
:10B2C80028BF9846059B08F1030803F5106303EBB4
:10B2D8004A134FEA98080693069B9969D7E90932F9
:10B2E80089B2414527D393420BD80121059B0AF027
:10B2F8000F00D3F83428814022EA0102C3F8342829
:10B308001BE0A3EB0209FB69079A994528BF9946F8
:10B31800A37905980093396A1FFA89F32EF061FF23
:10B328003B6A09F103084B443B62BB6A4FEA980841
:10B338004B44BB62D0E79342D7D9049B0AF1010A78
:10B348005B08049324370BF1200B68E520462DF0A9
:10B3580086FB7DE520462DF073FBA9E599601A6808
:10B36800203322F4001243F8202CC3F8E811D3F854
:10B37800E02122F40012C3F8E021D3F8E02142F0E2
:10B388000062C3F8E021039A01320392A1E500BFED
:10B398000A30544F0A31544F6B6943F4005343F059
:10B3A8002B036B612B6943F00B032B61A8E501228A
:10B3B8002427B36904F2572023F08003B36106F50C
:10B3C8003263217991427FF6DBAD07FB02F1415CE4
:10B3D800012907D1196841F000611960196841F025
:10B3E8008041196001322033EBE798F83C30D9F8F6
:10B3F8000020012B09D1002A07DA67F07F012046D7
:10B4080088F83B30C9B22EF0A0FC013708F12408B7
:10B4180009F12009BDE5013224332031CBE500BF15
:10B42800022A4AD1274B284A0B44934239D9274B41
:10B43800274A0B44934236D9264AA1F57403A3F54B
:10B448001053934231D9244AA1F18373A3F5E743FA
:10B4580093422CD3214B224A0B44934229D9214BA6
:10B46800214A0B44934226D3204B214A0B44934252
:10B4780023D3204AA1F1B773A3F5585393421ED39F
:10B488001D4B1E4A0B4493422CBF06230723C26858
:10B4980022F47052C260C26842EA8323C36000206B
:10B4A80070470F23F3E70E23F1E70D23EFE70C2393
:10B4B800EDE70B23EBE70A23E9E70923E7E708238E
:10B4C800E5E700BF405327FFFF340C00401E1BFF79
:10B4D8003F420F007F4F120020D6130060B6E5FEF2
:10B4E8005FE3160000D3CEFE40771B00C05BB3FEBF
:10B4F800C091210020753800E05459FEE09C4100BD
:10B5080084B02DE9F041044607A880E80E00002326
:10B5180019469DF81C709DF8268003F140020133FE
:10B5280004EB82020F2B5160F7D104F50066B8F1E5
:10B53800000F46D1736843F002037360A36B23F4D2
:10B548000013A363236843F040032360236843F098
:10B5580080032360002503212046C4F8005E2EF0F6
:10B5680016FD102120462EF0CEFC014620462EF076
:10B57800EDFC0843C0B2401B356118BF012075615E
:10B5880004F51063F561002F46D0D4F80029AA42CB
:10B598001CDA4FF00062C4F8002900224FF67F3110
:10B5A8000135AF421A61996003F1200311D9D3F82C
:10B5B80000C0BCF1000F09DA4FF0904CC3F800C08E
:10B5C800EEE7A36B43F40013A363C3E700221A60FA
:10B5D800E3E7D4F8002B04F53063002A18DA4FF0BB
:10B5E8000062C4F8002B002200214FF67F3501329B
:10B5F800974219619D6003F120030DD9D3F800C06B
:10B60800BCF1000F05DA4FF0904CC3F800C0EEE72C
:10B61800002200211960E7E7336923F4807333615E
:10B628000023A3616FF0804363619DF81E301BB94E
:10B63800A36943F01003A361A2690B4B1343A361F1
:10B648009DF822301BB1A36943F00803A361B8F148
:10B65800010F01BFA36943F0804343F00403A361D2
:10B66800BDE8F04104B0704700383C8030B54A78F6
:10B678000B78012A00EB431300F5006029D1D3F8B9
:10B688000029002A0BDAD3F8002942F00062C3F837
:10B698000029D3F8002942F08042C3F80029012488
:10B6A8000A78C56B02F00F0204FA02F225EA0202D8
:10B6B800C2630978C26901F00F018C4022EA0402D2
:10B6C800C261D3F80019174A0A40C3F800290020BC
:10B6D80030BDD3F8002B002A0BDAD3F8002B42F048
:10B6E8000062C3F8002BD3F8002B42F08042C3F865
:10B6F800002B01240A78C56B02F00F0204FA02F24B
:10B7080025EA0242C2630978C26901F00F018C4040
:10B7180022EA0442C261D3F8001B034A0A40C3F874
:10B72800002BD4E7007833EC0078F3EFF7B54B78CB
:10B738000F78012B6C4EDFF8B4C100EB471440F0D2
:10B7480089800D6904F5106345BB1D6935401D618D
:10B758001D6945F400251D611D6905EA0C05012ACE
:10B768001D614CD1CA6902B15A610B79012B0CD108
:10B77800D0F8083813F4807FD4F800390CBF43F0B0
:10B78800005343F08053C4F80039D4F8003943F02B
:10B798000443C4F80039002003B0F0BD1D6905EA70
:10B7A8000C051D611D6935401D610D698E6867B9FD
:10B7B800B54288BF0E611D6945F400251D610D69FC
:10B7C8001E69C5F312053543C9E73544013DB5FB8C
:10B7D800F6F5474FD3F810C0AEB207EAC54545EABB
:10B7E8000C051D610D79012DE9D11D6925F0C045B4
:10B7F8001D611F69750705F0C0453D43DEE7D4F8B4
:10B80800003943F00443C4F800390B79012B0DD0FB
:10B818000B69002BBFD001230A78D0F8344802F016
:10B828000F0293402343C0F83438B4E7D0F80838FF
:10B8380013F4807FD4F800390CBF43F0005343F071
:10B848008053C4F8003900920B8A0A78C9682EF030
:10B85800C8FCA0E7D4F8105B04F5306305EA0C05D2
:10B868001D611D6935401D610E698D683FBB06B1BC
:10B878000D610D621E69C5F3120535431D611D6911
:10B8880045F40025012A1D6102D1CA6802B15A6136
:10B898000B79012B0CD1D0F8083813F4807FD4F839
:10B8A800003B0CBF43F0005343F08053C4F8003B07
:10B8B800D4F8003B43F00443C4F8003B6BE7002E88
:10B8C800D8D02E44013EB6FBF5F6B6B275430D62EC
:10B8D800074D1F6905EAC6453D431D610D6A1E698E
:10B8E800C5F312053543CDE7FFFF07E00000F8FF79
:10B8F8000000F81F30B5114C056C00F53063A54207
:10B9080003D9D0F8004B002C16DB00241C611C69FD
:10B91800012944F400241C611C6944F018041C61CA
:10B928001C6944F0C0441C6101BF5A61D0F8003B57
:10B9380043F08023C0F8003B002030BD0A30544F4C
:10B94800A8B1304BDA6802F44032B2F5403F10D16A
:10B958002D4B984251D92D4B984250D92C4B984297
:10B9680035D92C4B984216D92B4B984231D9012006
:10B978007047DA6802F44032B2F5003F0DD1274B28
:10B9880098423AD9264B984239D9264B98421ED923
:10B99800254B9842EBD803201CE0DB6803F44033C6
:10B9A800B3F5803F0AD1214B984226D91B4B9842C8
:10B9B80025D91F4B98420AD9194BEAE71D4B9842E3
:10B9C8001BD91D4B98421AD91C4B9842CFD802203C
:10B9D80000E004201A4A136823F00F03034313609E
:10B9E800136803F00F0398420EBF0346136803F071
:10B9F8000F03C01A18BF012070470020EAE7012092
:10BA0800E8E700BF000802460048E8010090D003BC
:10BA180000D8B8050020A1070068890940787D0191
:10BA280080F0FA02C068780400E1F50520BCBE0089
:10BA380060343C0200127A000024F40000366E01E3
:10BA48000020024010B50A46044619B1024B0021F5
:10BA58001B68984710BD00BF34060020034600202D
:10BA6800094AC3E900009A6002F18832DA6002F1FB
:10BA78002942A2F59612A2F68B621A61A2F18832C7
:10BA88005A61024A9A61704701234567F0E1D2C3BF
:10BA98002DE9F04F4B68AFB01BBA08930B69D1F88A
:10BAA80000E093FA83F84B698E6893FA83FA8B69FE
:10BAB800CD681BBA0A93CB6901901BBA12930B6A23
:10BAC8009EFA8EFE93FA83FB4B6A36BA1BBA0B9327
:10BAD8008B6A2DBA1BBA0C93CB6A1BBA0D930B6BEE
:10BAE8001BBA0E934B6B1BBA03938B6B1BBA049355
:10BAF800CB6B1BBA059383680F93C36802930369E2
:10BB08000F9906934369029F10938369109A1393C0
:10BB1800069B83EA0200029B18405040DF4B139AB1
:10BB280003EBB7071A4402EBF16210440299069A34
:10BB3800704482EAB1020F992F440A4006998EEAAE
:10BB4800060E4A4010998EEA0B0E19440A440899C9
:10BB58000A440F9902EBF0624FEAB10C02998CEAA1
:10BB6800B104044084EAB1040699194431440C44F0
:10BB78008CEAB001114004EBF26481EA0C014FEA4F
:10BB8800B202394482EAB00727409C4401EBF461D1
:10BB9800C44482EAB40987EAB007674409EA01099C
:10BBA8000AEB030C07EBF1670CEBB00C4FEAB101A1
:10BBB8000A9889EA0209E14481EAB40C0CEA070C04
:10BBC800184410448CEAB40C129A09EBF7698444BF
:10BBD80081EAB70000EA09001A4402EBB4024840BF
:10BBE80010444FEAB9020CEBF96C82EAB7040BEB8C
:10BBF800030904EA0C0484EAB704894404EB090144
:10BC0800DDF82C9000EBFC6082EABC040440994407
:10BC180001EBF06109EBB7094FEAB0000C9F544003
:10BC28004C4480EABC0909EA01091F44174489EA1F
:10BC3800BC090D9A04EBF164B94480EAB1072740C6
:10BC48001A4409EBF46902EBBC024FEAB404DDF8CC
:10BC580038C04740174484EAB10202EA09029C440A
:10BC6800844482EAB1026244DDF80CC007EBF9674C
:10BC780084EAB90038409C4402EBF7620CEBB10C43
:10BC88004FEAB70704996040604487EAB90C0CEAA8
:10BC9800020C194421448CEAB90C059C00EBF260B3
:10BCA8008C4487EAB20101401C4404EBB904794092
:10BCB8000CEBF06C214401EBFC6903994FEAB000EE
:10BCC8008EEA010103EBF17E07910899BE4481EAEF
:10BCD80005070B9980EAB2044F40049904EA0C0462
:10BCE800794084EAB204744403EBF17E0EEBB20EA1
:10BCF8000C9A86EA080680EABC075640059A07EAC5
:10BD0800090756404740774403EBF67E86440D9872
:10BD180085EA0A054540079804EBF96485EAF0705E
:10BD28001190119D08914FEAF0704FEAB90107EBA5
:10BD3800F467159081EAB400384003EBF57303EB20
:10BD4800BC03484018440A9B4FEAF67288EA030885
:10BD58000E9B149288EA0308089B81EABC0288EAD1
:10BD6800F3730993099D4E4B224082EABC0203EB10
:10BD7800F57C8C441299039D724402EBF7628AEABF
:10BD880001014FEAB70787EAB409694081EAF67109
:10BD980089EA0209E14403EBF17C0CEBB40C0A9C40
:10BDA80000EBF26084EA0B08049C87EAB20A88EA8E
:10BDB8000408119C8AEA000A88EAF478E24403EB52
:10BDC800F87C129DBC440B9F09EBF06985EA070ECD
:10BDD800059D4FEAB0008EEA050E099D4FEAF874FA
:10BDE8008EEAF57E03EBFE7716944FEAFE7580EA3D
:10BDF800B20407EBB2070C9A1295079D84EA09046E
:10BE08008BEA02020AEBF96A644482EAF57280EA74
:10BE1800B90C04EBFA6482EAF1728CEA0A0C4FEA74
:10BE2800BA0A0A9203EBF27BBC440B9A8AEAB90776
:10BE38000D9D6740834407EB0B0082EA0507089ACB
:10BE48000E9D87EAF27787EAF8720B9203EBF27B92
:10BE58000C9A0BEBB90B82EA050989EAF67686EAB1
:10BE6800FE760CEBF46C8AEAB4074FEAF6750D9A85
:10BE7800179587EA0C07039D5F4403EBF67BD344D1
:10BE880082EA050A119A00EBFC608AEAF2754FEA29
:10BE9800BC0C0A9A8CEAB40904E000BF9979825A6A
:10BEA800A1EBD96E85EAF27589EA000907EBF0671C
:10BEB8008CEAB00AD94403EBF57B4FEAF5728AEABB
:10BEC800070A0BEBB40B0D920AEB0B040E9ADDF884
:10BED80010A009EBF76982EA0A0A099A4FEAB7073C
:10BEE8008AEAF27A0B9A04EBF9648AEAF27203EBB3
:10BEF800F27B87EAB00A8AEA090AE3440C920AEB61
:10BF08000B0C039ADDF814A00CEBF46C82EA0A0A15
:10BF18008AEAF17A8AEAF67203EBF27B039287EAFD
:10BF2800B90A049A0BEBB00B07988AEA040ADA44B8
:10BF38004FEAB40B82EAF07484EAF87484EAF57480
:10BF48008BEAB90003EBF4784FEAF47280EA0C004C
:10BF5800B8440E9200EB0807059A08980AEBFC6AA9
:10BF680082EAF0700C9A80EAFE7080EAF2708BEA3E
:10BF7800BC0E03EBF0784FEAF07208EBB9088EEAD2
:10BF88000A0E1192C644149ADDF81C8007EBFA6772
:10BF980082EAF8780A9A4FEABA0A88EAF278039AA3
:10BFA8000EEBF76E88EAF27203EBF2798AEABC08C4
:10BFB800D94488EA07080492C844159ADDF8209005
:10BFC80008EBFE6882EAF9790B9A89EAF27989EA3C
:10BFD800F47203EBF27B8AEAB70989EA0E090BEBE4
:10BFE800BC0B059209EB0B0C149ADDF824904FEA70
:10BFF800BE0E82EAF97989EAF67989EAF0794FEA98
:10C00800F97214928EEAB706159A03EBF97B86EA61
:10C018000806D34406EB0B0A82EAF176049A86EA0C
:10C02800F57686EAF2764FEAF67203EBF67B15921E
:10C038000BEBB70B169A099F0CEBF86C82EAF777B3
:10C048000C9A8EEAB80587EAF277059A85EA0C0514
:10C0580087EAF27207925D4403EBF27B129A0AEBCD
:10C06800FC6A82EAF1714FEABC0C039A8CEAB807C1
:10C07800F34481EAF27187EA0A075F4481EAF97BAF
:10C0880005EBFA658CEABA0E03EBFB7101EBB8011C
:10C098008EEA050E169A8E440A9907EBF56782EA2E
:10C0A800F17181EAF47484EAF6744FEAF47203EBEE
:10C0B800F4781692E044129ADDF82CC04FEAB505E0
:10C0C80082EAFC7C079A8CEAF07080EAF2700EEB48
:10C0D800F76E85EAB70C03EBF0734FEAF07203EBE7
:10C0E800BA038CEA0E0C12929C440A9A179B85EAB2
:10C0F800BA0183EAF272049B794082EAF37282EA17
:10C10800FB730893089AE74B414401EBFE6103EB8C
:10C11800F272154441EABE020CEBF16C01EABE086A
:10C1280002EAB70205EBFC6542EA08022A44DDF898
:10C138002C800D9D85EAF875DDF8148085EAF87580
:10C1480085EAF4754CEAB108099508EABE080CEAD4
:10C15800B10548EA0505DDF8248003EBF87808EB1B
:10C16800B70805EB0807179DDDF8308007EBF26785
:10C1780085EAF87888EAF97888EAF0784FEAF87575
:10C188000B9503EBF87505EBBE0E42EABC0502EA17
:10C19800BC0905EAB10545EA09050EEBF76EAE44A0
:10C1A800DDF80C900D9D85EAF97585EAF676089D0F
:10C1B80047EAB20986EAF5764FEAF6750D9509EA77
:10C1C800BC0907EAB20549EA050503EBF67909EB6C
:10C1D800B1094D440E99DDF8309005EBFE6581EA12
:10C1E800F971DDF81C9081EAF971DDF8249081EA93
:10C1F800F9710A9103EBF17101EBBC0C4EEAB7013E
:10C208000EEAB70901EAB2010CEBF56C41EA090143
:10C218006144DDF80C90DDF844C08CEAF97C8CEAC6
:10C22800FB7C8CEAF87C45EABE09CDF80CC009EA2B
:10C23800B70905EABE0C49EA0C0CDDF80C9003EBD3
:10C24800F97909EBB209CC440E9ADDF810900CEBA1
:10C25800F16C82EAF97282EAF47484EAF6744FEABD
:10C26800F4720E9203EBF47202EBB70741EAB502DF
:10C2780001EAB50902EABE0242EA090207EBFC67D5
:10C288001744DDF81490119A82EAF97282EAF07084
:10C298000A9A4CEAB10980EAF2704FEAF0721192F8
:10C2A80009EAB5090CEAB10249EA020203EBF0799E
:10C2B80009EBBE094A44DDF850E0DDF8109002EBC6
:10C2C800F7628EEAF97EDDF820908EEAF97EDDF8D5
:10C2D8000C908EEAF97E03EBFE7909EBB50947EA83
:10C2E800BC05CDF810E005EAB10507EABC0E45EA41
:10C2F8000E0509EBF269A944DDF814E0159D85EAFD
:10C30800FE75DDF824E085EAFE7585EAF475059585
:10C3180042EAB70505EABC0502EAB70E45EA0E0E81
:10C32800059D03EBF57505EBB105AE441499079D22
:10C338000EEBF96E81EAF57181EAF87888EAF0780F
:10C348004FEAF871149103EBF87101EBBC0C49EA60
:10C35800B20109EAB20501EAB70129430CEBFE6C08
:10C368008C4415990EEAB90581EAFB7A04998AEAA0
:10C37800F67A8AEAF17A4FEAFA7115914EEAB9012A
:10C3880001EAB2010D4303EBFA7101EBB701079E15
:10C398000D44169905EBFC6581EAF6710A9E81EA5F
:10C3A800F671059E81EAF67103EBF17707EBB207A8
:10C3B8004CEABE02079102EAB9020CEABE010A433E
:10C3C80007EBF5671744129A05EABC0182EAFB7B82
:10C3D800039A089E8BEAF27B45EABC028BEAF87B5B
:10C3E80002EABE02114303EBFB7202EBB9021144ED
:10C3F800169A01EBF76182EAF67686EAF47686EA1F
:10C40800FA764FEAF672169203EBF67447EAB5022B
:10C4180004EBBE0402EABC0207EAB50E42EA0E02C9
:10C4280004EBF1641444DDF824E0129A82EAFE7207
:10C4380082EAF070079A41EAB70E80EAF2720C922B
:10C448000C984FEAF27212920EEAB50E01EAB702A0
:10C458004EEA020203EBF07E0EEBBC0E089802EBEC
:10C468000E0C0B9A0CEBF46C82EAF072049804EA56
:10C47800B10E82EAF07282EAFB72089203EBF27262
:10C4880002EBB50244EAB10505EAB70545EA0E052F
:10C4980002EBFC622A440D98099D0CEAB40E80EA6E
:10C4A800F57501E0DCBC1B8F059885EAF07585EA17
:10C4B800F6704CEAB40505EAB10545EA0E0E03EB41
:10C4C800F07505EBB7050990AE44DDE90A5080EA3E
:10C4D800F5750C9885EAF87585EAF0754FEAF577F1
:10C4E800179703EBF57707EBB10742EABC010EEBB0
:10C4F800F26E02EABC0801EAB40141EA080107EB5E
:10C50800FE670F4403980D994EEAB20981EAF0716B
:10C51800089881EAFA7181EAF07109EABC090EEA21
:10C52800B20803EBF1734FEAF17049EA080803EB2C
:10C53800B4030D9008EB03040A980E9B4FEABE0A59
:10C5480083EAF07307988AEAB20E83EAF0730998CF
:10C558008EEA070E83EAF0730A930A98DF4B04EB1E
:10C56800F76403EBF07808EBBC081198DDF80CC011
:10C57800C64480EAFC7C8CEAFB7C8CEAF57003EB11
:10C58800F07C0B900CEBB20C04980E9A8AEAB70870
:10C5980082EAF07989EAF67989EAF1790EEBF46EA4
:10C5A8004FEAF97288EA04084FEAB4040E92E044AC
:10C5B80003EBF97284EAB70C52448CEA0E0C059826
:10C5C8009444119A08EBFE6882EAF0760C9A0CEB18
:10C5D800F86C86EAF2760A9A86EAF2764FEAF672FA
:10C5E8000C9203EBF67084EABE0200EBB70082EA15
:10C5F8000802149F02444FEAB800DDF8108080EA70
:10C60800BE0A87EAF877DDF820808AEA0C0A87EA0A
:10C61800F877DDF82C8002EBFC6287EAF8774FEABE
:10C62800F777039719971F442744BA44159C059F29
:10C638000AEBF26A84EAF774099F84EAF77484EAD9
:10C64800F9744FEAF4740494049F1A941F4480EA1E
:10C65800BC0407EBBE0754404FEAB20205923C44C3
:10C66800149A079F04EBFA6482EAF77888EAF57867
:10C67800059A88EAF6784FEAF87882EABC0508EB6A
:10C688000307159A074485EA0A053D4482EAFB77C1
:10C6980087EAF1770399059A4F404FEAF77782EADC
:10C6A800BA00F91801EBBC016040169A08440799D2
:10C6B80005EBF46582EAF1710A9A4FEAB40481EA5B
:10C6C800F271049A84EABA0E51404FEAF171059A60
:10C6D80001EB030C94448EEA050E129AE644DDF849
:10C6E8002CC082EAFB7282EAFC7282EA08024FEAF4
:10C6F800F27200EBF56084EAB50C02EB030B0BEB6E
:10C70800BA0B8CEA000CDDF858A0DC44DDF820B048
:10C718000EEBF06E8AEAFB7A8AEAF97A8AEA070A65
:10C728004FEAB0004FEAFA79CDF81490CDF87C9032
:10C7380080EAB50A9944A1448AEA0E0A129CCA44BE
:10C74800DDF824900CEBFE6C84EAF97484EAF67444
:10C758004C404FEAF4740794209480EABE061C44C7
:10C7680004EBB50486EA0C062644179C039D84EA6C
:10C77800FB746C4054400AEBFC6A4FEAF4744FEACD
:10C78800BC0C8CEABE09E518054489EA0A09CDF80B
:10C798006C801C971D911E92A9442194099D0D98A7
:10C7A80006EBFA6680EAF570049D09EBF6696840C5
:10C7B800059D68404FEAF0708CEABA0500EB030B60
:10C7C8000BEBBE0B7540DDF85CE05D44DDF828B08E
:10C7D8004FEAB6068EEAFB7E8EEA080EDDF81C806C
:10C7E80005EBF9658EEA080E4FEAFE7E0EEB030BA9
:10C7F80086EABA08E34488EA0908DDF834C0D84470
:10C80800DDF82CB008EBF5688CEAFB7C8CEA070CA9
:10C818008CEA040C4FEAFC7786EAB90407EB030CB0
:10C828000CEBBA0C6C40DDF828A06444DDF838C085
:10C838004FEAB5058CEAFA7C8CEA010C8CEA000C0C
:10C848004FEAFC7101EB030CB4440C9E229086EA7B
:10C85800FB76564086EA0E0685EAB9004FEAF67678
:10C8680004EBF864269685EAB80280EA08001E44BC
:10C8780006EBB9066044624000EBF460324402EB18
:10C88800F06C039E0E9A4FEAB4045640059A24971A
:10C8980056407E404FEAF67627961E440C9A2E4460
:10C8A800049D84EAB8075540079A474055404D40D3
:10C8B8004FEAB00018954FEAF5752591289584EA56
:10C8C80000011D4481EA0C01374405EBB80507EB6C
:10C8D800FC674B190F994FEABC0201E0D6C162CA46
:10C8E80003EBF763CDF88CE02D942A972C902993CD
:10C8F8002B920B4401998B60029B1F44069BCF60CF
:10C908001A44109B0A611844139B48611C448C61AB
:10C9180018A85821FFF796F800202FB0BDE8F08F2F
:10C9280003460846C1B9C3E910110D4A0D49DFF89D
:10C9380038C0C3E912120D4A0D49C3E914C20D4AA1
:10C94800C3E916120C4A1A6602F17452A2F52302C0
:10C95800A2F692425A6670476FF07300704700BFA4
:10C9680085AE67BB67E6096A72F36E3C3AF54FA578
:10C978007F520E518C68059BABD9831F2DE9F04F70
:10C988000446CFB0039100F1480346AD00F16806B4
:10C998002A4618685968083303C2B3421546F7D1C6
:10C9A800DDE94883DDE94B96DDE946154FF0000CDB
:10C9B80001933E4BDDF834B14A9804AA0293BCF1C6
:10C9C8000F0F5BD8039B53F82C301BBA4FEAF02E9D
:10C9D80086EA0907DDF808A08EEAB01E07408EEA4D
:10C9E800706E774077445AF804EB936077443B4481
:10C9F80045EA010E4FEA7137CDF808A087EAB1077A
:10CA08000EEA080E05EA010A4EEA0A0E87EAB1574D
:10CA180077440CF1010CDDF804E05B44BCF1400FF5
:10CA28009E44B3463B4402F10402CDF804801ED173
:10CA3800CDE94C96CDE94AE0CDE94858CDE94631F3
:10CA4800CDE9043745A904F14403643453F8042FAD
:10CA580051F8040FA34202441A60F7D104A84FF416
:10CA68009471FEF7EFFF00204FB0BDE8F08FA846A5
:10CA78004E460D46814619467046A0E7136852F89F
:10CA880034AC4FEAF34E8EEA734E52F8387C8EEA95
:10CA9800932E52F8143C3B444FEABA4787EAFA17F8
:10CAA800734487EADA073B4490E700BFFCD50408E3
:10CAB80010B50446F6F792FA03480121034A2AF012
:10CAC80007F920462DF0B2FDCCCE04087C97050866
:10CAD8002DE9F84304460D4600AFEFF31188102303
:10CAE80083F31288BFF36F8F0428294A98BF294B14
:10CAF800E9468AB09668117C98BF53F820306A4698
:10CB080088BF254BC2E9073140F20133234893849B
:10CB1800234BC2E9050442F8103F00234FF431517A
:10CB28002048F6F72BFBCD4645B1EB69C3F3080364
:10CB380023B101211C4A1B482AF0CAF82EB13046FD
:10CB48002DF0FBFF08B1037803B91848E9468AB00D
:10CB58006A46174BD061C2E9053640F201331384A7
:10CB6800144B42F8103F00234FF411510D48F6F7CB
:10CB780005FB2946CD462046FFF79AFF88F3118822
:10CB8800BFF36F8F3046F7F7E1F9BD46BDE8F8838C
:10CB98004C370020FCD604088B970508A197050898
:10CBA80005000001CCCE0408C99705089997050827
:10CBB800EA9705080400000138B50A4B53F82040ED
:10CBC800013053F82050A54200D838BD606830B114
:10CBD800037EDB0701D42DF006FD0834F3E7236854
:10CBE8009847FAE710D70408012270B5294B0320AB
:10CBF80086B01A70FFF7E0FF01F028FC0420FFF769
:10CC0800DBFF254C254D2646AE4204F1300410D3F7
:10CC180000F072FF204C224EAC4226D300F080FF79
:10CC280029F0C5F81F4A938923F00103938106B0C0
:10CC380070BD54F80C3C059354F8103C049354F818
:10CC4800143C039354F8183C029354F81C3C019389
:10CC580054F8203C009354E90A2354E90C0100F0ED
:10CC680035FD54F8303C5E65CDE7D4E90A23B3F1CD
:10CC7800FF3F08BFB2F1FF3F05D052EA0301206829
:10CC880003D101F01FF83034C6E73146183001F0FF
:10CC9800C5F9F8E73E3F0020C8CC0408F8CC0408E2
:10CCA80023AC0308302E0020A02370B5134E0122B8
:10CCB80003FB0066002386B0CDE904230F2201930D
:10CCC800CDE9023214234FF4A0720D4D0D4903FB38
:10CCD8000055044602FB00110B4B3046009500F04E
:10CCE800F5FC337C2C7423F004033374074B0134B4
:10CCF80003EBC423EE606B6006B070BD902D00207E
:10CD08004C370020C05E0020BDA70308C056002095
:10CD1800BFB50020FFF750FF294B03F5006282F3EF
:10CD2800088883F30A880024F023264D264F85F8C7
:10CD38002230EC772C766C76AC7685F820406B6ADE
:10CD480043F4E0236B62F7F7BBF8F7F707FA4FF005
:10CD5800FF33AB62EB62F7F7ABFBF7F729FAF6F7AD
:10CD6800A3F81A4800F034FDF5F750FF0120FFF74B
:10CD780023FF0220164DFFF71FFF00F005FF154B9C
:10CD880015495D61154B45F6E06205930123284678
:10CD9800CDE90343CDE901443B46009400F096FCFD
:10CDA80006462A7C284622F004022A742DF001FF48
:10CDB8002046FFF779FF3A4631462846F7F7ACF99F
:10CDC800C056002000ED00E0F1CB0008D02E002076
:10CDD800302E00204C37002000600020E87C050839
:10CDE80038B5064C064DAC4201D3002038BD20466C
:10CDF800D4E901122DF064FC1434F4E7AC0F0020E0
:10CE0800C00F002030B5054B85B0DDE90845029319
:10CE1800CDE900452DF012FC05B030BD8B6203084A
:10CE2800002038B5054C064DAC4200D338BD20462D
:10CE38002DF06AFC0028F9DB1C34F5E7900F002080
:10CE4800AC0F002073B50C46EFF31181102585F364
:10CE58001288BFF36F8FC5685DB125602B68C3600A
:10CE6800836901338361002081F31188BFF36F8FD9
:10CE780011E052EA030603D16FF00B002560F3E7D7
:10CE8800CDE900230246083000F07CFD18B9034BB9
:10CE98009B685B69236002B070BD00BF4C370020FF
:10CEA8002DE9F34104460E469DF8200004F10808D8
:10CEB800EFF31187102181F31288BFF36F8F256A72
:10CEC800E1688D4247D22568AC4218D0BDB12846EA
:10CED8002DF07BFC05F118002DF06AFF3146A268A1
:10CEE80068693FF0CFFB00232846C5F898302DF03D
:10CEF80060FE4046394600F0D9FD002038E0A268BF
:10CF0800D8B13146E0693FF0BDFBE369A26813443C
:10CF18006269E361934201D12369E361236A1021C5
:10CF28000133236204F124002EF021F80028E0D117
:10CF380087F31188BFF36F8F1AE0A16923699942BB
:10CF480008BF6369314608BFA361A069801AA06160
:10CF58003FF098FBE2E752EA03010CD0074940464C
:10CF680089684E61CDE900233946224600F00AFD62
:10CF780002B0BDE8F0816FF02200D9E74C370020FD
:10CF8800F7B50446084604F10807EFF311861021A7
:10CF980081F31288BFF36F8F216A00293AD0A26803
:10CFA800A1693FF06FFBA369A26825681344626911
:10CFB800A361934204BF2369A361236AAC4203F1CE
:10CFC800FF33236234D02846002D32D02DF0FDFBEC
:10CFD80005F118002DF0ECFEA2686969E0693FF0E0
:10CFE80051FBE369A268284613446269E3619342EE
:10CFF80004BF2369E361236A013323620024C5F86F
:10D0080098402DF0D6FD3846314600F04FFD2046B9
:10D0180003B0F0BD52EA030110D00A49896848619B
:10D02800CDE9002331462246384600F0ABFCEFE755
:10D03800002086F31188BFF36F8FE9E76FF02200B5
:10D04800F7E700BF4C3700202DE9F34104461746A7
:10D058001E46EFF31188102383F31288BFF36F8FF6
:10D06800C368314A7BB180689168884219D057EA11
:10D07800060318D188F31188BFF36F8F6FF00F0084
:10D0880002B0BDE8F081916891F90E100133E360B8
:10D0980093682161A36088F31188BFF36F8F002024
:10D0A800EEE72169F2E790F90E3091F90E109942F6
:10D0B800A8BF19468B422DDD2DF0F1FB054622460F
:10D0C8004146CDE90076194800F05CFC0028E6D01E
:10D0D800EFF31186102383F31288BFF36F8FA068D4
:10D0E800D0B1236821699C420AD04BB193F90E3024
:10D0F8009942A8BF19466FF07F039942B8BF1946F5
:10D108002DF0CDFB40B13146084800F0CFFC6FF060
:10D118000A00B5E70025D2E7002DF4D186F311887F
:10D12800BFF36F8FF3E700BF4C3700203F3F00206D
:10D13800F8B583680546002B40D0234A926893428D
:10D148003FD1C368012B03D9013BC3600020F8BD60
:10D15800EFF31187102383F31288BFF36F8F0169F0
:10D1680080682DF09CFB2C68AC4207D10023C5E9F0
:10D17800023387F31188BFF36F8FE7E7002CF5D0F0
:10D18800D4E90032002613605A60237CC4E90066A3
:10D1980023F002032374A66004F118002DF008FEA2
:10D1A800AC6094F90E3020462B61C4F898602DF0DD
:10D1B80000FD3946054800F079FCC7E76FF0150017
:10D1C800C5E74FF0FF30C2E74C3700203F3F002053
:10D1D80037B51146EFF31185102282F31288BFF399
:10D1E8006F8F04689CB12368426823F0030394425C
:10D1F800036008BF4360012120462DF0DDFB044693
:10D2080085F31188BFF36F8F204603B030BD51EA14
:10D218000302F5D000F10802CDE9001310462946B3
:10D2280000F0B0FB0028EFD1014B9B685C69EBE78D
:10D238004C37002070B5EFF31186102383F3128862
:10D24800BFF36F8F0468A0421BD0D4B1D4E9003279
:10D25800002513605A60237CC4E9005523F00203BB
:10D268002374A56004F118002DF0A2FD2046C4F82F
:10D2780098502DF09EFC3146BDE87040094800F0FA
:10D2880015BCD0E902329A4218BF013302218360EB
:10D2980010302DF06CFE0028EDD186F31188BFF315
:10D2A8006F8F70BD3F3F002013B5EFF3118110243D
:10D2B80084F31288BFF36F8F846844B1013C8460A3
:10D2C80081F31188BFF36F8F002002B010BD52EABE
:10D2D800030406D181F31188BFF36F8F6FF00F003D
:10D2E800F3E7CDE900230246014800F04BFBECE7E9
:10D2F8003F3F00202DE9F8430546EFF3118810233E
:10D3080083F31288BFF36F8F00266FF00A09374640
:10D318002C68A54216D0ACB1D4E9003213605A602B
:10D32800237CC4E9007723F002032374A76004F187
:10D3380018002DF03DFD2046C4F898902DF039FCDA
:10D348000126E5E700230221AB6005F110002DF06E
:10D358000EFE30B92EB988F31188BFF36F8FBDE880
:10D36800F8834146BDE8F843014800F09FBB00BF81
:10D378003F3F00202DE9FF41044610274E4EEFF3B2
:10D38800118887F31288BFF36F8FD4F8A450F5B9CA
:10D39800022104F1BC002DF050FB002868D004F1F4
:10D3A800B4050022012128462DF097FC0028F8D169
:10D3B80000234FF0FF3202934FF0FF334146CDE98F
:10D3C80000233E4804F1AC0200F048FDD7E7D4F84A
:10D3D800A8202B689542C4F8A43008BFC4F8A83028
:10D3E800D4F8BC3043F00203C4F8BC30EB6823F037
:10D3F800040343F00103EB606B6888F31188BFF303
:10D408006F8F28469847EFF3118887F31288BFF388
:10D418006F8FEB68D80623F0010236D4EA60EB6818
:10D428009A0716D5306823F00203EB6088B1002113
:10D43800036870B14268954235D1036869BB726868
:10D448003360824200D17360002340F8083BFFF745
:10D45800F1FED4F8BC3023F00203C4F8BC3088F3E2
:10D468001188BFF36F8FDB0589D400F0ABFB86E72B
:10D47800D4F8BC30D9069BD5C4F8BC0088F3118811
:10D48800BFF36F8F04B0BDE8F08123F01103EB60A8
:10D4980005F11000FFF7CEFEC1E70B607368834209
:10D4A80008BF7160D0E723B11A68014618461346D1
:10D4B800BFE71A46F9E700BF703700203F3F00205A
:10D4C800F8B5C36804469A070F46C3F340062ED43E
:10D4D8005B071CD40B680BB983680B60E368DD0736
:10D4E80042BFA36802263B603D6858BF0126002D55
:10D4F8003CD0204B9A68D5F8A0309A420AD0D5F88B
:10D50800BC30D807C3F3800214D46FF0120600238E
:10D518003B6025E02DF008FBD5F8BC300028F0D1A1
:10D52800D907C3F3C002F0D552B15B0708D46FF036
:10D538000F06ECE7002AFAD1C3F3C003002BF6D19B
:10D5480000232360D5F8A83063B9C5E929442846E3
:10D558002DF08DFAE36843F00403E3603B68A360B1
:10D568003046F8BD1C60C5F8A840F0E76FF0150616
:10D57800CDE700BF4C370020014601482DF0B8BA6E
:10D58800902F0020F0B50446002089B0C4E9290096
:10D598000E9D04F1AC00C4E92B0004F1B400C4E909
:10D5A8002D0055B32879002840F2011008BF01204A
:10D5B800C4F8BC0000204FF0FF364FF0FF37CDE92C
:10D5C8000330CDE90100CDE9066720460C4B0094F5
:10D5D80000F0D2F855B1296811B120462DF0AAFA09
:10D5E8006B791BB1A38943F00103A381204600F0A6
:10D5F80069FBC4F8A04009B0F0BD0120D8E700BF1E
:10D608007DD3000837B501900846EFF31184102147
:10D6180081F31288BFF36F8FC16811F01E0F16D106
:10D6280053EA020508D101A9FFF74AFF84F31188DC
:10D63800BFF36F8F03B030BD41F00801C16001999D
:10D6480010308161034900F0E9FC0120EEE7002079
:10D65800ECE700BF85AA030801460148FFF7D2BFDF
:10D66800902F0020F7B50C4616461D460190EFF3A3
:10D678001187102383F31288BFF36F8F08462DF0AC
:10D68800E7F955EA060309D1204601A9FFF718FF73
:10D6980087F31188BFF36F8F03B0F0BDE36832469C
:10D6A80043F00803E360019B0449A36204F11000FE
:10D6B8002B4600F0B3FC0120EAE700BF85AA030867
:10D6C80001460148FFF7CEBF902F00202DE9F04F0B
:10D6D800984685B000F15803C0E91633129B00261E
:10D6E80083810423073222F0070A0374119B01EB9C
:10D6F8000A090F46C0E90666494686608373C67301
:10D708000446DDF838B0F6F795F9109BC51D25F0ED
:10D718000705C4F88850C4E9207A02930F9BA9EB47
:10D728000505CDE900B32A46434639462046F6F7B3
:10D73800D7FC0F9BC4E91B8B6367109B6665A367C7
:10D74800EFF31182102383F31288BFF36F8F094B15
:10D75800196A1C62E16782F31188BFF36F8F9B68B7
:10D768000BB1D3F88C302846C4F88C3005B0BDE82E
:10D77800F08F00BF4C370020F0B5002587B0059525
:10D78800109DDDE9127604950F9D044603950E9DC4
:10D7980002950D9D01950C9D0095FFF797FFB6F139
:10D7A800FF3F08BFB7F1FF3F05D056EA070305D191
:10D7B800204600F087FA204607B0F0BD3A463346C7
:10D7C80004F11800014900F029FCF4E723AC030830
:10D7D8000123037483810023C0E92033C0F88C300F
:10D7E800014B9860704700BF4C3700206FF00A016A
:10D7F800094A9368C3F898100849C3F894004B681D
:10D8080043F080534B60002383F31188BFF36F8F7D
:10D818009368D3F8980070474C37002000ED00E07B
:10D8280070B590F91020037C002A36DBD90634D174
:10D838001B4C63F07F032246037452F8183FE169DA
:10D84800934207D1C0E900210860E06111E09942E4
:10D85800F8D01B68002BF5D090F90E5093F90E60A4
:10D86800B542F4D0AE42F2DD5968C0E90031086033
:10D878005860A569954200D005B9E568A3681A7C87
:10D88800D20604D1DA897F2A01D9AA6932B1AB421A
:10D8980002D0284600F024FB656170BD6361FCE797
:10D8A8004C37002038B590F910200146002A037C37
:10D8B80004DA03F07F0303742DF041F90D4D2A4675
:10D8C80052F8184FAB68944200D004B9EC688B4208
:10D8D80007D01A7CD20604D1DA897F2A01D9A26935
:10D8E8002AB1A34202D0204600F0FAFA23466B611F
:10D8F80038BD00BF4C370020B3F1FF3F08BFB2F17D
:10D90800FF3F03D00249183000F088BB704700BFC2
:10D9180023AC030838B5194CA168E0690B6881424B
:10D9280014BF1A46002249680B605960A368E16970
:10D938002AB9134AC3E900210B60E3610CE093F9AB
:10D948000E0092F90E50A84214D0854212DD51689B
:10D95800C3E900210B605360A569094B9D4200D0C3
:10D9680005B9E568A3689D4202D0284600F0B8FAD8
:10D97800656138BD9142DCD01268D9E74C37002088
:10D9880064370020F8B5DDE906670D4B0C4698684A
:10D9980011460C4A1060EFF31182102282F31288AC
:10D9A800BFF36F8F9D6828462DF0DBF82846324676
:10D9B8003B46FFF7A1FF2046BDE8F840FFF716BF3A
:10D9C8004C37002078370020F8B50446EFF311876C
:10D9D800102383F31288BFF36F8F037C49B203F0DF
:10D9E8001F02002A0CBF0126002639D103F07F034D
:10D9F8002D4D03742DF0A3F82A46037C817363F040
:10DA08007F03037452F8183F934227D1E869C4E9A9
:10DA180000200460EC610FE09842F8D01B68002BEE
:10DA2800F5D093F90EC06145F6D08C45F4DD596800
:10DA3800C4E900310C605C60AC69944200D004B960
:10DA4800EC68AB689C4202D0204600F049FA6C6151
:10DA580087F31188BFF36F8F3046F8BDE869DEE7BA
:10DA68009B071ED585682DF06AF881732B689D4247
:10DA780009D16B68C4E900531C606C60E8E76A6808
:10DA88009342F6D01B68002BF3D093F90E209142F5
:10DA9800F5D08A42F3DD5A68C4E9003214605C604C
:10DAA800D6E78173D4E700BF4C37002049B9EFF3BC
:10DAB800058030B9054B5A699B689A4201D0FFF737
:10DAC80095BE81F31188BFF36F8F70474C370020E4
:10DAD800034648B9EFF3058232B9064A516992689C
:10DAE800914201D0FFF782BE83F31188BFF36F8F95
:10DAF800704700BF4C370020EFF31181102383F3E8
:10DB08001288BFF36F8F054B9A68D37B013BD373A1
:10DB180081F31188BFF36F8F704700BF4C37002027
:10DB280070B5EFF31186102383F31288BFF36F8F5C
:10DB3800144DAB68DA7B0132DA732A4652F8184F73
:10DB4800944200D004B9EC681A7CD20604D1DA8970
:10DB58007F2A01D9A2692AB1A34202D0204600F047
:10DB6800BFF923466B6186F31188BFF36F8FEFF31C
:10DB78001180102383F31288BFF36F8FBDE87040C4
:10DB8800FFF7A6BF4C370020024B03F11802C3E988
:10DB9800062270474C37002008B5FFF715FF70B113
:10DBA800074B9B68DB7B53B9EFF31180102383F39A
:10DBB8001288BFF36F8FBDE80840FFF789BF08BD23
:10DBC8004C37002070B5EFF31186102383F31288C9
:10DBD800BFF36F8F1B4CA168E0690B68814214BFCB
:10DBE8001A46002249680B605960A368E1692AB99E
:10DBF800154AC3E900210B60E3610CE093F90E00BC
:10DC080092F90E50A84218D0854216DD5168C3E932
:10DC180000210B605360A5690B4B9D4200D005B9EC
:10DC2800E568A3689D4202D0284600F059F965616D
:10DC38003046BDE87040FFF7D9BD8A42D8D0126897
:10DC4800D5E700BF4C37002064370020F8B550EA0C
:10DC5800010306460C4603D1FFF7B4FF0020F8BDC8
:10DC6800EFF31187102383F31288BFF36F8F124DE0
:10DC7800124BA8681860FFF715FEA86823463246BD
:10DC88000F49183000F0CAF9AA680446137C3846D0
:10DC980043F004031374FFF7A9FDAB68D3E90A2323
:10DCA800B3F1004F08BF002AD8D12DF0A9F8201AE7
:10DCB80020EAE070D3E700BF4C3700207837002017
:10DCC80023AC030838B50446EFF31185102383F31A
:10DCD8001288BFF36F8F037C5B070FD518302DF0C8
:10DCE80067F8237C204623F004032374FFF798FD8C
:10DCF8002946BDE838400448FFF7D8BE85F31188A7
:10DD0800BFF36F8F38BD00BF3F3F0020014B9868BD
:10DD1800704700BF4C3700202DE9F8430446878937
:10DD2800EFF31185102383F31288BFF36F8F037C01
:10DD3800190705D585F31188BFF36F8FBDE8F88300
:10DD4800D90943F0080260D10274A36813B12046D0
:10DD58002CF0FDFE04F118002DF02AF8A66D04F150
:10DD68005808B04511D04FF0000976B130462CF074
:10DD7800EEFE06F118002DF01BF83046C6F8989014
:10DD8800FFF74EFDA66DB045EFD1DFF8C480D8F897
:10DD980008309C4241D1EFF30589B9F1000918BF59
:10DDA8004FF00109D8F818602A4A964200D00EB9F7
:10DDB800D8F80C60B34202D0304600F091F8204603
:10DDC800C8F8146029F039F9204600F0DBF8B9F1F9
:10DDD800000F02D02048FFF7FBFCD8F808309C421F
:10DDE80031D1EFF3058373BBA289D20718D4284633
:10DDF800FFF7FCFCFB07A1D5002383F31188BFF3D1
:10DE08006F8F0423184602DF98E703F07F0343F07F
:10DE1800080303742CF093FE97E74FF00009C1E75D
:10DE280085F31188BFF36F8F83F31188BFF36F8F6A
:10DE38000423184602DFEFF31180102383F31288BE
:10DE4800BFF36F8FD4E785F31188BFF36F8FD1E7E6
:10DE58004C37002064370020D02E0020D3B5DDE9F0
:10DE68000667089CCDE90067FFF78CFD1CB1034BE2
:10DE78009B685B69236002B0D0BD00BF4C370020AF
:10DE8800027C034612F01F0210D10A4988420DD0C5
:10DE98000949086868B1D9897F2909D893F90E20FA
:10DEA800064B1B689A42B8BF002070470020704795
:10DEB80010467047902D0020380600207C3700203F
:10DEC8000122044BC01A044BC0105843034B1A5488
:10DED800704700BF702F0020ABAAAAAA3F3F0020BE
:10DEE80070B50D4B0D4D1E7CFFF7CAFF06EB4603C0
:10DEF80005EBC305044628462CF05AFF0022084BC0
:10DF08009A553CB1621E2846BDE870400549D317B2
:10DF180000F084B870BD00BF4C370020702F00207F
:10DF28003F3F0020C9DE000838B5EFF31185102304
:10DF380083F31288BFF36F8F0F4B104A9C681068E9
:10DF4800A04206D1FFF7CCFF85F31188BFF36F8F8E
:10DF580038BD00211B7C1160094AD35C002BF3D02B
:10DF68002046FFF78DFF0028EED0237CDB0601D189
:10DF7800FFF7D0FC2046E5E74C3700207837002033
:10DF88003F3F0020EFF31181102383F31288BFF382
:10DF98006F8F0A4A136A834207D1DB6F136281F3DA
:10DFA8001188BFF36F8F70471346002BF7D0DA6FD5
:10DFB8008242F9D1C26FDA67F1E700BF4C3700201F
:10DFC800024B1868984208BF002070473C060020A2
:10DFD800034B1B680BB9FCF757BD0020704700BF07
:10DFE8008037002030B570B10B4B5B6898420AD07F
:10DFF800036843B1D3E90421D0E90445121941EB80
:10E008000501C3E90421D0E9003213605A600023F6
:10E01800C0E9003330BD00BF3C060020B3F1FF3F2C
:10E0280008BFB2F1FF3F2DE9F84F0446994615465F
:10E038001F467AD08160EFF31188102383F312888A
:10E04800BFF36F8FB9F1000FDFF8E4A020DBFFF713
:10E05800BFFFDAE90027013549F100092D1849EB1E
:10E06800E07306464FF00109C4E90453AD1843EBC9
:10E078000707FFF7A5FF0346DFF8B8E0DEF804A0BE
:10E08800EBB9C4E900EACAF80040CEF8044028E039
:10E098006FF00103DAE900125B1A4FF0FF3161EB10
:10E0A80002025B1B62EB0902012B72F10001BCBF8B
:10E0B800012300224FF00009C0E90432D9E7D3E96F
:10E0C800041CD4E904208A4270EB0C0B24DA891A68
:10E0D8005A686CEB0000C3E90410C4E9003214600C
:10E0E8005C60FFF76DFF84420ED1134B1B685BB970
:10E0F800B9F1000F02D1FFF76BFF064630462CF04E
:10E1080040FE0021FCF742FC88F31188BFF36F8FB3
:10E1180028463946BDE8F88F521A60EB0C009A453C
:10E12800C4E90420ADD01B68AAE700252F46EFE715
:10E13800882F00203C060020803700202DE9F0477A
:10E14800EFF31185102383F31288BFF36F8FDFF885
:10E15800A0900026C9F800000027FFF731FFDFF87C
:10E168009480D9F80030D8E900ECD91750B1D0E93B
:10E178000442A34271EB020A1BDAE41A62EB0102C1
:10E18800C0E90442002413EB0E034CEB01012046C6
:10E19800C8E90031C9F800402CF0F3FD2146FCF72E
:10E1A800F5FB85F31188BFF36F8FBDE8F047FFF7E4
:10E1B800BBBE14EB0E024CEBE473C0E90467C8E97C
:10E1C8000023FFF70FFF85F31188BFF36F8F836874
:10E1D8009847EFF31185102383F31288BFF36F8FED
:10E1E800D9F800301B1BC9F80030FFF7E9FEB8E783
:10E1F80080370020882F002010B5EFF311841023FA
:10E2080083F31288BFF36F8FFFF7E2FE0346054AD8
:10E21800D2E90001181841EBE37184F31188BFF3C8
:10E228006F8F10BD882F0020F8B50646EFF31187D1
:10E23800102383F31288BFF36F8F026822B187F32C
:10E248001188BFF36F8FF8BDD0E90A54691C44F1F7
:10E258000003022973F1000334D3013D44F1FF3474
:10E26800002CBCBF15462C462CF0CEFD013041F1E8
:10E278000001401944EB0101012871F100014ADB5A
:10E288002CF0C2FD6FF00203013041F1000140198A
:10E2980044EB010183426FF000438B4140DB2CF0DB
:10E2A800B3FD6FF001024FF0FF33013041F100017F
:10E2B800401944EB0104121A63EB040330461A496F
:10E2C800FFF7ACFE336B01333363336A6BB187F30B
:10E2D8001188BFF36F8F3046336A9847EFF3118781
:10E2E800102383F31288BFF36F8F334653F8184F08
:10E2F8009C42A4D0002CA2D020462CF069FC00231C
:10E30800C4F8983087F31188BFF36F8F2046BDE8B3
:10E31800F8402CF04EBC6FF001024FF0FF33CDE710
:10E3280000224FF00043C9E731E200082DE9F0412F
:10E3380005461C4690461F46EFF31186102383F3CB
:10E348001288BFF36F8FB4F1FF3F08BFB2F1FF3FF0
:10E3580005D186F31188BFF36F8FBDE8F081002CDB
:10E3680009DB012A74F10003BCBF0122002412F169
:10E37800FF3844F1FF3728462CF01AFDDDE9060185
:10E388000023C5E90A012B6342463B462846024959
:10E39800FFF744FEDDE700BF31E2000838B5034669
:10E3A800EFF31185102282F31288BFF36F8FC160DB
:10E3B800012181600068834206D185F31188BFF38B
:10E3C8006F8F0024204638BDD0E9003213605A60B0
:10E3D8000023C0E900332CF087FD29460446024893
:10E3E800FFF764FBEEE700BF403F0020F8B50746A3
:10E3F8000C4616462CF098FB08B10020F8BD0E4BD1
:10E408009B68D3F88C50002DF7D0221DF5D2EFF37E
:10E418001184102383F31288BFF36F8F284647F0C7
:10E428000401B04784F31188BFF36F8F0028E4D04C
:10E4380040F8045BE2E700BF4C3700200146024A7F
:10E448000020FFF7D3BF00BF85620308014828F00A
:10E458007CB800BF4C98050807B5074B4FF480629D
:10E46800009306494FF0FF330548FFF78BF800206B
:10E4780003B05DF804FB00BF28D70408E0BE002005
:10E48800902F0020F0B5042804468BB02BD0344DD3
:10E49800286818B114F09CFF00232B601CB3314B83
:10E4A8009C4220D0002601AB02932F4B214602A8A4
:10E4B8000393019630F054F901983146013014F075
:10E4C80067FF0246286070B106AF384601992EF002
:10E4D80096FC264B214604A80593049730F040F992
:10E4E8002A68019BD65402F07BFD33F042FD2CF0E4
:10E4F8002BFE01F031FF00221D4D1E4BD5F8F040D8
:10E508001A7084B120460EF065FC30B3A06804F0A0
:10E5180035FCD5F8F040002CF4D1D5F8F0301C4685
:10E52800DB68002BFBD1C5F8EC400025124C01F04C
:10E538009BFA08F00FFB0EF03FFD206814F048FF2F
:10E5480025600E4C206814F043FF25602CF06AFD0E
:10E558000BB0BDE8F0402CF0EEBDE468DBE700BF8F
:10E56800DC38002058390020DDAF03087FCD0308D0
:10E57800E0380020403F0020C0370020BC37002092
:10E58800002270B50446154B00EB8105C3E9002253
:10E598009A60264630682EF0B2FB022804F1040483
:10E5A80018D130680E4C206098B10E482DF057F8FD
:10E5B80020682CF05FFD0C4802F0BAF902F008F967
:10E5C800064920682CF051FD0023236002F000F971
:10E5D800012070BDA542DCD10020E3E78837002088
:10E5E800B8370020DC990508C5EF050810B50446C2
:10E5F80008482CF03FFD02F089F840B1064802F0C7
:10E6080097F934B1BDE81040044802F091B90448C4
:10E61800F5E710BDDC990508B0ED050875E80508B3
:10E62800DDED050873B506462CF085FD08F04EF8BB
:10E6380014F0BAFD054614F0C3FD0446641B00251A
:10E6480008F04CF8A4F5806008F04EF801F084FE5C
:10E6580000F05CFC6B464FF4006230461F490095A1
:10E668002CF0BCFC01461E4B1E4C1860009B194444
:10E6780009F0D6FD4FF4005201AB30461A49019516
:10E688002CF0ACFC0146194B1860019B19440EF0A4
:10E6980073FB05F0A1FD2946D4F8E80012F0BAFB97
:10E6A8001621D4F8E80032F0A2F96621D4F8E8007F
:10E6B80032F09DF940F6B651D4F8E80032F097F9F7
:10E6C800294604F1D80012F0A5FB094804F0CCF85B
:10E6D8000122084B1A7002B070BD00BF839805086C
:10E6E800BC370020E03800209A980508C037002081
:10E6F800A97D0508403F00202DE9F0470928044678
:10E70800A4B000F08F8001F041FE00287FD0002CDB
:10E718007DD1464BD3F8F030002B78D0204602AD9F
:10E72800DFF80C81FFF77EFF2CF0BFFF02F0BAF88C
:10E738004FF4007128462EF047FBC8F8005001F04E
:10E748002DFE0121064600F180072CF0C9FD394B4A
:10E75800394A3A493A482EF0D7FC06A800F040FB5F
:10E76800384937482EF0F5FCDFF8DCA0DFF8D09008
:10E7780006AD5146484615F8012B01342EF0E9FC48
:10E78800202CF6D131492E482EF0BEFC33F0F2FB96
:10E7980002212F48FFF7F4FE0023C8F8003002F0EA
:10E7A80087F8012338462B4A0EA934F07BFBA0B921
:10E7B800029830F02AFD039A0446014601AB013263
:10E7C8000EA834F094FC40B9039A019B9A4204D1F4
:10E7D800214604983DF085FFA0B14FF47A702CF0E3
:10E7E800D3FD0A231B4A0EA9384634F05BFBDDE94A
:10E7F800032101AB0EA834F02CFD0EA834F092FED4
:10E8080001F0AAFD002130462CF06AFD04E0204604
:10E81800FFF708FF2CF049FF0F4C6068FFF732FE46
:10E828000023636024B0BDE8F08700BFE038002013
:10E8380084370020B4980508C79805081D9905086D
:10E8480018E3040864E70508B2EF05086ED905085F
:10E8580064D704082D990508883700202DE9F04F62
:10E8680089B007462CF0D4FE804640B1B1482CF060
:10E87800F6FE3846FFF7BAFE384601F0CDF9DFF864
:10E88800B892CDF80880002F40D0D9F80030B3F501
:10E89800007F40F0D780002520262C464FF0020943
:10E8A8004FF4401B2CF06CFD4FF4C87303FB09F3C5
:10E8B800049303F59C53083303900093002C40F015
:10E8C8007681A2464FF0010901F09CF801F042FF61
:10E8D80005460190002800F0BD8046F0100601F0C2
:10E8E800EDFE964C206828B103781E4002D114F042
:10E8F8006FFD2660BAF1000F04D0002001F0AEFDD4
:10E9080001F0A6FD284609B0BDE8F08F01F024FD0E
:10E9180001F03EFF0546002840F08680874EFFF74D
:10E9280081FE2CF0C4FE3368002B5CD01A7822F0EC
:10E9380020021A7033689A681C78127892B1586865
:10E9480008B103F091FF336801219B6807A807937A
:10E95800FFF716FE98B9336898682CF080FE78485F
:10E9680001F0E6FF04217748FFF70AFE38B90821CD
:10E978007548FFF705FE10B1744801F0D9FFD9F8C2
:10E9880000301B0531D501F00DF801282DD1704854
:10E998004FF0000A01F0CCFF6E4BD9F8040083F861
:10E9A80000A0FFF76FFD3268C9F804A02AB11378F8
:10E9B800980644BF43F020031370D9F800301905B6
:10E9C80015D500F0EFFF441E18BF01243026D9F8F2
:10E9D8000030DA051BD5B3F5007F4FF001043FF492
:10E9E8005DAFA1462BE03C46BCE75B48D0E71BB9CE
:10E9F800242604F00104EAE714F0020418BF83F4A3
:10EA080080634FF0280618BFC3F38024DFE7B3F50F
:10EA1800007F254615BF4FF001094FF002094FF45A
:10EA2800405B4FF4401B3DE7D9F80030B3F5007F59
:10EA38003FF431AF3D463C4620264FF001094FF4E4
:10EA4800405B2FE7002520262C464FF00309DFF80E
:10EA58000CB127E72CF0DCFD059080B12CF0F7FD18
:10EA680068B101F095FE054648B92CF0DEFD042892
:10EA78007FF437AF032000F09BFF059D31E7CCB949
:10EA88002CF0C6FD0546A8B101F082FE90B9B8F198
:10EA9800000F02D13846FFF7A9FD029B13B938468B
:10EAA80001F0BAF82C4623482CF0D9FD2C4801F087
:10EAB8003FFF02952CF0ACFD0546002814BF4546E3
:10EAC8002C46B9F1000F05D001F062FE10B902F032
:10EAD800D7FF81462CF054FC039B049AC31A9A4230
:10EAE80080463FD94FF4C871B3FBF1F201FB1238ED
:10EAF800B8F1630F11D9BAF1000F04D0002001F06A
:10EB0800ADFC01F0A5FCC8F5C870B9F1000F47D1FC
:10EB180014F07AFB14F0C2FB2CE0BAF1000F04D118
:10EB280001F0B6FC584601F099FC0123C8F16400D5
:10EB38000193EAE7579A050888370020D83800205B
:10EB4800CCEF050854D7040834D7040893E6050821
:10EB580007E60508403F002020E6050800303000A1
:10EB6800F4E80508009A9A4208D22CF009FCCDF87E
:10EB780004A00390A846DDF804A0A5E6BAF1000FAA
:10EB880004D0002001F06AFC01F062FC009B039AAB
:10EB98001344A3EB0800B9F1000F05D00028E9D011
:10EBA800484528BF4846B3E70028E3D0B0E74FF010
:10EBB800000A96E607B5114A114B1068596820B14A
:10EBC80003B05DF804EB2CF04ABD1A6892050ED527
:10EBD8009A68002A0BDD51B109680C33C9880948C5
:10EBE800009109492EF090FA03B05DF804FB07483C
:10EBF80003B05DF804EB01F09BBE00BFB8370020FE
:10EC08008837002018E304083B99050839EC050803
:10EC18002DE9F74314F0ACFA00F06CFF2CF002FA7F
:10EC280014F05EFB2CF0FBFB01F0AEFC53482CF01B
:10EC380021FA00F059FF18B900F062FF00F05AFFFE
:10EC48002CF030FD01F03EFE00F04EFFB0FA80F0EF
:10EC58000021400901F0B4FA10B9082000F04AFF79
:10EC680033F087F92CF070FA2CF06DFA02F0F2FA12
:10EC780042482CF0FFF9002000F09AFE00F034FF23
:10EC880008B901F021FD0125012001F079FB0120DF
:10EC980001F070FB00F028FFFFF72EFD2CF04CFA76
:10ECA800012001F089FD4FF480742846344E354F19
:10ECB800DFF8D48014F4106957D015B9384601F03C
:10ECC80037FE3578002D3ED100F00EFFFFF7C6FD68
:10ECD8000028EFD100F008FF044601F03DFB204674
:10ECE800FFF7A0FC2CF0E3FC012001F0FFFC00F092
:10ECF800FBFE28B9254B012101A80193FFF740FC31
:10ED080001F0C6FB404601F0A9FB01F0A1FB3378F6
:10ED1800012B1AD101F0C6FD00F0C0FC044601F039
:10ED2800C7FD0420FFF7AEFB01F0B2FB002001F0A5
:10ED380095FB01F08DFB012001F0E0FC032000F0C1
:10ED480037FE0020B6E70025C4E7114BDFF84490F2
:10ED5800C9F8003001F03CFD00F030FD0023044606
:10ED6800C9F8003001F034FDDBE7002CB0D02EF0FC
:10ED780022FB484603B0BDE8F08300BFDC990508D4
:10ED8800413F002035DE0508303030004499050841
:10ED98004C990508B837002008B50EF02BF800F09C
:10EDA80037FB0421064830F09EF82CF051FB00F0A8
:10EDB8008FFE02F091F9BDE808400EF02FB800BFB1
:10EDC800D0390020014B1878704700BF403F002021
:10EDD800004870470068890900487047333353403A
:10EDE80038B505462021FAF777FB041E11DA2146CB
:10EDF800094827F0AAFB002421462022074827F0CB
:10EE0800A4FBC4F1200228190021BDE838403DF0D8
:10EE180060BC1F2CF0DD38BDE5990508FF99050891
:10EE28000428034607B506D801460F4803B05DF825
:10EE380004EB01F0EFBB062168460C4A24F0FAFD0A
:10EE4800011E0DDD052901DD28F030F9442201F10C
:10EE580008036B446846013103F8082C01F0DAFB1B
:10EE680003B05DF804FB00BF269A05082B9A050835
:10EE7800F8B5244DAB7DDB0732D52E6870680128C4
:10EE88002ED9B168431ECA5C0A2A29D14A1E002B12
:10EE980001DC1A4608E0D45C0A2CFAD0013BF6E7FC
:10EEA8008C5C202C02D101329042F9D8002B0CDD69
:10EEB800541CA04209D15C1E0C44A14205D014F890
:10EEC800017D0A2F0CD0202FF7D00144D21A11F857
:10EED800023C94083A2B0C4F08BF0134013C00D285
:10EEE800F8BD0422394630462DF045FF0421384646
:10EEF80001F090FB2B6904332B61AB7D43F00203D7
:10EF0800AB75EBE7C43700200EF30508202200217B
:10EF180001483DF0DEBB00BF98390020002238B51B
:10EF28000B4C0546A26062754FF0FF326B680846CD
:10EF3800C4E9032363602560A1612CF09BF86B682A
:10EF48000BB90123A375BDE83840FFF791BF00BF97
:10EF5800C4370020F8B503780446DBB10E4FD7F864
:10EF6800B80018B12146F2F70BFA98B12046F2F72B
:10EF780019FA461C304630F04BF9054650B1324676
:10EF880021463DF07FFB05491C22081D3DF087FB0B
:10EF9800C7F8B850F8BD00BFE03800209839002005
:10EFA8002DE9F347AC4C06462368D3E9011031F04C
:10EFB800FEFAA5680746002D40F03A81731E042B1F
:10EFC8001AD8D4E900325B689A4279D0012E15D15B
:10EFD800236865689868D4F8108000EB0801284415
:10EFE800A8EB050800252CF028F8A8450646A560DA
:10EFF80040F3BC80A946AAE00D2E13DC022E40F394
:10F00800B580F31E0A2B00F29180DFE813F0590057
:10F018008F00CF018F008F0060008F008F008F005E
:10F028003E004E001B2E4FD07F2E50D0A37D990757
:10F0380000F181801F2E40F3998020682169836840
:10F048005A5C06F0C003802B0CBF237DF2B202F19C
:10F05800400508BF0133EDB214BF0023DBB2372DE2
:10F0680097BFE5250025D20802F0060298BF154192
:10F0780019443246237598BF05F003052DF065FF46
:10F08800237DAB4272D1013597E074482BF0F2FF33
:10F09800A0692BF0EFFF2268636821699068C91A9C
:10F0A800184401F0B7FA002587E06D482BF0E2FF1D
:10F0B80020682DF0D9FE636800261844FFF74AFF40
:10F0C800304602B0BDE8F0870123A3604EE0226914
:10F0D80061688A424AD900232068561AD0F808E0A5
:10F0E800B34203EB010C18D1032BCCBF0426012635
:10F0F800961B33461EF803C019460CF0C00CBCF131
:10F10800800F03F1FF33F5D0A2EB01084246761ACF
:10F118002DF028FF4FF0010919E01EF80CC0BCF1D2
:10F12800200F01D10133DBE70126E1E7A37D9A0730
:10F1380023D5092E18D0202E7FF47CAF002603217A
:10F148002068A675B1462DF006FF4FF00308A8EB1E
:10F158000600FFF765FE2369A3EB08032361B9F1F5
:10F16800000F00F0298128E00023A375A37D4FF04C
:10F17800FF3623F00203A375A2E7092E7FF45AAFE6
:10F1880022682169D2E90123002A40D00B4413F8F0
:10F19800010C10F061FA002839D00425314B019395
:10F1A8000026019B21695A1C019231441A78206873
:10F1B80001362DF0C4FEB542F3D12368D3E901101E
:10F1C80031F0F5F9B84203D20321274801F022FAB9
:10F1D80023682769D3F80880D3F80490781908EBD6
:10F1E800090140442BF029FF0646A9EB070108EB6B
:10F1F800070001F00FFA236822695B689B1A5B1B02
:10F20800981BFFF70DFE23692B442361AEE72368A3
:10F2180060689D682169154A091A01AB28440BF0FA
:10F22800CFFA05460028A1D0431C3FF431AFB7E719
:10F23800013D032D00F2E880DFE815F004001A0014
:10F24800A000E1004F2E04D05B2E40F0DD800223A9
:10F258003BE7042339E700BFC4370020309A05088C
:10F26800579A05080EF30508399A050818E30408A3
:10F27800A6F13003092B03D803236675A36075E74D
:10F288000023412EA3602ED1E368062B3FF76EAF13
:10F298005E4D03F1010A2D3305EB8305AB68002BA6
:10F2A8003FF464AFD4F80080D4F80490D8F808008C
:10F2B8002169014448442BF0C0FE06464046C8F880
:10F2C8000490A968C4F80CA02DF02CFE636822698C
:10F2D800A2EB03082268B8F1000F5568A5EB0305F7
:10F2E8007FF76BAF16E7423E062E3FF63FAF01A30E
:10F2F80053F826F019F300085FF300086FF30008CD
:10F3080075F10008B5F3000875F10008D9EF000899
:10F31800E568002DFFF62AAFD4F80080D4F80490F1
:10F32800D8F808002169013D014448442BF085FEC6
:10F33800D8F804100646A1EB09014046E5602DF017
:10F348000AFEE268002AC1DB304B206803EB820327
:10F35800D3F8B810B8E7236822695B689A42BFF40B
:10F3680005AF01252BE0226963689A427FF6FEAE5D
:10F3780000254FF00108A9462E46E8E67E2E43D127
:10F38800637D312B3FF424AE333B052B3CD801A2DF
:10F3980052F823F0D7F30008B5F3000811F4000879
:10F3A80011F40008D9EF0008B5F3000823685D6878
:10F3B8002369ED1A0023A360002D7FF7D7AE2368D9
:10F3C800294698682369184401F024F91BE7206846
:10F3D80021694368994217D2012285685B1A0D4456
:10F3E80015F8016F06F0C006802E01D19A4204D1AB
:10F3F8002DF0B8FD0023A36055E60132F0E7462E54
:10F40800D4D0482E3FF4E4AD00235EE6E038002077
:10F418002DE9F04F8BB068460A4BCDE900451968D5
:10F42800CDE90267091A8908CDE90489CDE906AB57
:10F43800CDF820C0CDF824D02FF055FD0BB0BDE895
:10F44800F08F00BFE038002070B5067804461EB182
:10F458004FF0FF35284670BD2CF00BF9C31E012B69
:10F4680005460CD801210C48217001F0D3F8032D72
:10F47800EED10A48836E60309E600EF023FBA388AD
:10F48800013B9BB2A380002BE4D10121044801F089
:10F49800C1F86388A380DDE73D9A0508E0380020BD
:10F4A8005B9A05082DE9F0431D46002391B00446F8
:10F4B80003A81746049388460EF0F0FA07F00106F1
:10F4C800034600285BD1F90641D5D4E90121DC20A7
:10F4D8002EF025FA0446B8F1010FD4F8009007D1B0
:10F4E8004FEA091140F2D22041F0060104F0DCFE97
:10F4F8002146424601A811F08BF94946C7F380021C
:10F5080001A80FF0D9FEB8F1010F044601D1FFF7A9
:10F5180043FC380602D4032000F0FCF914B120465D
:10F528002DF081FF4FF0FF3000F0F4F9012012F0C8
:10F538001FFF07F0A1F8EEB9CDB900241EB10121D3
:10F54800474801F067F8204611B0BDE8F0837A0615
:10F5580005D594E80E00DC202EF099F9BAE7BB0631
:10F56800B9D520462EF0B9F82EF0E7F9B2E7002316
:10F578002B60E2E701213A4801F04CF8DCE74FF054
:10F58800FF3000F0C7F9022012F0F2FE790602D52A
:10F59800A368206898471EB10121314801F03AF864
:10F5A800049C20460BF0DEFE2E490DF0BDF9002824
:10F5B80041D004982EF0D4FC0E283AD0C20705D4C6
:10F5C80083072BD10268284B9A4227D12EF084FF5B
:10F5D80040F48074002DB1D04FF0FF33049F2C60AD
:10F5E80038466F60AB602EF0A6FC0028A6D06946AE
:10F5F800384601AA2EF0CEFC019B002B9ED05A68FB
:10F60800AA60002285F82C2018682EF086F820229F
:10F61800014605F10C003DF093F88FE70146002202
:10F6280012480BF0BBFE124910482DF0E9FC0120EE
:10F63800CEE70020CCE70F4B9C420DD004990B4835
:10F648002FF08EF8049B0C4918680DF06DF908B17D
:10F658008224BFE70124BDE74FF40064BAE700BF86
:10F668003D9A0508500805084018050818E30408DD
:10F678006ED90508583900202C08050808B5037804
:10F688004BB901210170044800F0C4FF2BF0F1FFD1
:10F6980003380128FAD808BD3D9A05082DE9F0433A
:10F6A8008BB0202106A82DF08FFB0026DFF8E8801C
:10F6B8003A4F40462BF0DEFC384607962BF0DAFC32
:10F6C8002BF0D7FF0128044635D107990229F0D13C
:10F6D800089B1A78052AECD193F80190B9F1410FEB
:10F6E80006D02F4800F096FF00232C480793E5E743
:10F6F80080252C4800F08EFF03216846ADF80050A5
:10F708008DF8024000F086FF002301AA0392264AE2
:10F7180021460492254A03A805924A468DF80430EA
:10F72800ADF80650ADF80850FFF7BCFEC305DBD5B1
:10F738000BB0BDE8F083022809D11D482BF09AFCD4
:10F7480006A82DF063FB00201A4B1870F0E7032879
:10F7580002D100230793B3E7042804D0C1B206A856
:10F768002DF091FBACE714482BF084FC079B43B9C0
:10F778000F482BF07FFC06A82DF048FB4FF4807053
:10F78800D6E700231122012106A8FFF78BFE10F40B
:10F79800106F91D0CCE700BF3F9A05087BD90508C8
:10F7A80094CF04085A9A050851F4000885F6000811
:10F7B800579A0508413F00205D9A05082DE9F04158
:10F7C80092B0202101A82DF0FFFA494EDFF82481DC
:10F7D80030462BF04FFC48482BF04CFC30462BF0C1
:10F7E80049FC464FBA8A002302B1BB8205A802939E
:10F7F80006930EF053F9044690B9414901A82BF03D
:10F808002AFC012805462CD139482BF033FC01A8E5
:10F818002DF0FCFA20463B4B1D7012B0BDE8F0817C
:10F82800022012F0A5FD30462BF024FC069936483C
:10F838002EF096FF029B002BD4D001A82DF014FBCC
:10F848000AF0FAFE58B10A2101A82DF01CFB414626
:10F8580001A82BF000FC03280BD00428EDD10021CF
:10F868002CE0022803D122482BF004FCB0E703283F
:10F8780001D1304619E0042808D11D482BF0FAFBC5
:10F8880001A82DF0C3FA4FF48070C6E70528D1D13E
:10F898001E482BF0EFFB02941D4C2BF0EAFEC1B280
:10F8A80003298DF8031003D111482BF0E3FB99E7E6
:10F8B80004290CD10E482BF0DDFB01210023162270
:10F8C80001A8FFF7EFFD10F4106F8BD0A5E701A892
:10F8D8002DF0D9FA9DF803300D2B03D120462BF0DB
:10F8E800C9FBDAE701210DF1030000F093FED4E72C
:10F8F800579A05089C9A0508C7980508E03800201B
:10F90800609A0508413F002018E30408659A050835
:10F91800959A0508014B1860704700BF44060020FF
:10F92800024B986A003818BF01207047E038002061
:10F938002DE9F04106460D4600270DB9BDE8F081D6
:10F9480033780A2B16D1AFB90121104800F062FEB6
:10F95800012406EB040843461FB998F800200A2A38
:10F9680001D0A54208D13046214600F053FE464654
:10F978002D1BE2E70024ECE71F7808F10108A7F146
:10F988000D035F425F410134E5E700BFA19A050816
:10F99800024B0348197831F072B900BF423F00208A
:10F9A80064E00408014B1878704700BF423F00200C
:10F9B800014B1870704700BF423F002010B5044645
:10F9C80002F0A6FDE3681BB90C4A1168A14203D1F5
:10F9D800BDE8104002F0B6BDA360094B1968E160AC
:10F9E800196809B119688C60116801B914601C6044
:10F9F80002F0A8FD13F0D2FB10BD00BFE8370020CD
:10FA0800E43700202DE9F041144E34F099FF3368B3
:10FA18000BB3134D02F07CFD2C681CB1BDE8F0411E
:10FA280002F090BD01230F4A2B60336834601460E4
:10FA38001BB92B68013B2B60F0E79F68C3E90244C0
:10FA4800D3E9006802F07EFD0EB14046B04702F0EF
:10FA58005FFD3B46ECE7BDE8F08100BFE8370020DA
:10FA6800E0370020E43700202DE9F7430025A846B9
:10FA7800144E019502F04CFD346801AF54B9019B56
:10FA88003360114B1D60114B1C6003B0BDE8F0439F
:10FA980002F058BDD4F808902046C4F808800DF04C
:10FAA80099F918B10023E3604C46E7E760680DF068
:10FAB80091F90028F6D12B463C60254604F1080749
:10FAC800F1E700BFE8370020E4370020E0370020E6
:10FAD80010B5044B1C6804B910BD60682FF037FAE4
:10FAE800A468F8E7E8370020014B1878704700BF92
:10FAF800433F0020014B1870704700BF433F002070
:10FB08002DE9F04132F038FA294B044620F47F0001
:10FB180020F47F409842274E0AD114F47F4FC4F353
:10FB2800072505D032F027FA35702846BDE8F08160
:10FB3800002333702BF07FFA28B1062833D85423DA
:10FB4800C340DB072FD51C4832F015FA00F0A0FCA3
:10FB58002BF007FC064600200F460146DFF85C80C4
:10FB6800FA220023F1F7B2FB7D2A73F1000334BFB8
:10FB78004046002000F072FC2BF068FC054648B9AE
:10FB88002BF0EFFB801B61EB0701B0F57A7F71F179
:10FB98000003E5D3002000F061FC00F059FC25B912
:10FBA800204632F0E8F90025BFE71125BDE700BF80
:10FBB800AF0000AD433F0020AF1100AD0030300072
:10FBC800024B43EA002032F0D6B900BFAF0000ADC7
:10FBD8000D4D08B52B780446012B0FD901280DD9F6
:10FBE8000A4826F0B2FC2146094826F0AEFC2978DE
:10FBF800084826F0AAFC27F02AFAFCE72046FFF777
:10FC0800DFFF32F0B2F900BF433F0020A39A050896
:10FC1800B99A0508C59A050810B50446002838D0D1
:10FC28001C4800F085FE631E112B12D8DFE803F094
:10FC38002D1111111111112B112911112721252312
:10FC4800091F154800F074FEBDE81040134800F085
:10FC58006FBE023C1248E4B200F06AFE0A2C16D8C5
:10FC6800104B53F8240000F063FE0F48EAE70F48F2
:10FC7800E8E70F48E6E70F48E4E70F48E2E70F48F0
:10FC8800E0E70F48DEE70F48DCE70F48DAE70F4800
:10FC9800E9E710BDB2E505083AE60508C6E5050836
:10FCA800B4EC0508D4D80408D7E5050806EB050820
:10FCB8007BED050834E705084AE7050836E8050836
:10FCC8001AE805081CED050814E90508F0E605081A
:10FCD800012910B502460C4617D9042915D00B493D
:10FCE8000B482DF036FA022C03D0052C0BD009490D
:10FCF80000E0094906482DF02CFABDE810400749F4
:10FD080003482DF001BA0649F4E710BDE9ED0508EE
:10FD180018E3040817EB0508C7EA05086ED90508B3
:10FD2800D2EA05082DE9F04F9DB000AF80460C4699
:10FD3800924600F033FB28B9012528467437BD46A2
:10FD4800BDE8F08F01239F4A07F11801803033F096
:10FD5800A9F80028F0D1D7E91402D7E90A139A4282
:10FD680008BF884200F02B8197F84930002B40F0FB
:10FD7800268107F118002BF0F7F95B28064606D113
:10FD8800D7E90A2307F1180033F0A1FCE3E7002EB6
:10FD9800F6D008F1FF3919F8015F2DBB30460FF096
:10FDA8005BFC20B107F118002BF0DEF906463D2E6A
:10FDB8001CD107F118002BF0D7F922280CBF01231A
:10FDC80000238AF8003040F0CA8007F118002BF0B1
:10FDD800BCF922282AD016D830B30A2824D0C1B2B8
:10FDE80020462BF0D9F9F0E7B54206D00A2EB2D05A
:10FDF80007F118002BF0C7F9ADE707F118002BF051
:10FE0800A4F90646C7E75C28E9D107F118002BF0EA
:10FE18009CF97628E3D861281DD80A2804D05528EB
:10FE280000F089800028DAD1052509E007F11800DB
:10FE38002BF09AF90A2803D0232807D00028F3D1F9
:10FE4800EDB207F1180033F06DFB76E707F1180003
:10FE58002BF099F9F4E7A0F16203142BBFD801A2A3
:10FE680052F823F063FF0008E7FD0008E7FD0008EB
:10FE7800E7FD0008D1FE0008E7FD0008E7FD0008DF
:10FE8800E7FD0008E7FD0008E7FD0008E7FD0008BA
:10FE9800E7FD0008C5FE0008E7FD0008E7FD0008CB
:10FEA800E7FD0008C1FE0008E7FD0008C9FE0008DC
:10FEB800D5FE0008CDFE00080D2090E70A208EE749
:10FEC80009208CE70B208AE70C2088E73B1D6E464B
:10FED8009B464FF00409D84609EB0B0A07F11800B6
:10FEE8002BF033F908F8010BD045F7D10023394638
:10FEF8000BF809301022584623F03CFE3B680146B7
:10FF0800434528D1B0F5881F22D27F281AD9B0F5E9
:10FF1800006F19D3B0F5803F34BF03230423227B3D
:10FF280022B16268134422689A420FD920462CF005
:10FF3800B1FFB54649E707F10C036E469B464FF003
:10FF48000809C8E70123EAE70223E8E76360F0E766
:10FF58000225B54674E7B54666E708203FE70A2854
:10FF68003FF462AF00283FF45FAF00250D281CD096
:10FF780009DC092819D00A2800D040B963685B1B3E
:10FF8800636000255CE720280FD0232805D0C1B284
:10FF980020462BF001F900250CE0636807F11800F2
:10FFA8005B1B63602BF0EFF8EBE7C1B220462BF048
:10FFB800F3F8013507F118002BF0C7F8D6E7042548
:10FFC8003FE700BFDC9A050870B586B00E461022E0
:10FFD8000DF1070302A92BF0EAF8044648B99DF889
:10FFE80007507DB9084902A8F1F7CAF920B90125D7
:08FFF8003570204606B070BD13
:020000040801F1
:10000000044902A8F1F7C0F90028F5D00524F4E767
:10001000EB9A0508F09A05082DE9F0418EB002AC84
:100020000E46302221460DF103032BF0C4F805469D
:1000300028B99DF80380B8F1000F04D005252846A3
:100040000EB0BDE8F0812046F1F7B0F92718A742BD
:100050000CD99DF808302B2B01D02D2B06D12D3B30
:10006000D3F1000848EB03080DF10904391B0229FC
:1000700021DD2378692B13D163786E2B1BD1A378F4
:10008000662B18D14FF0FF43E01C0193B842D5D145
:10009000019BB8F1000F01D003F100433360CEE7BC
:1000A0006E2B08D16378612B05D1A3786E2B02D11A
:1000B000054BE01CE9E7204601AA06F0D9FB002821
:1000C000BCD08442E2D1B9E70000C07F70B50446DD
:1000D00088B004A80E4620212CF07AFE20460DF1AF
:1000E000060204A9FFF722FE054630B99DF8063046
:1000F00033B104A808F020FD3060284608B070BD78
:1001000020460DF10701FFF763FF30B99DF8073076
:10011000002B0CBF1E203E20EEE7204602A92BF04C
:100120006FF818B902982EF09EF9E5E7204603A96A
:10013000FFF772FF70B9039C21462046F1F71EF8C5
:1001400030B924F0030444F00204A4F1FF40D3E7E3
:100150000148D1E70525D0E70200400000B597B07F
:1001600002460A236946044832F0A0FE684633F08E
:10017000DDF917B05DF804FBC012002010B5064C85
:1001800023783BB14FF47A72044B1A6000F0CAF93D
:100190000023237010BD00BF443F0020480600200C
:1001A000074B1A685AB11A68012A09BF05491A682B
:1001B0000A704FF47A7218BF02F1FF321A6070476A
:1001C00048060020443F00202DE9F0414FF0000890
:1001D000514EADF5287D0746504C30460D46A6F8E9
:1001E000048000F0ADF906F18000C4F8048032F01C
:1001F00059FE0D2806D147B93DB900200DF5287DDF
:10020000BDE8F081002D00F084804FF400730022DF
:1002100000930721424828AB14F00CFA0028ECD1D7
:1002200000F080F93F493E4814F01EF90028E4D15F
:100230003D493B4833F029FD0028DED13B48FFF71C
:100240008DFF3B48FFF78AFF3A48FFF787FF3A48A0
:10025000FFF784FF3949324833F017FD384B03AAC2
:1002600003F13807154618685968083303C5BB42BF
:100270002A46F7D11B88334A2B80392312A90293CF
:1002800027480A2332F012FE029A02AB03A912A8F1
:1002900032F0E3FF12A833F049F92B48FFF75EFF75
:1002A0002A4B03AA03F1100715461868596808334A
:1002B00003C5BB422A46F7D1186899889B79286004
:1002C000AB711623A980224A029312A90A2314486B
:1002D00032F0ECFD02AB03A91A6812A832F0BDFFA0
:1002E00012A833F023F91B490D4833F0CEFC002847
:1002F00083D100F017F9184B012523600023E36038
:10030000164BC4E90156C3E93B442CF062F8284679
:1003100074E70028EFD070E740120020EC3700208F
:10032000C012002077A70508F69A0508029B050869
:10033000159B05082C9B0508369B0508439B050863
:10034000699B0508479B0508DC9A0508A39B0508DF
:100350005B9B0508649B0508A97D0508E038002023
:100360004FF47A7208B5044B1A6000F0DBF8BDE870
:10037000084012F0B3BD00BF480600200146014806
:100380002AF08CBF40120020014601482AF0A2BF8B
:1003900040120020024B5868003818BF01207047F7
:1003A000EC370020034B04485B68002B08BF00209B
:1003B000704700BFEC3700204012002008B534F031
:1003C000C0FA2BF075F900F089FDFFF7D7FE34F085
:1003D000BAFA2BF06DF9002031F0D4FD034BC3E9DC
:1003E0000001BDE8084034F0ADBA00BF5030002035
:1003F00008B5FFF7D5FEBDE80840002201490248D4
:100400002AF099BEBD0301080038002010B5074C42
:1004100002F082F823680BB912F0E6FE236801337C
:100420002360BDE8104002F091B800BFFC37002007
:1004300008B502F071F8074B1A6812B11A68013A50
:100440001A601B680BB912F0DDFEBDE8084002F02F
:100450007DB800BFFC37002001482BF05FB900BF1A
:100460001438002038B5094D04462B6883420CD05F
:10047000074B19782AF0C0FF2C60011E18BF01211C
:10048000BDE83840034800F0EFBC38BD103800200C
:10049000DF0A00201438002070B50B4C257895B980
:1004A00001260A490A48267000F0C2FC2A46314655
:1004B00007482BF05BF94FF08072064B18681A6002
:1004C000FFF7D0FF257070BD453F002008360508B6
:1004D0001438002010380020014B1870704700BFFE
:1004E000DF0A0020014B1878704700BFDF0A0020A8
:1004F000F8B50E461C4615466AB1094F3B781BB944
:10050000FFF784FF01233B7022463046691EBDE899
:10051000F84012F06DBD012B94BF00200120F8BD02
:10052000463F002010B5054C12F0C0FC23780BB1FB
:10053000FFF77EFF0023237010BD00BF463F002061
:1005400010B50F4B04460360838843F00503838096
:1005500031F003FD01230E220A4984F88430231D63
:10056000C4E90823C4E90D2323616161064B0749EF
:10057000A060C4F88040E260A162E36310BD00BFE8
:10058000E01C05085BB40308B9B50308F1040108D1
:1005900010B5054C23782BB92BF02EF831F015FD52
:1005A0000123237010BD00BF473F002073B50546EF
:1005B0000C46C1B10E4B1B78C3B90A4601AB0146CC
:1005C0000C482CF05FF906460B4B1B7853B902F030
:1005D00013FB40B1214628462BF016F82146284649
:1005E00012F0ACFF3446204602B070BD0E46EBE779
:1005F000483F002050070020493F0020024B1A7856
:1006000018701046704700BF493F0020024B1A780F
:1006100018701046704700BF483F00202DE9F8438E
:10062000DFF87C8000AF05460E462AF0FEFED8F8C3
:10063000003043B31B482BF03FF8C0F5007204466E
:10064000D8F8000043689919914223D90734D21A87
:10065000294624F007042CF092FBE946ADEB040D8B
:1006600069461048D8F8004000F070F9014620466D
:100670002CF05CFC0A21D8F800002CF008FC0023C8
:10068000C8F80030CD4631462846FFF78FFFBD46FB
:10069000BDE8F883324629462CF071FBF3E700BF32
:1006A000843700202DE6050808B5FFF785F9044BCF
:1006B00003F178029A62BDE8084012F073BD00BFF2
:1006C000E03800200022014B1A60704720380020DB
:1006D0000122034B1A700022024B1A60704700BFC0
:1006E0004A3F0020203800200022014B1A7070473A
:1006F0004A3F0020024A136803431360704700BF5B
:1007000024380020024A136823EA0003136070476C
:1007100024380020014B1878704700BF4A3F002062
:1007200038B50B4B1B7893B10A4B1B687BB90A4C4D
:1007300025682AF029FE2060236813B92368013355
:10074000236025B9BDE838400120FFF7ADBF38BDB3
:100750004A3F0020243800202038002010B50C4CDF
:10076000206890B10B4B1B6883B92AF00DFE2368FB
:1007700083422368A0EB030040F2EE2388BF00F120
:10078000FF30984294BF0020012010BD0020FCE7FC
:100790002038002024380020024B1868003818BF89
:1007A0000120704720380020034B1B7813B9034801
:1007B0002AF059BF704700BF4B3F0020BA9B050885
:1007C00010B10122024B1A700248FFF7FBB800BFBC
:1007D0004C3F002028380020F8B5254B1D7825B166
:1007E000BDE8F8400120FFF7EBBF224B22481D7007
:1007F0002BF035FF20482BF018FF58B91E482BF07E
:1008000026FF80F001040120FFF7F8FE01270546CE
:10081000E4B20AE02AF000FF0028EFD016482BF0DF
:1008200016FF2F4680F00104E4B2F4B10120FFF777
:10083000EDFE064611482AF016FF11482AF013FF74
:10084000FEF7BCF90F482AF00EFF0F482AF00BFF05
:100850000E482AF008FF17B12846FFF7CFFE34B143
:100860003046BDE8F840FFF7D1BE2646E2E7F8BDC6
:100870004B3F00204C3F002008070020C19B05088B
:10088000C69B0508CB9B0508CF9B0508BE9B0508AA
:10089000044B1B7823B9044B1B780BB1FFF79CBFAB
:1008A000704700BF4B3F00204C3F00200122014B0E
:1008B0001A7070474B3F00200022024B02481A700A
:1008C000FFF780B84B3F002028380020034B044A34
:1008D00004481A6000225A602BF0BBBE2838002062
:1008E0009108010808070020A1F180034F2B70B583
:1008F000064618D8194602230D480E4C10F8012B55
:10090000914205DA03FB0144E518A54205D870BD04
:1009100003FB0244891A0133F0E7304614F8011B47
:10092000FFF7E2FFF1E7BDE870402CF0B7BA00BF77
:10093000E19B0508EB9B05080246024902482CF0A2
:10094000E7BB00BFDE9B0508801305082DE9FF41CA
:10095000054680240A4615F8011B684601312CF033
:1009600052FA009E254FDFF89880013E019B9E427F
:1009700005D868462CF07CFA04B0BDE8F08100236D
:10098000184619461A4695F800C0520014EA0C0F92
:1009900014BF4FF0010C4FF0000C64084CEA020247
:1009A00004BF8024013501318242C9B205D317F852
:1009B00001C00CEB40006344E5E71B1A4244D15CE4
:1009C000012917D10B2300202A784000144214BFBC
:1009D00001220022640804BF80240135013B40EA63
:1009E0000200F1D101302CF09CFE014668462CF04B
:1009F0009DFABBE76846FFF777FFB7E70E9E05084D
:100A0000689D050808B5024825F0A3FD002008BD33
:100A10001B9E050838B5FFF7C5FC044620B90D48F4
:100A200025F097FD022038BD2AF04BFC20B90A487A
:100A300025F08FFD0420F6E7084D2B782BB92046D2
:100A40002AF075FC08B90648F2E7012300202B7054
:100A5000E9E700BF2E9E0508409E05084E3F002096
:100A6000539E0508F8B514460E461F46FFF79AFC3C
:100A700005460420FFF73EFE3B4622463146284607
:100A800033F088FBD5F8CC30A34207D134B14FF412
:100A90000072314605F580703BF0F8FDD5F8BC30AA
:100AA0000020A3429EBF0122014B1A70F8BD00BF77
:100AB0004D3F002038B50C461546FFF773FC022C5D
:100AC00003D0052C07D0012C15D12A46214614F05D
:100AD0008FFB002038BD2A4600210A4C14F088FB09
:100AE0000420FFF70FFE2378002BF2D0FFF718FE4B
:100AF00000232370EDE70448214625F02AFD6FF01E
:100B00008500E7E74D3F0020639E050808B5F3F731
:100B1000BBFF30B1BDE808400121024A024826F07F
:100B2000DBB808BD809E05084CCE040838B50446E5
:100B30000D4626F09CFB90B12B7843B92046F3F785
:100B40005DFF20B10121064A064826F0C5F82B7842
:100B5000012B04D12046BDE83840FFF7D7BF38BD90
:100B6000A19E05084CCE040837B5844825F0F1FC59
:100B7000834825F0EEFC8349834826F0D8FB0346E2
:100B800038B1824A0121824803B0BDE8304026F0E6
:100B9000ACB880497C4826F0CAFB034608B17E4ABF
:100BA000F0E77E49784826F0C2FB034608B17C4A4C
:100BB000E8E702F021F898B90E2002F06FF802F091
:100BC00021F8D8B90E2002F077F87648F2F780FEC7
:100BD000014608B3744803B0BDE8304025F0B9BC05
:100BE0000121802012F0D8FB03460028E4D08022A7
:100BF0006E496F4802F022F86D48DEE7012180203F
:100C000012F0CAFB03460028DCD0802269496A48FA
:100C100002F014F86848D6E75B4826F0E8FA0128A5
:100C2000044640D1654825F094FC2146644A564864
:100C3000F5F7F4F838B1634A0121554803B0BDE82F
:100C4000304026F049B8604825F083FC01F0D4FF1D
:100C500048B15E49234622464B48F5F70FFA014654
:100C600008B15B48B7E701F0CDFF40B10123594916
:100C70001A464548F5F702FA01460028F1D101234A
:100C800055491A464048F5F7F9F9014608B1534865
:100C9000A1E7534825F05DFC01210223EF223A48E9
:100CA000009126F0ABFA4F4825F053FC00214E4A44
:100CB0003548F5F7B3F8044608B14C4ABCE701F0F3
:100CC0009BFF78B14A4825F044FC012322463F4966
:100CD0002D48F5F7D3F928B1464803B0BDE83040B8
:100CE00025F037BC01F08EFF50B1414825F031FCB2
:100CF0000123002237492448F5F7C0F90028EBD139
:100D00000123002234492048F5F7B8F9044608B118
:100D10000146BCE701250223EF22014600951A484F
:100D200026F06CFA344825F014FC2146164826F0CB
:100D300089FA324825F00DFC3149134826F075FD3B
:100D400008B1304A78E7304825F003FC0E48F3F745
:100D500017FE08B12D4A6FE72D4825F0FAFB0A4827
:100D600026F085FA38B90848F3F748FE08B1294A51
:100D700062E72948B1E703B030BD00BFC19E050856
:100D8000D39E0508EC0600200C110020EF9E0508FC
:100D90004CCE0408D40600201D9F0508BC06002088
:100DA0004F9F05084C0600207C9F0508B0CB040827
:100DB000A830002094CB0408583000209F9F0508DD
:100DC00064060020C09F0508E79F0508C78B05083B
:100DD0000DA00508A78B05085F8C050830A0050845
:100DE00055A005087AA00508780600209BA00508F4
:100DF000C2A00508E8A0050808A105081EA105086D
:100E00002D0B010834A1050858A1050863A10508A8
:100E100087A10508A19E050898A1050808B501F05D
:100E2000EBFE0028014808BF002008BDA8300020C4
:100E300038B50C46054608462AF0FCF86C60606838
:100E400029F0EDFB20B9074825F083FB012038BDD0
:100E50004FF48032217A60682AF04FFC0028F5D1E7
:100E60002872F4E711A2050838B50C460121436841
:100E7000054658681B7A994003691B6819420CBFE4
:100E8000234684F001034BB18368DB689847014631
:100E900010B1044825F05DFB6C7238BD83681B6996
:100EA000F4E700BF28A2050838B543680129094ABC
:100EB00004460D4618BF4FF40032197A58682AF0DC
:100EC0001CFC014620B1044825F043FB012038BD3D
:100ED000A572FCE70600020040A2050808B5FEF76F
:100EE00023FD10B9FFF73AFC70B108BD0D4A9342DB
:100EF00003D1BDE808402BF067B80B4A9342F4D108
:100F0000BDE8084000F058BD08480368002BECD04D
:100F1000074A9342E9D0074A9342E7D1BDE8084027
:100F200034F041B850DC040828DA0408F830002016
:100F3000800E0508C44305084FF0FF3370B5204EFE
:100F4000204C336023682BB93368E3B9BDE87040A7
:100F500015F022BD1C4DAB42F6D01C4A934204D181
:100F6000204634F039F82560EEE7194A934203D160
:100F7000204600F051FDF6E7164A9342F3D1204691
:100F800001F0ACF8EFE7144C2368002BDED00E4DD7
:100F9000AB42DBD0114A934204D120462AF0F1FC47
:100FA0002560D3E70E4A934203D1204601F010FAA0
:100FB000F6E70C4A9342F3D1204601F019FDEFE722
:100FC00004070020F8300020800E0508C4430508FF
:100FD00028DA040850DC040838380020C8DB04088C
:100FE000CCDD04081CE00408F8B5334C334E23680C
:100FF0000BB1B3420DD1266031480368002B59D0A4
:10100000B34257D02F4A934246D1BDE8F84016F07C
:1010100099BF2D4A934216D16568A54203D304F1C6
:1010200098039D42E8D928460BF0D8FE0028E3D06B
:10103000264B6C22294618463BF028FB6060284668
:1010400034F081F8D8E7224A93421ED16568A54260
:1010500003D304F198039D42CED928460BF0BEFE7F
:101060000028C9D0194A2B46944605F1200E174690
:1010700018685968083303C773453A46F7D12846BC
:10108000C4F804C034F0A0F9B6E7124A9342B3D1D1
:1010900020462BF020FAAFE70F4A934203D1BDE878
:1010A000F84000F0E5BC0D4A934203D1BDE8F8409A
:1010B00001F026B8F8BD00BF38380020800E0508C2
:1010C000F8300020C4430508C8DB0408403800207D
:1010D000CCDD04081CE0040828DA040850DC04080D
:1010E00008B5144803681BB9134803684BB908BD19
:1010F000124A9342F8D0124A9342F5D12BF07EFA6D
:10110000F2E70E4A9342F2D00E4A934203D1BDE871
:10111000084033F070BF0C4A934203D1BDE8084049
:101120002AF06BBF094A9342E1D1BDE808402AF09A
:10113000BEBB00BF38380020F8300020800E050804
:101140001CE00408C443050850DC040828DA04083D
:1011500010B5084B084C1B68A34200D043B9074B9D
:10116000B422002118463BF0B8FA40F8044D10BDF7
:101170000020FCE7F8300020800E0508FC3000203D
:1011800008B5FFF7E5FF10B9014803F0B7F908BD4E
:1011900081E7050810B5084B084C1B680BB1A3424A
:1011A00008D1074B9422002118463BF096FA40F8EC
:1011B000044D10BD0020FCE738380020800E0508E3
:1011C0003C38002008B5FFF7E5FF10B9014803F0EF
:1011D00095F908BD87E70508094B1B685A1C0DD017
:1011E000002B0BDCB8225343064A9818D358064A02
:1011F000934203D0002B08BF0E2070470E2070478B
:1012000004070020F8300020800E05080E2807B5DE
:1012100013D00E4A9042136803D10D4A934200D076
:1012200093B90AF0A3F8C388E922009340F215119C
:101230004FF4AC73074803F09DF94FF0FF33064AB3
:10124000136003B05DF804FB0023F8E7F8300020DA
:10125000800E05084EEF050804070020074A1368B2
:10126000013304D1064B07491B688B4200D17047FC
:10127000002BFCD000231360704700BF0407002040
:10128000F8300020800E05082DE9F04F04461F4677
:101290004FF0000885B0CDE9021200F15009B845C1
:1012A00002D305B0BDE8F08F039B03EB080694F86A
:1012B000B530757896F901B0002B37D0B57806F1C6
:1012C000030A484618F0EEF9A8B301230093002161
:1012D000334694F8B620206DD4F860C0E0470095FE
:1012E0005346012194F8B620206DD4F860C0E04741
:1012F000484634F05FFBBBF1000F23DB00202BF0EE
:101300004EFC029B3BB1D4F88430164A934202D083
:1013100020462AF05BFAFEF707FB0028C1D194F8BB
:10132000B5304544DBB905F10208B8E706F1020A19
:1013300005F07F05C5E7FEF7F7FA0028C5D1FEF7EF
:1013400065FBBEE76B1C94F8B520DDB256FA83F35B
:1013500013445878FF2808BF4FF4FA70CFE705F11F
:1013600003089CE7800E0508F0B54B6B05460C465C
:101370008BB0002B00F0C980012380F84030486B0F
:1013800035F0A8F885F83C00636B002B00F0C080B6
:10139000A36B002B00F0BC804FF48073A5F84030A5
:1013A000A06B35F097F885F83D00B4F85630002B67
:1013B00014BF0123002385F8B43094F8573018BFC8
:1013C000042185F8423094F8563085F8433094F87B
:1013D00055600CBF01230026626B0CBF19463346D3
:1013E0000AB9A26B32B1228EB2F5807F02BF00260D
:1013F0000221334601220027CDE90422CDE9022251
:10140000CDE9001305F10800638C228BE18A34F0EA
:10141000A6FD94F859300897099394F8543005F1D3
:101420005000CDE90673638D0593238D0493E38CFF
:101430000393A38C0293B4F920300193B4F91E30C6
:101440000093628BA38B216818F0A4F8A38D324916
:10145000A5F8AA3094F82E3085F8B030238EA5F880
:10146000AC3094F8323085F8B130606CEFF7C0FCE6
:10147000EFF7C0FEA5F8A80094F84C3085F8B270DC
:1014800085F8AF30206D2449EFF7B2FCEFF7B2FEDC
:10149000C5F8900094F8543085F8B36085F8B630FC
:1014A00063681D49C5F894302389A5F8A030E06829
:1014B000EFF79EFCEFF79EFEA5F8A6002369C5F89E
:1014C0009830A38AA5F8A230E36BC5F89C30B4F835
:1014D0004030A5F8A430114BC5F8843094F858304A
:1014E00085F8B530A36C4BB128460D4B40F8843FCE
:1014F000A16CFFF79DFCA06C29F09AFD28460949D4
:101500000BB0BDE8F0402AF0A6B980F840303BE7C8
:10151000002385F8413048E700007A44800E050832
:10152000D84805085C09002010B50B680446C0F8CF
:1015300094304B680549A0F8A0301046EFF758FCEE
:10154000EFF758FEC4F8900010BD00BF00007A44C9
:1015500010B5038F04465A2B02D0B3F5877F19D1FB
:101560005A2902D0B1F5877F19D104F1080034F06F
:10157000B5FC0E4B9C4205D115F00EFAE18EA08E03
:1015800015F0ACF8A06878B104F11801BDE810407E
:1015900034F010B95A2902D0B1F5877FE5D1A38E76
:1015A000E28EE386A286E0E710BD00BFF83000209F
:1015B0002DE9F04F97B090F8B230044602AFE3B196
:1015C000D0F88420B14B9A4217D184302AF0B1F878
:1015D00094F8AF30834204D100205437BD46BDE8B3
:1015E000F08FFEF725FF00212046B4F8A230D4F892
:1015F000982084F8B210FFF747FEA368002B00F094
:10160000BF8120462AF030F90028E5D104F1500AC4
:10161000504634F0C4F90028DED094F84810002970
:1016200000F09A800023236304F12803FB6294F8FE
:10163000B430002B40F0A180FEF776F978610028E5
:10164000CAD120462AF0D4F804F1080B5846F96AAA
:1016500007F13802C7F810D034F01FFD002800F061
:10166000848107F1380034F07CFE202594F83A306C
:10167000064607F13800B5FBF3F534F077FE8146F6
:1016800007F1380034F072FEB0EBC51F4FEAC51801
:1016900000F2CA8001233B6280231FFA89F09B007D
:1016A0004009BB610130073323F007037863ADEBDA
:1016B000030D7B6B0DF108089B00073323F0070334
:1016C000ADEB030D02ABBB62B4F8AC300025B3F553
:1016D000807F14BF02230123BB60BB694344FB60CE
:1016E00007F1380034F03DFEB4F87A307862B3F593
:1016F000807F05D05946504607F1380234F05DF935
:10170000B4F8AA3087F833301DB1B4F8AC3087F89C
:101710003330504617F0C6FF002800F02681012321
:1017200094F8B6200093002107F13303206DD4F81C
:1017300060C0E047504634F03DF900239946FB6114
:10174000BB8B3A6A9A4200F2A380BA686B1C9A4239
:101750004FF00105C4D808E1A068002800F010810E
:1017600017F0C6FEF862002800F00A81B4F87A305B
:10177000B3F5807F7FF45BAF54E7204604F10806A1
:101780002AF036F83046C7F828D034F04BFC05462E
:10179000304634F049FCC5F34F05EB1D23F0070339
:1017A000ADEB030D0DF108092A4677218046484626
:1017B0003AF093FFB4F8AA30504687F8443017F057
:1017C00071FF834688B12046D7F828D02AF02FF839
:1017D00094F8B230002B3FF42FAFFEF7A5F80028A5
:1017E0007FF42AAFFEF712F9F2E70123014694F8DD
:1017F000B6200093266E07F14403206DB047504693
:1018000034F0D8F81FFA8BF39845DCD9504617F01E
:1018100049FF0BF1010B0028D5D094F8B6200095B4
:101820004B460121266EE8E707F1380034F094FDBD
:10183000B8FBF0F0002808BF012086B207F138009D
:1018400034F08FFDB0FBF6F083B207F138003B6255
:1018500034F087FDB0FBF6F303FB160080B218B13D
:101860003B6A01339BB23B6207F1380034F074FDF0
:1018700016FB00F080B2B0FBF5F293B205FB12024A
:10188000002A3FF40CAF01339BB208E7D8480508A3
:101890007B69786A7A8FFB643B8F8642A7F8443075
:1018A00002EB090388BF7A6A9BB298BF9219A7F826
:1018B000463095BF4A449B1813B21BB2A7F84A3072
:1018C0007B6AB7F93C109B1B9BB2A7F8481007F145
:1018D00044007B6234F04AFD082294F83A3000213B
:1018E000B2FBF3F3B0FBF3F37A6BB86A92007B6060
:1018F0003AF0F3FE00214046BA693AF0EEFE94F861
:10190000B43013B940F20713E387D5B194F8B3307C
:1019100063B1062384F83E3043465846BA6A07F15D
:10192000440134F0ADFB94F8B13013E094F840205A
:1019300012B184F83F30EFE7B4F84230002BF2D018
:10194000EAE743465846BA6A07F1440134F098FB87
:1019500094F8B030B3B9504617F0A4FEFB69B14417
:101960000133FB611FFA89F9A8B9FB6AD7F810D0D7
:101970009B68FB62002B7FF467AE204629F057FF7F
:1019800001202AE64346FA689342E4D01A68D2431B
:1019900043F8042BF7E7BB8894F8B62000930121A5
:1019A0004346206DD4F860C0E047504634F002F85A
:1019B000FEF72CF8C4E600BF10B590F8B23004462C
:1019C0003BB3D0F88420134B9A4214D1843029F0D1
:1019D000B0FE94F8AF3083421BD0FEF729FD002102
:1019E00084F8B2102046B4F8A230D4F89820BDE8AC
:1019F0001040FFF749BC29F0B8FCD4E90432C01A02
:101A0000B4F8A83061EB020183424FF000038B4130
:101A1000E3D310BDD848050810B590F8B23004469D
:101A200093B1D0F88420104B9A4201D029F0CEFE19
:101A3000FEF7FEFC00212046B4F8A230D4F898202E
:101A400084F8B210FFF720FC04F1080034F00CFB1E
:101A5000D4F88420054B9A4205D104F18400BDE8F6
:101A6000104029F05BBE10BD800E0508D84805085F
:101A700010B504490446083034F0A6FA012384F86E
:101A8000483010BD5C09002010B50B4C0B4B226890
:101A90009A420ED1A2680A4B9A420AD1204629F0F6
:101AA000E3FE28B92046FFF783FD80F00100C0B2B5
:101AB00010BD0020FCE700BFF830002028DA040841
:101AC0005C09002008B5014802F010FD18EE050879
:101AD00010B504492CF090FF04460AF00BFF204695
:101AE00010BD00BF28DA0408F0B50C4689B00646E0
:101AF00054F8040B1746FFF7EBFF03AB01930C4BB5
:101B000005463A4621460093701E022304F024FC49
:101B100005A90522039809F0D5FF049809F0D8FD1E
:101B200005A902462846FFF7FFFC0E2009B0F0BDCC
:101B300018DA040808B5FFF7CBFFFFF739FD10B935
:101B4000024802F0DBFC0E2008BD00BFACE805082F
:101B500010B5FFF7BDFF29F087FEA0B16430EEF7A6
:101B6000ADFC00220A4BEEF74DFEEEF7E3FF014617
:101B70000446EFF703FB40B924F0030040F00200F5
:101B8000A0F1FF4010BD0348FCE70348FAE700BF9F
:101B900000408F4002008080020040002DE9F04F9D
:101BA000CBB0084611461A462AAB01936A4B009304
:101BB00020232BF06EFD2A9B05220AA92B98039364
:101BC00009F080FF05220DA92C9809F07BFF4FF446
:101BD000477140982AF050FB5A22339F049097FB9C
:101BE000F2F302FB137313B15C4802F069FCFFF7D8
:101BF000C7FA05463F9809F06BFD8346429809F005
